:020000040800F2
:10000000F0FF001095EC040885E00308017001087A
:1000100031ED040831ED040831ED04080000000062
:1000200000000000000000000000000091E0030854
:100030008DE003080000000089E00308BD3C0108D2
:1000400031ED040831ED040831ED040831ED040808
:1000500031ED040831ED0408BD9A0008F99A000852
:10006000819A0008E17E0108A57E0108E1D500081B
:10007000D1D50008C1D50008B1D500089DD500082C
:1000800089D5000875D5000831ED040831ED040864
:1000900031ED040831ED040831ED0408697E0108F2
:1000A000511E0108DD23010831ED04089D240108DB
:1000B0001D2301085D22010891210108F9040108AE
:1000C00001050108E9040108F104010831ED040803
:1000D00031ED04086D3F0108D13E0108353E0108AD
:1000E0002D7E010831ED0408A926040831ED04082D
:1000F000211F010831ED0408F11F010861D5000836
:1001000031ED040831ED0408C120010831ED040887
:10011000993D0108FD3C010889E3010875E30108E8
:100120004DD5000839D5000825D5000811D500089F
:10013000FDD4000831ED040831ED040831ED040868
:1001400031ED040831ED040831ED0408DD15040833
:10015000E9D40008D5D40008C1D4000831ED040862
:10016000D9040108E104010831ED040831ED040867
:1001700031ED040831ED040831ED040831ED0408D7
:0801800031ED040831ED040823
:080188003CE804000100000046
:1001900010020100103200200C320020000000008C
:1001A000080700081A023C003C5200203C56002080
:1001B000000000001D9300082700040038520020B2
:1001C00078560020000000000A070008070202001D
:1001D000D05D0020145E0020000000000E07000823
:1001E00002000C00A85D0020185E00200000000046
:1001F0000000000006020C009C5D0020245E002030
:10020000000000000D92000808120900205D002087
:10021000305E0020000000006D840008F701060039
:100220001A5D00203C5E002000000000100700085E
:100230000A020A00845C0020445E002000000000E6
:100240001607000803000100A0570020505E0020A0
:10025000000000000000000014000300EC66002015
:1002600004690020000000002007000810100200B0
:1002700044680020086900200000000024070008EE
:1002800028101000346800200C69002000000000D5
:100290006129020823001000D86300201C69002097
:1002A0000000000079290208F82106002C680020CF
:1002B0002C69002000000000260700080E502001D5
:1002C000FC60002034690020000000005D7E04080E
:1002D00013000400A0640020546A00200000000005
:1002E0002C0700080101040076600020586A0020F5
:1002F0000000000000000000000104006E6000200B
:100300005C6A0020000000003007000802010300C2
:1003100069600020606A002000000000E18F010891
:100320000902010038670020646A00200000000014
:10033000340700080C106C0046620020686A002038
:1003400000000000B98F0108010205007E60002056
:10035000D46A002000000000F51F0208000205001A
:1003600058640020DC6A002000000000000000004B
:100370001B0208009C710020A085002000000000E6
:10038000C584000801200800F4830020A88500200F
:10039000000000003607000819000500A4840020B2
:1003A000B0850020000000003E07000837001E0056
:1003B0007C840020B885002000000000440700086D
:1003C0001E000500786F0020D88500200000000086
:1003D000620700081B00F400846C0020E085002008
:1003E00000000000E1B702080E020200D8760020EB
:1003F000D486002000000000680700082F001100CC
:100400003C850020D8860020000000006A07000814
:100410000510060080850020EC860020000000000A
:100420007C070008F5317000FC6B0020F48600208A
:1004300000000000D5DF020826000E0074870020AF
:100440006487002000000000959F02080B20100028
:100450006E6C0020A88700200000000082070008C2
:100460001F201C00DC6B0020B8870020000000006B
:100470009207000805020400E4710020D4870020E0
:1004800000000000AE0700081600080044880020A5
:100490004C88002000000000B2070008031233005F
:1004A000988D00205292002000000000BC07000838
:1004B00025009600CC8D0020AC91002000000000AB
:1004C00000000000F6210C00CC8F002028910020B5
:1004D00000000000F007000815007000D88F002011
:1004E000B890002000000000000000002A0060001A
:1004F000D48B00205890002000000000357E0408B6
:100500002C001000489000204292002000000000C3
:10051000297403082B002400E08E0020859200201F
:1005200000000000F973030829107800688E00208D
:1005300034910020000000000000000003010A00C8
:100540005CA50020F4A5002000000000FC070008C6
:10055000130203001C9B002000A6002000000000E6
:100560000608000804008000F0E30020A8E4002052
:1005700000000000000000000D0044006CE30020BB
:1005800028E5002000000000F1130308FD0124000D
:100590009CDA00206CE500200000000059070108EB
:1005A00018202C006CDA002090E5002000000000EC
:1005B000E593000806101800C4CD0020BCE500201B
:1005C00000000000B97E0408FB010100C0CD00203E
:1005D000D4E5002000000000B9930008FC010900E8
:1005E0008CCC0020D8E5002000000000C993000852
:1005F0000A40200064CC0020E4E500200000000058
:100600000A0800083400100094CB002004E6002003
:10061000000000008D7E0408110208006CCB002051
:1006200014E60020000000002A080008121204004E
:1006300064CB00201CE60020000000003208000807
:1006400012200D0054CB002020E600200000000006
:1006500036080008FF01080040BF002030E60020F7
:1006600000000000D1D10008F9010400D4BE002030
:1006700038E6002000000000D1070108180202003F
:10068000DCB800203CE60020000000000000000074
:1006900017020B00D0B8002040E600200000000048
:1006A00029840008FA010200ACB800204CE60020C2
:1006B00000000000C58500080202030058B60020B3
:1006C00050E6002000000000000000000C020300C3
:1006D00014B6002054E60020000000001984000831
:1006E000FE01090084B8002058E600200000000048
:1006F000A58400081A000E0080FA0020B0FB00203C
:0807000000000000440800089D
:10070800000020030000013C3D0100000000000043
:100718004A01B400D60100000300000000050401EE
:10072800F401190048040430B30000001300E80382
:100738006400040A000100002801000020003200C3
:10074800C800D0079600140032002800B004400604
:100758000005500014000F0008010000010000000F
:100768000000000000000000000000000000000081
:10077800000000002000020100002B21231E64015C
:100788000100000001000A0129000000000000012A
:100798000000000500000102030000000000000046
:1007A80000000000000000000000C409000019015A
:1007B80028280000000000000000000000000000E1
:1007C8000000000000000000000000000000000021
:1007D8000000000000000000000000000000000011
:1007E80000000000000001000000000001000000FF
:1007F80002020000040101006C1600000000000065
:100808000000003001000000000064002C0100001E
:100818000000000000000000020000019E077D00AB
:1008280046320000000001010101FFFFFFFF000048
:1008380000010000054D4B46340000007E05EA0526
:0A084800B4053200E803D0070000F9
:100852001A03000000000000000000000000000079
:100862000000000000000000000000000403090472
:10087200120100020000004083042057000201021E
:1008820003010000E1990008218500084199000850
:10089200058500089D99000851990008F584000813
:1008A200DC00002071B900080D85000809850008E8
:1008B2000185000849940008FD840008F9840008B5
:1008C200CC0805081511040825D70308FD0F0408F4
:1008D20000000000000000004D0504087505040832
:1008E20000000000000000000000000085D50308A1
:1008F200B9850008AD8500083D9A0008599A00089C
:1009020065850008219A0008059A00080100000088
:10091200500100000700000002000000000000007B
:100922000000000001020304060708090080020219
:100932001F00000053544D202020202050726F646D
:10094200757420202020202020202020302E3031BD
:10095200685E0C00010102FFFF00000001000000C0
:100962000000803F000000000000000000000000C6
:10097200FF00000000000000045E002008000000EC
:1009820000000000F45D00200800000014160508B5
:1009920005080400000000009C1F0508384A0508ED
:1009A200881F05080000000000000000401605082E
:1009B20005080A00000000009C1F0508384A0508C7
:1009C200681E05080000000000000000E0010101AF
:1009D20001000000E521020800000000F8020020EA
:1009E200046D050800000000000000000000000087
:1009F20000000000A46F05080000000000000000D5
:100A02007903002004000000506B05080D0000006F
:100A120035420208641D0020000000008C640508B5
:100A22000D0000005D420208581D00200000000079
:100A32000C66050808000000000000004C1D0020A4
:100A420004000000F86405080D0000009922020865
:100A5200401D002000000000BC65050803000000E6
:100A6200AD440208341D002000000000146D05088A
:100A720003000000AD440208281D00200000000011
:100A8200C86005080100000000000000000000002E
:100A920000000000000000000E0000000000000046
:100AA2000000000000000000046D050800000000C6
:100AB200000000000000000000000000A46F050814
:100AC2000000000000000000790300200400000084
:100AD200FC6A050803000000292E02081C1D0020E4
:100AE20008000000F86405080D00000099220208C1
:100AF200401D002000000000BC6505080300000046
:100B0200AD440208341D002000000000146D0508E9
:100B120003000000AD440208281D00200000000070
:100B2200C86005080100000000000000000000008D
:100B320000000000000000000E00000000000000A5
:100B420000000000000000001C6D0508000000000D
:100B5200000000000000000000000000A46F050873
:100B620000000000000000007903002004000000E3
:100B7200046B050803000000AD440208701D00204C
:100B820000000000C860050801000000000000002D
:100B92000000000000000000000000000E00000045
:100BA2000000000000000000000000002070002093
:100BB200702D720000010101000800000000000019
:100BC20000000000D8180020012D202D2D202D2DF1
:100BD2002D2D202D2D2D0000000000000000000012
:100BE2000000000000000000FFFFFFFFFA0000000D
:100BF20001000000010000000100000098600508EB
:100C0200A0600508C06005080000000000000000A8
:100C12000000000000000000795A050804000000EE
:100C2200FD3F02080000000000000000C860050847
:100C320001000000000000000000000000000000B1
:100C4200000000000E000000000000000000000094
:100C52000000000090E400200100C4090000000030
:100C62008EE400200100C409000000008CE4002092
:100C72000100C409000000008AE400200100C40948
:100C82000000000086E400200100C409000000000A
:100C920088E400200100C4090000000084E4002070
:100CA2000100C4090000000082E400200100C40920
:100CB20000000000906000200100C8000100000058
:100CC2008E60002032003075320000008C600020FF
:100CD200055A05008960002000FF01008B6000209A
:100CE20001000000AC030020876000200200000029
:100CF2004C2305088860002000FF01008A60002064
:100D020001000000AC030020866000200200000009
:100D12004C2305087C60002080C1803E0500000055
:100D22007A60002080C1803E0500000074600020CF
:100D320080C1803E050000007260002080C1803EBC
:100D4200050000006C60002000FF010068600020C8
:100D52000A3201006760002004000000481E0508F6
:100D620066600020020000005C1E05080000000012
:100D720000000000B4030020A0A500209CFF2C016D
:100D8200000000007E0100200A000000681E050825
:100D92005C600020E0150C170000000080010020BC
:100DA20008000000384A05087F0100200500000005
:100DB2009C1F05085E60002002000000801E0508DE
:100DC200CC6200200100FF7F01000000CB62002006
:100DD200020000008C1E0508EF60002003000000E6
:100DE2009C1E0508EE600020030000009C1E050802
:100DF200266200200000F4010100000024620020AD
:100E02000000F40101000000226200200000F40151
:100E120001000000206200200000F4010100000037
:100E22001E6200200000803E010000001C620020C3
:100E32000000803E0100000042620020E803D0076B
:100E42000A00000040620020006401000A00000065
:100E52003562002000640100346200200064010059
:100E62003C620020006401000A0000003B62002096
:100E7200006401000A0000003A62002000640100E0
:100E82000A0000003F620020006401000A00000026
:100E92003E620020006401000A0000003D62002062
:100EA200006401000A0000003962002000FF010016
:100EB2000A0000003862002000FF01000A00000062
:100EC2003762002000FF01000A000000F8600020E5
:100ED2000000F40101000000F66000200000F401AF
:100EE20001000000F46000200000F4010100000095
:100EF200F26000200000F40101000000F060002018
:100F02000000F401010000003262002000640100D0
:100F1200306200201400E803010000002E6200206D
:100F2200E80330750A0000002C62002000C80100AE
:100F32002B62002000C801002A62002000C80100C4
:100F420029620020006401000A000000C062002043
:100F52000000D00701000000BB62002000C80100B1
:100F6200BA62002000C80100B962002000C8010076
:100F7200BE6200200000D00701000000B86200201D
:100F820000C80100B762002000C80100B66200205C
:100F920000C80100BC6200200000D0070100000070
:100FA200B562002000C80100B462002000C8010040
:100FB200B362002000C80100F860050800000000CC
:100FC20000000000000000000000000008610508A9
:100FD2000900000000000000580400200400000086
:100FE2001061050809000000000000004C04002008
:100FF20004000000D068050809000000000000009D
:10100200400400200400000074710508090000007B
:1010120000000000340400200400000018610508EC
:101022000900000000000000280400200400000065
:101032002061050809000000000000001C040020D7
:1010420004000000286105080900000000000000FB
:1010520010040020040000003061050809000000AF
:10106200000000000404002004000000C86005081D
:10107200010000000000000000000000000000006D
:10108200000000000E000000000000000000000050
:10109200000000006C630508000000000000000072
:1010A2000000000000000000FCA10508070000008D
:1010B200000000007C040020000000007C630508A2
:1010C2000800000000000000700400200000000082
:1010D2008863050808000000000000006404002086
:1010E20000000000C86005080100000000000000C8
:1010F2000000000000000000000000000E000000E0
:1011020000000000000000000000000090630508DD
:1011120000000000000000000000000000000000CD
:10112200A06305080D00000000000000B8040020C4
:1011320000000000A86305080D0000000000000088
:10114200AC04002000000000B063050807000000A6
:1011520000000000A404002000000000B86305089D
:101162000D000000000000009804002000000000B4
:10117200C06305080D000000000000008C04002080
:1011820000000000C863050807000000000000001E
:101192008404002000000000C8600508010000006F
:1011A200000000000000000000000000000000003D
:1011B2000E0000000000000000000000000000001F
:1011C200D0630508000000000000000000000000DD
:1011D20000000000FCA105080C0000000000000057
:1011E2009260002000000000E46305080C0000008B
:1011F200000000009460002000000000F463050875
:101202000C00000000000000CA6000200000000086
:10121200046405080C00000000000000BE6000200D
:1012220000000000186405080C0000000000000027
:101232009660002000000000246405080C000000F5
:101242000000000098600020000000002C640508E7
:101252000C000000000000009A6000200000000066
:10126200406405080C000000000000009C600020A3
:1012720000000000486405080C00000000000000A7
:101282009E60002000000000506405080C00000071
:1012920000000000DC600020000000006864050817
:1012A2000C00000000000000A06000200000000010
:1012B200746405080C00000000000000A260002019
:1012C200000000007C6405080C0000000000000023
:1012D200A460002000000000886405080C000000E3
:1012E20000000000A66000200000000094640508D1
:1012F2000C00000000000000A860002000000000B8
:10130200A06405080C00000000000000AA60002094
:1013120000000000AC6405080C00000000000000A2
:10132200AC60002000000000B86405080C0000005A
:1013320000000000AE60002000000000C464050848
:101342000C00000000000000C2600020000000004D
:10135200CC6405080C00000000000000C060002002
:1013620000000000D46405080C000000000000002A
:10137200CE60002000000000E06405080C000000C0
:1013820000000000D060002000000000EC640508AE
:101392000C00000000000000D660002000000000E9
:1013A200E06105080C00000000000000B0600020B1
:1013B20000000000F86405080C00000000000000B6
:1013C200B860002000000000006505080C00000065
:1013D20000000000B2600020000000000C6505085B
:1013E2000C00000000000000B460002000000000BB
:1013F200186505080C00000000000000B66000201F
:1014020000000000206505080C000000000000003C
:10141200BA600020000000002C6505080C000000E6
:1014220000000000C46000200000000034650508D0
:101432000C00000000000000BC6000200000000062
:10144200406505080C00000000000000CC60002090
:10145200000000004C6505080C00000000000000C0
:10146200C660002000000000546505080C00000062
:1014720000000000C8600020000000005C65050854
:101482000C00000000000000D260002000000000FC
:10149200646505080C00000000000000D460002014
:1014A200000000006C6505080C0000000000000050
:1014B200E660002000000000C8600508010000008E
:1014C200000000000000000000000000000000001A
:1014D2000E000000000000000000000000000000FC
:1014E2007465050800000000000000000000000014
:1014F20000000000806505080D00000000000000EB
:101502001005002000000000886505080D0000009D
:10151200000000000405002000000000906505089E
:101522000700000000000000FC0400200000000092
:101532009C6505080700000000000000F40400207C
:1015420000000000A8650508090000000000000076
:10155200E804002000000000B4650508090000004E
:1015620000000000DC04002000000000C065050847
:101572000900000000000000D0040020000000006C
:10158200D06505080900000000000000C404002026
:1015920000000000C8600508010000000000000013
:1015A2000000000000000000000000000E0000002B
:1015B200000000000000000000000000E4650508D3
:1015C2000000000000000000000000000000000019
:1015D200F46505080500000000000000ED60002031
:1015E20000000000C86005080100000000000000C3
:1015F2000000000000000000000000000E000000DB
:10160200000000000000000000000000FC6505086A
:1016120000000000000000000000000000000000C8
:10162200A46F050800000000000000003C25002017
:1016320004000000086605080D0000006140020871
:101642006405002000000000506B05080D0000003A
:101652009D21020858050020000000008C64050846
:101662000D000000812102084C050020000000004E
:101672000C6605080800000000000000400500207C
:1016820004000000F86405080D000000C9200208EB
:10169200340500200000000014660508090000005F
:1016A200000000002805002004000000BC650508B9
:1016B20003000000AD4402081C05002000000000E9
:1016C200C8600508010000000000000000000000E2
:1016D20000000000000000000E00000000000000FA
:1016E20000000000000000001C6605080000000069
:1016F2000000000000000000000000002C66050849
:101702000D000000000000007C0500200000000029
:10171200346605080A00000000000000FD64002095
:1017220000000000406605080A00000000000000FA
:101732000565002000000000486605080A00000058
:10174200000000000D650020000000005066050842
:1017520008000000000000007005002000000000EA
:101762005866050804000000CD460208000000008B
:1017720000000000C8600508010000000000000031
:101782000000000000000000000000000E00000049
:101792000000000000000000000000006466050870
:1017A2000000000000000000000000000000000037
:1017B200786605080D000000000000009405002076
:1017C200000000008866050804000000D9420208F3
:1017D2000000000000000000906605080D000000F7
:1017E200000000008805002000000000A466050833
:1017F20004000000B54202080000000000000000E2
:10180200C8600508010000000000000000000000A0
:1018120000000000000000000E00000000000000B8
:101822000000000000000000AC6605080000000097
:10183200000000000000000000000000C066050873
:101842000800000000000000DC050020000000008D
:10185200CC6605080800000000000000D00500204A
:1018620000000000D8660508080000000000000023
:10187200C405002000000000E4660508080000001E
:1018820000000000B805002000000000F066050816
:101892000800000000000000AC050020000000006D
:1018A200FC6605080800000000000000A0050020FA
:1018B20000000000C86005080100000000000000F0
:1018C2000000000000000000000000000E00000008
:1018D200000000000000000000000000086705088A
:1018E20000000000000000005F0300200000000074
:1018F200146705080B0000000000000070060020BD
:1019020000000000206705080B0000000000000036
:1019120064060020000000002C6705080B00000090
:10192200000000005806002000000000386705088B
:101932000B000000000000004C0600200000000028
:10194200446705080B00000000000000400600206C
:1019520000000000506705080B00000000000000B6
:1019620034060020000000005C6705080B00000040
:10197200000000002806002000000000686705083B
:101982000B000000000000001C0600200000000008
:10199200746705080B00000000000000100600201C
:1019A200000000008067050807000000000000003A
:1019B20008060020000000008867050807000000F4
:1019C20000000000000600200000000094670508E7
:1019D2000B00000000000000F405002000000000E1
:1019E200A06705080800000000000000E8050020CC
:1019F20000000000C86005080100000000000000AF
:101A02000000000000000000000000000E000000C6
:101A1200000000000000000000000000AC670508A4
:101A220000000000000000000000000000000000B4
:101A3200C06705080800000000000000AC06002096
:101A420000000000CC67050808000000000000004C
:101A5200A006002000000000D8670508080000006A
:101A6200000000009406002000000000E467050862
:101A720008000000000000008806002000000000AE
:101A8200F067050808000000000000007C06002046
:101A920000000000C860050801000000000000000E
:101AA2000000000000000000000000000E00000026
:101AB200000000000000000000000000F8670508B8
:101AC20000000000000000005C0300200000000095
:101AD200086805080B00000000000000F006002066
:101AE2000000000014680508070000000000000064
:101AF200E80600200000000020680508070000003A
:101B020000000000E0060020000000002C6805082C
:101B12000700000000000000D806002000000000BE
:101B2200386805080800000000000000CC0600200C
:101B320000000000406805080800000000000000E6
:101B4200C0060020000000004868050807000000E9
:101B520000000000B806002000000000C860050870
:101B62000100000000000000000000000000000072
:101B7200000000000E000000000000000000000055
:101B8200000000005468050800000000000000008A
:101B92005C030020000000006068050807000000E8
:101BA20000000000600700200000000068680508CF
:101BB200070000000000000058070020000000009D
:101BC20070680508070000000000000050070020B0
:101BD200000000007868050808000000000000000E
:101BE200440700200000000080680508070000008C
:101BF200000000003C070020000000008868050883
:101C02000700000000000000340700200000000070
:101C12009068050807000000000000002C07002063
:101C2200000000009868050808000000000000009D
:101C32002007002000000000A0680508070000003F
:101C4200000000001807002000000000A868050836
:101C52000700000000000000100700200000000044
:101C6200B068050807000000000000000807002017
:101C720000000000B868050808000000000000002D
:101C8200FC06002000000000C860050801000000FA
:101C92000000000000000000000000000000000042
:101CA2000E00000000000000000000000000000024
:101CB200000000000D25020868070020EB600020EC
:101CC2002B000000AC1E0508EA60002000C80100DD
:101CD200E8600020E803D007010000004D415445B0
:101CE2004B463430350000008560002000030100BF
:101CF2008460002000030100552402082D240208FC
:101D020044080020E92302089D230208BC080020A1
:101D1200952402087D240208700900200923020884
:101D2200BD220208900C00202325020885420208E9
:101D32006C0D00200921020800000000BC0D0020EB
:101D4200A9460208C1270208980E00204925020868
:101D5200000000004C0F002001260208CD250208D9
:101D6200D80F002091260208DD2602088C100020E0
:101D72003362002001060100912502085D25020858
:101D8200CC11002035260208FD4202086C12002008
:101D92000D2702085943020834130020286200204C
:101DA20001030100C06805080000000000000000F7
:101DB2000000000000000000CC68050808000000D8
:101DC200000000008014002000000000D468050814
:101DD200070000000000000078140020000000004E
:101DE200E46805080D000000000000006C140020EB
:101DF20000000000F068050803000000AD4402087E
:101E02006014002000000000C86005080100000006
:101E120000000000000000000000000000000000C0
:101E22000E000000000000000000000000000000A2
:101E3200F868050800000000000000000000000033
:101E420000000000086905080A0000000000000008
:101E52001069050800000000186905080A00000062
:101E62000000000075580508000000002069050800
:101E72000A00000000000000C26200200000000012
:101E8200286905080A000000000000008C140020E8
:101E920000000000C860050801000000000000000A
:101EA2000000000000000000000000000E00000022
:101EB200000000000000000000000000306905087A
:101EC2000000000000000000000000000000000010
:101ED2003C69050803000000AD440208C01400205C
:101EE200000000004869050803000000AD44020834
:101EF200B41400200000000050690508030000002F
:101F0200AD440208A814002000000000586905082A
:101F120005000000000000008360002000000000B7
:101F2200606905080700000000000000A0140020FE
:101F3200000000006C6905080700000000000000B6
:101F42009814002000000000C8600508010000008D
:101F5200000000000000000000000000000000007F
:101F62000E00000000000000000000000000000061
:101F72007869050800000000000000000000000071
:101F8200000000008C69050803000000AD4402084F
:101F9200F01400200000000098690508030000000A
:101FA200AD4402088401002000000000A069050879
:101FB20003000000AD440208E41400200000000009
:101FC200A869050803000000AD440208D8140020E7
:101FD20000000000F864050803000000AD44020898
:101FE200CC14002000000000C860050801000000B9
:101FF20000000000000000000000000000000000DF
:102002000E000000000000000000000000000000C0
:10201200B469050800000000000000000000000094
:1020220000000000C469050807000000B54302086B
:102032004C150020000000001C650508030000008C
:10204200AD4402084015002000000000D0690508D8
:1020520003000000AD440208341500200000000017
:10206200D869050803000000AD44020828150020C5
:1020720000000000E069050807000000994302081B
:102082002015002000000000B471050803000000C4
:10209200AD4402081415002000000000EC69050898
:1020A20003000000AD4402080815002000000000F3
:1020B200F869050803000000AD440208FC14002082
:1020C20000000000C86005080100000000000000D8
:1020D2000000000000000000000000000E000000F0
:1020E200000000000000000000000000DD240208E3
:1020F200AD240208541500208D27020800000000BC
:10210200E015002079230208552302086C160020EE
:1021120000000000000000002017002065270208D0
:10212200D1430208C0170020046A0508000000001D
:10213200000000000000000000000000106A050816
:1021420003000000AD440208CC180020000000008B
:10215200186A050803000000AD440208C0180020F8
:1021620000000000246A050803000000AD440208D4
:10217200B418002000000000286A050803000000CF
:10218200AD440208A818002000000000346A0508C7
:1021920003000000AD4402089C180020000000006B
:1021A2003C6A0508020000006147020800000000C6
:1021B20000000000446A05080200000061470208AE
:1021C2000100000000000000506A05080200000043
:1021D2006147020802000000000000000000000049
:1021E2000E000000000000000000000000000000DF
:1021F2006260002088136F170100000064600020F5
:1022020088136F17000000005C6A050800000000D8
:102212000000000000000000000000006C6A0508D9
:102222000800000000000000AC19002004000000BB
:10223200786A05080800000000000000A0190020CC
:1022420000000000BC650508040000008940020887
:102252000000000000000000C86005080100000046
:10226200000000000000000000000000000000006C
:102272000E0000000000000000000000000000004E
:102282006060002088136F1701000000E2A50020A3
:1022920088136F17000000004D22020800000000A2
:1022A200B81900209D640020010000005C1F050891
:1022B200E4A5002001000000681F0508DAA500203F
:1022C20002000000701F0508F2A3002000000000B9
:1022D20000000000F0A30020000000000000000049
:1022E200EEA300200000000000000000ECA300208C
:1022F2000000000000000000EAA30020000000002F
:1023020000000000E8A30020000000000000000020
:102312007825002000000000000000005F6000201F
:10232200020000007C1F0508B46A050800000000D6
:102332000000000000000000000000006C6A0508B8
:1023420008000000000000003C1A00200400000009
:10235200786A05080800000000000000301A00201A
:1023620000000000BC650508040000001D220208F0
:102372000000000000000000C86005080100000025
:10238200000000000000000000000000000000004B
:102392000E0000000000000000000000000000002D
:1023A200C46A0508000000000000000000000000F0
:1023B20000000000D46A05080D000000D94102089F
:1023C2006C1A002004000000E06A05080D000000FD
:1023D20075220208601A002004000000EC6A050859
:1023E2000D0000009D410208541A00200000000068
:1023F200F86A050803000000492E0208481A002066
:1024020008000000046B050803000000AD44020848
:10241200701D002000000000C860050801000000D7
:1024220000000000000000000000000000000000AA
:102432000E0000000000000000000000000000008C
:10244200C06005080000000000000000000000005D
:1024520000000000795A050804000000A1400208AB
:102462000000000000000000C86005080100000034
:10247200000000000000000000000000000000005A
:102482000E0000000000000000000000000000003C
:10249200586B05080000000000000000000000006A
:1024A200000000000C8805080D000000000000007C
:1024B200CC1A002004000000686B05080800000028
:1024C20000000000C01A002004000000746B050820
:1024D2000800000000000000B41A00200400000000
:1024E2007C6B05080800000000000000A81A00200C
:1024F20004000000846B05080800000000000000D2
:102502009C1A0020040000008C6B050808000000E3
:1025120000000000901A002004000000946B0508DF
:102522000800000000000000841A002004000000DF
:102532009C6B05080800000000000000781A0020CB
:1025420004000000C860050801000000000000004F
:102552000000000000000000000000000E0000006B
:102562000000000000000000000000003522020808
:1025720000000000D81A0020000000000000000047
:10258200501B00200000000000000000F01B002093
:10259200E0A5002004000000881F0508DEA5002039
:1025A200E0150C1700000000DDA500200800000067
:1025B200384A0508DCA50020050000009C1F05081C
:1025C2000000000000000000401C0020010000008C
:1025D200000001FFFF0100000000803FFF1FFF1FFE
:1025E2008487002000000000242300200400000053
:1025F200B872050860720508000000007113030834
:10260200A08601000400000000000000000000009D
:1026120000000000000000000000000000000000B8
:1026220000000000B8720508C07205080000000032
:10263200950D0108E80300000400000000000000FE
:102642000000000000000000000000000000000088
:1026520000000000000000001C650508C8720508A3
:10266200000000007D9A01087D00000006000000C5
:102672000000000000000000000000000000000058
:10268200000000000000000000000000D0720508F9
:102692000000000000000000E1320108E803000031
:1026A2000300000000000000000000000000000025
:1026B2000000000000000000000000000000000018
:1026C200D4720508000000000000000079810408AF
:1026D20010270000030000000000000000000000BE
:1026E20000000000000000000000000000000000E8
:1026F20000000000506D050800000000257003086E
:10270200417001085F760000050000000000000033
:1027120000000000000000000000000000000000B7
:102722000000000000000000E8A30508000000000F
:10273200000000001D7F01081027000001000000BA
:102742000000000000000000000000000000000087
:10275200000000000000000000000000E072050818
:102762000000000000000000F9050108E803000075
:102772000500000000000000000000000000000052
:102782000000000000000000000000000000000047
:10279200EC72050800000000000000003D0F020876
:1027A200204E0000030000000000000000000000B6
:1027B2000000000000000000000000000000000017
:1027C20000000000FC72050800000000000000008C
:1027D200290D0208204E0000030000000000000046
:1027E20000000000000000000000000000000000E7
:1027F20000000000000000000C730508000000004B
:1028020000000000250B0108400D0300030000003A
:1028120000000000000000000000000000000000B6
:102822000000000000000000000000001C7305080A
:102832000000000000000000E11F03081027000054
:102842000100000000000000000000000000000085
:102852000000000000000000000000000000000076
:102862004C6D0508000000000000000065EB020846
:10287200102700000300000000000000000000001C
:102882000000000000000000000000000000000046
:102892000000000024730508000000000000000092
:1028A200ED970208A0860100010000000000000070
:1028B2000000000000000000000000000000000016
:1028C20000000000000000002C730508000000005A
:1028D20000000000510A010850C30000010000007E
:1028E20000000000000000000000000000000000E6
:1028F200000000000000000000000000E061050888
:102902000000000000000000E1070108A8610000CB
:1029120001000000000000000000000000000000B4
:1029220000000000000000000000000000000000A5
:102932003473050800000000000000006166020810
:10294200A08601000100000000000000000000005D
:102952000000000000000000000000000000000075
:1029620000000000407305080000000000000000A5
:10297200BD400108A00F000001000000000000009F
:102982000000000000000000000000000000000045
:1029920000000000000000004C7305080000000069
:1029A20000000000DDB30208102700000100000053
:1029B2000000000000000000000000000000000015
:1029C200000000000000000000000000246A05086A
:1029D2000000000000000000010B03081A41000083
:1029E20001000000000000000000000000000000E4
:1029F20000000000000000000000000000000000D5
:102A0200A06105080000000000000000499C0208C7
:102A1200102700000100000000000000000000007C
:102A220000000000000000000000000000000000A4
:102A320000000000747205080000000000000000A1
:102A4200A16A02081A410000010000000000000013
:102A52000000000000000000000000000000000074
:102A6200000000000000000058730508000000008C
:102A72000000000045C40208400D030000000000F1
:102A82000000000000000000000000000000000044
:102A92000000000000000000000000006073050854
:102AA2000000000000000000AD130308400D030009
:102AB2000000000000000000000000000000000014
:102AC2000000000000000000000000000000000004
:102AD20068730508000000000000000039F90208D0
:102AE20050C30000030000000000000000000000CE
:102AF20000000000000000000000000000000000D4
:102B020000000000747305080000000000000000CF
:102B12009D0C020840420F0000000000000000006F
:102B220000000000000000000000000000000000A3
:102B32000000000000000000807305080000000093
:102B420000000000CD14030850C300000000000084
:102B52000000000000000000000000000000000073
:102B62000000000000000000000000000100000062
:102B7200FFFFFFFF000200051002700B9DDB030840
:102B820069D70308C109040800000000D5D503086D
:102B92007511040851DB0308F9060408000000005F
:102BA2000000000091D5030851D4030845D403085E
:102BB20015FE030831FE0308F9FD0308DDFD0308D5
:102BC200C1FD030855DB030845D7030801090408C2
:102BD20000000000A9D50308FD06040825DB030850
:102BE2005906040800000000000000009DD50308FB
:102BF200D60101FFFF000000FFFFFFFF04030904ED
:102C020012010002EF020140830456320002010267
:102C12000301000012010002020200408304405737
:102C2200000201020301000009022000010104C0A8
:102C3200320904000002080650050705810240001F
:102C4200000705010240000009026400030100C000
:102C520032090400000103000000092111010001F2
:102C62002226000705830308000A080B010202025C
:102C72000100090401000102020100052400100103
:102C820005240100020424020205240601020705AC
:102C920082030800FF09040200020A00000007057F
:102CA20001024000000705810240000009024300C2
:102CB200020100C0320904000001020201000524E1
:102CC200001001052401000104240202052406006B
:102CD20001070582030800FF09040100020A00003F
:102CE20000070501024000000705810240000000C4
:102CF200FF00000000FFFF0000000000AA550501D0
:102D02000000000005010905A101A100050109302B
:102D12000931093209330935093409400938158165
:102D2200257F750895088102C0C0000009022200B3
:102D3200010100E03209040000010301020009213F
:102D4200110100012226000705830308000A000082
:102D5200000000000102030401020304060708093F
:102D6200A1070408690E0408E509040811D603083E
:102D720035D8030821D603083DD60308E9D5030850
:102D8200D9D5030800000000000000002D202D2DE1
:102D9200202D2D2D2D202D2D2D2D00000000000089
:102DA2000000000000000000000000AA550B010016
:102DB20000AA5507010000AA550902000000AA5501
:102DC20003009F0001000000C01200000800000084
:102DD20041D403083DD4030839D403082DD4030891
:102DE20029D4030835D4030831D403080060024013
:102DF200106002400000000000000000000B000014
:102E0200000000000000000000000000006002401E
:102E1200286002400100000000000000060C0000D3
:102E220000000000000000000000000000600240FE
:102E3200406002400200000000000000100D00008F
:102E420000000000000000000000000000600240DE
:102E5200586002400300000000000000160E00004F
:102E620000000000000000000000000000600240BE
:102E7200706002400400000000000000200F00000B
:102E8200000000000000000000000000006002409E
:102E920088600240050000000000000026100000CB
:102EA200000000000000000000000000006002407E
:102EB200A060024006000000000000003011000087
:102EC200000000000000000000000000006002405E
:102ED200B86002400700000000000000362F00002A
:102EE200000000000000000000000000006402403A
:102EF20010640240000000000000000000380000E2
:102F02000000000000000000000000000064024019
:102F120028640240010000000000000006390000A1
:102F220000000000000000000000000000640240F9
:102F3200406402400200000000000000103A00005D
:102F420000000000000000000000000000640240D9
:102F5200586402400300000000000000163B00001D
:102F620000000000000000000000000000640240B9
:102F7200706402400400000000000000203C0000D9
:102F82000000000000000000000000000064024099
:102F92008864024005000000000000002644000092
:102FA2000000000000000000000000000064024079
:102FB200A06402400600000000000000304500004E
:102FC2000000000000000000000000000064024059
:102FD200B86402400700000000000000364600000E
:102FE20000000000000000000000000001000000DE
:102FF2000000803F00000000000000000000000010
:103002000000803F000000000000000000000000FF
:1030120000000000000000000000000000000000AE
:103022000000000000000000010000000000803FDE
:103032000000000000000000000000000000803FCF
:10304200F427002000000000000000000000000043
:10305200000000000000000000000000000000006E
:10306200000000000000000000000000000000005E
:10307200000000000000000000000000000000004E
:10308200000000000000000000000000000000003E
:10309200000000000000000000000000000000002E
:0830A200000000000100000025
:1080000090ED057A90ED004AD0ED066AD0ED014A78
:10801000D0ED047A90ED035AD0ED025AA4EE007A26
:10802000B0EE406AB0EE470AB0EE667AA4EE867A09
:1080300067EEC07AA5EE407AE5EE867A80ED057AA5
:10804000C0ED067A704700BFD0ED057A90ED013A99
:10805000D0ED003AD0ED064A90ED024A90ED077A55
:1080600090ED035A90ED086AD0ED045AC0ED067AFF
:10807000F0EE406A27EE830AC0ED056AA3EEA60A79
:1080800080ED087AA4EE240AA5EE470AA5EEC60AFA
:1080900080ED070A704700BFD0ED007A90ED017ABD
:1080A00030EE670AE7EE007AB0EE670AC0ED007ABC
:1080B000704700BF704700BF2DE9F04714461D46CA
:1080C00006464FF47A7200232046294646F016FCF5
:1080D0004D4BDFF848814D4A4D4F034488FB031058
:1080E0001844D91782FB032CC1EB601088FB0028D1
:1080F00087FB03279C44474AC1EBEC2CC0EB001ED6
:1081000082FB0C29A3EB8E0E1F44434A86F806E03F
:10811000C1EB27474FEAEC7E08EB000ACEEBA90E35
:1081200082FB07824FEAE0780EEB4E0EC8EB6A182E
:10813000ACEBCE0CC8EB0818DFF8E4E086F804C01E
:10814000A0EB880070718EFB0303F817C0EBE212FE
:1081500040F2B55000FB1272C1EBE353B2F5896FE8
:108160004FEA83073CDA40F2DA239A4242DCB2F566
:10817000B77FB4BF4FF0000E4FF0010E4FEA4E092B
:10818000DFF8A08009EB0E0308EBC3031FFA8EFC97
:10819000D88A09EB0E0108EBC10116310B2301E06F
:1081A00031F8020D904218DD013BF9D1CE44012394
:1081B00038F83E00B37007F5FA670132121ABC4472
:1081C000F270A6F800C0204629464FF47A720023C8
:1081D00046F094FB3281BDE8F0870133DBB2E9E77A
:1081E0004FF0030CE64640F29650DFF838804FF02F
:1081F0000609CEE74FF0020CDFF82880E64640F291
:1082000029404FF00409C4E780BC92C7C5B3A291CE
:1082100007452EC2ABAAAA2A73B06D168988888832
:10822000792D03116006050830B403888278C4787C
:10823000154DA3F5FA6303F0030101EB4101013A87
:1082400002EB81029B0835F812500279611E40F260
:10825000B55404FB03132B4403EB430302EBC303AA
:108260004279847909490089C3EB031302EB830344
:108270002144C3EB031301EB83034FF47A72002113
:10828000C2FB030130BC70476006050880436D38AF
:108290000028F0B403DA2D230B7040420131092885
:1082A00004464FF0010307DD03EB83035B00B0FBE3
:1082B000F3F2092AF8D883B10F48A0FB0326B4FBD8
:1082C000F3F2092A02F1570C02F1300709DD03FB32
:1082D0001244F30801F801CBEFD100230B70F0BC7E
:1082E000704703FB1244F30801F8017BE5D100233A
:1082F0000B70F0BC704700BFCDCCCCCC884270B4C2
:108300004FF0010442D301FB04F4B0FBF4F58D42BD
:10831000F9D2ECB142BB092D04FB150005F157065B
:1083200005F130020EDDB4FBF1F403F8016B7CB112
:10833000B0FBF4F5092D04FB150005F1570605F116
:108340003002F0DCB4FBF1F403F8012B002CEFD188
:1083500000221A7070BC704703F8016BB4FBF1F493
:10836000002CF5D0B0FBF4F5092D04FB150005F148
:10837000370605F13002EFDCB4FBF1F403F8012B12
:10838000002CEFD100221A7070BC70470546002AFD
:10839000EAD1C0E703685A1C02601970704700BF39
:1083A0002DE9F047089C2578002B804689460CBFB4
:1083B0004FF0200A4FF0300A661C25B3002A26DD54
:1083C000334601E0024698B113F8011B501E002904
:1083D000F8D1971E60B13D46013D51464046C84721
:1083E0006B1C002BF8DC257827EAE770013045B1DB
:1083F000041B29464046C847301916F8015B002D7A
:10840000F7D1BDE8F087002A03DC2846F9E7002011
:10841000EEE7571EDFE700BF01212A220223017089
:1084200042708370704700BFF0B400250E4E00F11B
:10843000FF3C2F46322165B103788B420BD00346B7
:108440000CEB050403E013F8012F8A4203D0A3428A
:10845000F9D1C155013701350B2D02D016F8011F96
:10846000E9E7F0BC704700BFC00605080C4AF0B44D
:10847000002302F1080717261625152403EB4303F2
:10848000C118BA42C4544D708E7006D092F90430AF
:1084900054799579D6790432F0E7F0BC704700BF83
:1084A000CC060508012310B4342135242122447060
:1084B0004171C27003720370037183705DF8044BE5
:1084C000704700BF06224FF47A7302704360704712
:1084D00030B41D6995420AD314460A4621448D42A0
:1084E000996938BF2A1B214430BC46F057BC30BCC8
:1084F000704700BF00207047002070470120704780
:108500000120704700207047002070474FF4007032
:10851000024B10609B680B600020704748BF002032
:1085200003484FF40073806A0860002013607047AE
:10853000D8BE0020013A30B4D2B28C1C04EB420405
:108540000025020F092AD3B203F130028ABF373364
:108550000A700B704D7002318C424FEA0010F0D15E
:1085600030BC70470B4A0C4B10681B681A22C018AD
:108570000A8001D10948704710B5094B09491C68A8
:108580000822FFF7D7FF204604220749FFF7D2FF52
:10859000024810BDE8F7FF1FECF7FF1F00000020A6
:1085A000EAF7FF1F020000201200002004230B80C6
:1085B000004870471C00002012230B8000487047C1
:1085C000200000203022032302704370704700BF58
:1085D00008307047704700BF816170476D4B2DE9CF
:1085E000F04F1C686C4BB3F80AE0B3F804809A892A
:1085F0004FEA0E2AB4EB0A044FEA1E6B4FF0000557
:1086000087B065EB0B05CDE900450746009C18894E
:10861000019EA0FB044500FB0655E00940EA4560C9
:108620004FEA08448C46E9114FEA184510EB04085C
:10863000D888009C41EB0509CDE90489A0FB0445DD
:10864000B3F8028000FB0655200A40EA05604FEAB5
:10865000C83429124FEA584510EB040841EB0509CC
:108660000099A2FB010102FB06114FEAD05A4AEA27
:10867000412A1AF5FA634FEAE15B4BF10004B3F5C6
:10868000FA6FCDE9023474F10003424E64DA052436
:10869000AAFB040104FB0B1100FB0BF40AFB0144D1
:1086A000DDE90423A0FB0A0121444D104FEA300408
:1086B000121B4FEA900463EB050344EA8174B8EBA4
:1086C0000408CDE90423DDE9023434484FEAA1056A
:1086D00069EB05094FF0FF31834274EB010326DAA1
:1086E00040F6AC501AEB00024FF000014BEB0103D7
:1086F00002FB03F1A2FB022303EB4103D400DD00E4
:10870000101B45EA527563EB0501DDE904452418A9
:108710004D41CDE904450B24A2FB040104FB0311E8
:1087200049104FEA3000B8EB000869EB0109DDE9B8
:1087300000325343009ADDE90201A2FB02AB0BEBCE
:10874000430B4FEADA7242EA4B02801A4FEAEB73AC
:1087500061EB0301CDE9020197B17168A1FB082328
:1087600001FB0933540D5D1544EAC324DDE90423FC
:10877000A21A65EB03031D46D30B43EA45433B6056
:10878000BCF1000F02D0029BCCF8003007B0BDE86E
:10879000F08F00BF582800209468002024FAFFFFC3
:1087A0002DE9F04FDFF8DCC1754CDCF80850228869
:1087B000B4F90AA0C2EB25135200C2EBE502B4F9EA
:1087C00002505B436A43B4F904501B135D43AD137D
:1087D00005EBE225B5F5FA324FEAE57B85B04BF1C2
:1087E000FF33CDE90023DDE900325343009AA56150
:1087F000A2FB0289CDE90201B4F908200199009891
:1088000009EB43095143D31700FB0311A2FB0023DB
:108810000B444FEAEA7B0AFB09F11F0308FB0B1329
:10882000AAFB080119444FEA102A4AEA016A160312
:108830004FEA212B47EA12571AEB0602E6884BEB68
:10884000070312F1000A43F5004BAAFB060106FBE1
:108850000B114A10CB1752EA030100F08E80B4F9D5
:108860001060009806FB09F1F71708FB0711A6FB3B
:1088700008673944B4F90E808B4601994FEAE879CC
:1088800008FB01F100FB0911A8FB00898944DCF811
:108890000C104FEA4947C1F5801C47EAD837B24669
:1088A0004FEA4846B4F90C801AEB060A66464BEBD1
:1088B000070BF7174FEAC806019600260096F9073E
:1088C000DDE900674FEACC7016EB0A0647EB0B07B1
:1088D00041EA5C01801B61EB070140F6354C89469B
:1088E000A0FB0C010CFB091146F008F8B4F91620A6
:1088F000B4F914A04E13470B47EAC14702FB06FC2C
:10890000D31707FB03CCA2FB07236344564307FBA3
:108910000366A2FB07233344560E46EAC3163218F9
:108920004FEA636747EB010380460AFB01F14FEA18
:10893000EA7B08FB0B17AAFB08013944C60C46EA80
:10894000413612EB06084FEAE147B4F9122043EB37
:1089500007094FEA182141EA096113010B44029A01
:108960000AB11B0A1360039B23B105EB8505803513
:108970002D121D6005B0BDE8F08F0023EFE700BFAA
:10898000A868002058280020704770472DE9F04162
:10899000334B344E1A8A7489B6F91450B6F90480F0
:1089A000B6F90E70B6F920C05B69121B34895443C6
:1089B000E213B6F912401544E40294FBF5F4B6F95B
:1089C00002501444A4F57A6E0EFB0EF20EFB05F570
:1089D0000EFB08FEB6F90C80F4611213574302FB3C
:1089E00008F2121402EB6E32ED1205EBE7270232A9
:1089F000B6F90050B6F806E0921002F5004207EB17
:108A000085070EFB02F207FA0CF74FEAD23E023757
:108A10004CF25032A3EBA70742FA0CF37B4355BF4D
:108A20005B00B3FBFEF3B3FBFEF35B0078B11A12FD
:108A300002FB02F540F6DE326A430B4D12145D4331
:108A400002EB254202F6CF6203EB2213036021B151
:108A50000A235C43083424110C60BDE8F08100BF98
:108A6000582800207068002043E3FFFF4FF40063A4
:108A7000838270474FF4006383827047012380F83C
:108A8000543070474FF4006383827047F0B4037C26
:108A9000456902681F2B37D9203B20215468994033
:108AA0000C4223D010249C40D160D4605168D9403E
:108AB000CE074ED4EFF31183502282F31288EA6B73
:108AC0001168C90709D45468002C52D1D5E909614D
:108AD0008E4243D1012285F86020DBB283F31188F6
:108AE000037C02681F2B194614D9203B08215068CB
:108AF0009940084200D0D1600421506801FA03F384
:108B0000184223D1F0BC7047202416689C402642AE
:108B10000FD11946082310688B40184200D093608B
:108B20000423106803FA01F10842EBD09160F0BC15
:108B3000704710219940946091601168D940CC072A
:108B4000B8D5012101FA03F39360B3E7D360F0BC19
:108B50007047012101FA03F3D360ABE7AF690F441B
:108B6000D7600ED82E69711A5160AC62002185F869
:108B70006010116841F00101DBB2116083F31188CC
:108B8000AEE7711A5160AE62F0E700BF70B4037CCB
:108B900001681F2B26D9A3F1200520224C68AA408A
:108BA000224214BF01220022D2B142691B481C4C50
:108BB00002EB420200EB4212257854682068CDB9DE
:108BC000E56856892C6824F001042C6082891F2BEB
:108BD00022EA060282811AD8202202FA03F38B606D
:108BE00070BC704720220C689A40224214BF0122B8
:108BF0000022D9E7A469226822F00102226082895A
:108C000022F480721204120C1F2B8281E4D9A3F18A
:108C1000200220239340CB6070BC7047E0CD002041
:108C20001813001070B59D4C2368002B40F005818F
:108C30009B4B1A78002A68D09A4B19789A4B0029D6
:108C400064D11868B3F82C5141628489012A44EA3E
:108C500005048481A3F82C1157D0D3F83001B3F860
:108C60005C5241628489022A44EA05048481A3F8A3
:108C70005C124AD0D3F86002B3F88C534162848905
:108C8000032A44EA05048481A3F88C133DD0D3F869
:108C90009003B3F8BC5441628489042A44EA050471
:108CA0008481A3F8BC1430D0D3F8C004B3F8EC55D9
:108CB00041628489052A44EA05048481A3F8EC15FD
:108CC00023D0D3F8F005B3F81C5741628489062AF3
:108CD00044EA05048481A3F81C1716D0D3F82007B2
:108CE000B3F84C5841628489072A44EA0504848118
:108CF000A3F84C1809D0D3F85028B3F87C49516236
:108D0000908920439081A3F87C1970BD5C68198913
:108D100061602568186845F0010540F20D31256055
:108D2000A0F848108489012A44F480748481ECD02E
:108D3000D3F83441B3F83851D3F830016560256871
:108D400045F001052560A0F848108489022A44F402
:108D500080748481D9D0D3F86442B3F86852D3F8D0
:108D600060026560256845F001052560A0F848109F
:108D70008489032A44F480748481C6D0D3F8944350
:108D8000B3F89853D3F890036560256845F0010562
:108D90002560A0F848108489042A44F480748481F2
:108DA000B3D0D3F8C444B3F8C854D3F8C004656052
:108DB000256845F001052560A0F848108489052A3A
:108DC00044F480748481A0D0D3F8F445B3F8F85506
:108DD000D3F8F0056560256845F001052560A0F829
:108DE00048108489062A44F4807484818DD0D3F895
:108DF0002447B3F82857D3F820076560256845F065
:108E000001052560A0F848108489072A44F480747D
:108E100084813FF47AAFD3F85428B3F85808D3F8D4
:108E200050385060106840F001001060A3F84810FE
:108E30009A8942F480729A8170BD05460AF0EAFD73
:108E4000217AA9B16DB1194A002316890133002E88
:108E500018BF0021AB4202F16002F6D100293FF4B5
:108E6000E7AE00F51C501030002320602372DFE6CF
:108E70002368C31A002BFFF648AF637A3BB1013B6E
:108E8000DBB263722BB100F57A702060D0E623600C
:108E9000CEE6636803442360CAE600BF8056002024
:108EA000E0D0002018130010E4D00020E0CD002016
:108EB00010B5027C01681F2A4FF020030ED94C68C0
:108EC000203A93401C4208D00B4A4068002414709A
:108ED000026822F001020260CB6010BD0C68934072
:108EE0001C42FAD0044A406800241470026822F040
:108EF000010202608B60F0E7456F00202DE9F04130
:108F0000C40023189B00B749CA585268958AADB26D
:108F1000EFB2FE070B4461D4BE0737D5BFF35F8FB6
:108F20001D7EEDB2012D00F0BB80AF4E138BBFF361
:108F30005F8F231801EB83031D7E022D00F0CE808E
:108F4000231801EB83031D7E032D05D19B7E1BB1EE
:108F5000737E002B40F01A81938896F918C043F471
:108F600080639380231801EB83031B7E01336345E9
:108F70000AD1B37E00257576002B40F08A8020440C
:108F800001EB800000234375BDE8F081964E17F099
:108F9000040F96F918C04DD117F0400700F0B280C9
:108FA000178A1D6AFFB205F80C705FFA8CF56F1C0A
:108FB00093F818E07BB2DF1CBE4533769C4600F088
:108FC0000981271801EB87073F7EBB42CAD105F113
:108FD000020C4FFA8CFC86F818C0C3E71588824E45
:108FE00025F400652D042D0C1580158845F4806549
:108FF00015809D7E00273776002D3DD0757E002D93
:1090000037D0231801EB830301251B7E7576022BD5
:1090100003D1138843F400631380231801EB830307
:109020009B7D43F001031382204401EB8000037E0B
:10903000BDE8F0819F7E757E4FF0010E86F81AE044
:10904000002F5CD0002D78D1231801EB83035B7EC9
:10905000002B00F0A48013880CF1010C4FFA8CFC5B
:1090600043F4007386F818C013801388DF05FCD41E
:1090700078E7DB7DFF2BC4D0231801EB83039D7DB4
:1090800005F0FE051582DB7DFF2BCDD0FF23337667
:10909000CAE7938823F440731B041B0C93806EE78C
:1090A0009B7E514E002B3FF441AF737E002B3FF46B
:1090B0003DAF138823F480631B041B0C1380BFF3A4
:1090C0005F8F138B1388B57643F4007313809388F6
:1090D00096F918C043F48063938043E79B7E002B8E
:1090E0003FF42EAF737E002B3FF42AAF138896F91E
:1090F00018C023F480631B041B0C138016E0002DA2
:10910000A2D0A8E72D067FF52DAFBCF1FF3F6DD0B3
:10911000DD6915F80C5015820CF1010C1D7E4FFA1B
:109120008CF39D429C4633767FF41CAF938823F4E6
:1091300080631B041B0C938014E71F7ED3F82080F0
:109140005FFA8CF5AE44022F4FFA8EFE17882DD9A8
:1091500027F480673F043F0C1780178AFFB208F896
:109160000C701788D3F820C047F400731380138A5B
:10917000DBB20CF80E30938805F1020C4FFA8CFC30
:1091800043F4806386F818C093806EE7938896F95D
:1091900018C023F480631B041B0C9380E2E6138841
:1091A000012543F48073138075765EE747F40077FA
:1091B0001780178AFFB208F80C70178AD3F820803E
:1091C00005F1030C4FFA8CFCFBB286F818C008F8C6
:1091D0000E304AE7978827F480673F043F0C97805A
:1091E000EFE600BF305D002058280020DD7D1582AD
:1091F0009D7E37761DB91B7E002B7FF415AF9388BB
:1092000023F480631B041B0C93800DE710B427210B
:10921000262401220023047041708270C3705DF81F
:10922000044B70472DE9F84FDDE90A64894617467B
:10923000002120229846054645F016FE5EB1D6E98B
:1092400000327189EB81C3F30F432B82C2F30F43CA
:10925000EA822B836982484644F064FE17F0100BC3
:1092600010D1431E70B119F803202E2A18BF09EB44
:10927000030104D14AE011F8016D2E2E3ED013F106
:10928000FF33F8D208280246CA46A8BF08224FF08A
:10929000000B4FF020336B602B60C5F80730494658
:1092A000284605F1080645F079FD5A4651463046F4
:1092B00045F074FD6B1EE81D13F8012FA2F161014A
:1092C00019299CBF203A1A708342F5D105F10B0190
:1092D00016F8013BA3F16102192A9CBF203B06F856
:1092E000013CB142F4D11823C8F30F42EF722B7343
:1092F000A5F81A80AA82EC61BDE8F88FC01A00F1C7
:10930000FF3BBBF1030FA8BF4FF0030B082B03F18A
:10931000010AA8BF0823CA441A46BAE738B51D4B4C
:109320001B78044600F1250593B104221A49203028
:1093300045F0D8FD28461422184945F0D3FD0123F5
:1093400084F83A30164B1B7873B984F83B3038BD3B
:1093500028461422134945F0C5FD012384F83A300C
:109360000F4B1B78002BF0D00F4B186859689A6888
:10937000DD68E56020606160A260DD691869596997
:109380009A69A2610123E5612061616184F83B3043
:1093900038BD00BF7D8D00207E8D0020838D002094
:1093A0005C8D0020C05505085D8D0020014B1868BC
:1093B0000AF080BEEC55002010B5002104460120C3
:1093C00009F0CEFA207010BD38B500240472451E95
:1093D000E1B2022009F0C4FA0134082C05F8010FAB
:1093E000F6D138BD38B52C22002145F03DFD0346AD
:1093F000642140F2DC5240F2022019745A82132197
:10940000202240F21A4540F26C74188399760E209F
:1094100002211A7701229D82DC8240F2753540F6E6
:10942000430483F82200197283F82A109A7383F890
:109430002920DD831C8419460248BDE8384031F0FC
:10944000A9BA00BFCC5505082DE9F04F002087B020
:109450000C461D46012192460DF0B8FD002D63D04B
:1094600005EB0A03DFF8D094DFF8D0B40393554638
:109470001CE0002D00F0C581D9F81430AB4264D057
:10948000D9F81030AB4200F09780D9E90631AB42F1
:1094900052D8A94200F26F81691A20463AF0F8FFCB
:1094A000039B01359D4204F500743DD0D9F820603E
:1094B000AE42DED8D9F83080AE1B4FEAD60AD8F8D3
:1094C00030300AF1020A9A4506F0070603D3D8F8AD
:1094D00038309A4509D9414650463AF0A7FF8046B0
:1094E000002800F04D81C9F8300098F80430002BB6
:1094F00040F0E280D8F82870002F00F0DF81D8F823
:109500003030D8F80C20AAEB030A06EBCA0A43460F
:10951000204602EB4A224FF40071B847039B013505
:109520009D4204F50074C1D1002108460DF04EFDA6
:10953000002007B0BDE8F08FA942ADD94FF400720A
:109540000021204645F090FCAAE7522261204123E9
:10955000002622706270A070722284F8E70184F8FD
:10956000E631D9F82800E3704FF0FF33314684F834
:10957000E42184F8E521C4F8E8014FF4F07284F89E
:10958000EC3184F8ED3184F8EE3184F8EF31201DB0
:1095900045F06AFC55216FF05502C4F8F061C4F83B
:1095A000F461C4F8F86184F8FC6184F8FD6184F822
:1095B000FE1184F8FF2173E74FF40072002120466A
:1095C00045F052FCD44BD54F03CBEB230222237042
:1095D0004FF0080C9026F8234FF0580EC4F8030003
:1095E000227484F80DC0C4F8071084F801E0A67056
:1095F0006375D9F81010D9F80830D9F81C602273B7
:10960000591A21624FF0FF3100233F20A1763E21FD
:10961000A273E372E3736374A374E3742375A37595
:10962000E3756376E3766377A377E3772076217734
:1096300084F82C2007CFD9F8187084F82830F61B4E
:1096400084F8293084F82A3084F82B3084F82D30BF
:1096500084F82E3084F82F3084F8313084F832309A
:1096600084F8333080236662C4F8470004F147066B
:1096700084F8403029209423A94F84F846C084F808
:10968000420084F843300E200D234FF0010C84F883
:10969000440084F8453084F830C0716003CF33460D
:1096A0005527AA269A60C4F85200C4F8561084F8C8
:1096B000FE7184F8FF61F3E64FF40072002120464A
:1096C00045F0D2FBD8F84030002E61D104F12007DC
:1096D000002B77D0D8F8303092491122CDE90066BE
:1096E0002046FFF79FFDD8F840301A6C04F1400A7D
:1096F000002A79D01B6B8C49CDE9006638461122CF
:10970000FFF790FDD8F84460002E3FF4C9AE4FF447
:10971000E078CDE904450CE00024CDE900C4FFF772
:1097200081FDB66CBA46A8F120080EB3B8F11F0F40
:109730001ED93468356B96F804E011222B46214679
:1097400050460AF1200706F11C0CBEF1000FE3D1D0
:1097500072793369019342F021022B46CDF800C0A3
:10976000FFF760FDB66CBA46A8F12008002EDDD1E7
:10977000DDE9044594E6E91A20463AF089FE8FE6D1
:10978000231F04F5FE7243F804BF9A42FBD187E61B
:10979000002BD8F844200CBF01230223C3EB06138F
:1097A000002A3FF47DAE966C013B002E3FF478AE6C
:1097B000013BB66CF9D1002E3FF472AEA2464FF4D5
:1097C0000078A6E7CDE900663346D9F80C100822E8
:1097D0002046FFF727FDD8F84460002E3FF460AE26
:1097E000BA464FF4F07894E7CDE900663346384640
:1097F00011224D49FFF716FDD8F84460002E86D19E
:109800004EE64FF400722946204645F02DFB80229B
:109810000C2384F8BE2184F8C231D9F81000434BE0
:10982000D9F8086084F8B85183FB0032C117C1EB46
:109830002232B2F5806F84F8B95184F8BA5184F8B5
:10984000BB5184F8BC5184F8BD51C4F8C601C4F8BA
:10985000CA6142DBFF2384F8BF3184F8C13184F848
:10986000C031324B711E83FB0132CE17C6EB223260
:10987000B2F5806F29DA2E4B84F8C52183FB0103F2
:109880000B442C48C6EB6313C3EB831680FB0370B9
:10989000891B1844DE17921022F03F020131C6EBFB
:1098A000E0100A43034484F8C42184F8C3315522EC
:1098B000AA2384F8FE2184F8FF31F1E539464FF4FC
:1098C0000072204645F0D0FAEAE5FF2384F8C33160
:1098D00084F8C53184F8C431E9E7154B84F8C12117
:1098E00083FB00730344134FC1EB631387FB031720
:1098F000C3EB831C9110A0EB0C02F818DF1721F0CA
:109900003F010132C7EBE0100A43034484F8C02151
:1099100084F8BF31A5E700BFE0550508EC55050800
:10992000FC550508D8550508DC55050897554541EF
:10993000832008828180808048BF0020DEADBEEF9A
:1099400008B535F08FFF80F00100404240B208BDFD
:1099500070B50C4601211E46084615460DF036FB33
:10996000AEB104EB462601E035F07CFF0022214633
:1099700028463AF0F5FB0028F6D135F073FF0028B1
:10998000FBD004F50074B44205F10105EED10021CD
:1099900001200DF01BFB002070BD00BF70B50C4610
:1099A00001211E46084615460DF010FB96B104EB4A
:1099B00046260022214628463AF06AFC0028F8D0C4
:1099C00035F050FF0028FBD004F50074B44205F1D7
:1099D0000105EED1002101200DF0F8FA002070BD44
:1099E000002108B508460DF0F1FA3AF08BFC35F08D
:1099F00039FF0028FBD0012100200DF0E7FA0020FC
:109A000008BD00BF10B5044C04480A46214636F094
:109A1000B1F9204610BD00BF742800200856050883
:109A200010B5044C04480A46214636F0A3F92046F6
:109A300010BD00BF742800201856050810B5044C4E
:109A400004480A46214636F095F9204610BD00BF6D
:109A500074280020245605080A4608B5054920B197
:109A6000054836F087F9034808BD044836F082F906
:109A7000004808BD742800205056050838560508CF
:109A80002DE9F0410B4E346873691C400FD0DFF8AC
:109A900028800127B4FA84F3C3F11F0307FA03F502
:109AA00058F8230003689847AC437561F2D1BDE8CC
:109AB000F08100BF003C014028B800202DE9F041B2
:109AC0000B4E346873691C400FD0DFF828800127E3
:109AD000B4FA84F3C3F11F0307FA03F558F823001F
:109AE00003689847AC437561F2D1BDE8F08100BFCF
:109AF000003C014028B800202DE9F0410B4E3468AD
:109B000073691C400FD0DFF828800127B4FA84F372
:109B1000C3F11F0307FA03F558F8230003689847B9
:109B2000AC437561F2D1BDE8F08100BF003C01405B
:109B300028B80020084A094808B5536C43F480430C
:109B400053640021402245F08FF9054B4FF0FF325E
:109B50001A60C3F8032008BD0038024028B800206E
:109B600068B8002010B58B68016004469847002251
:109B7000FF230121A2736373217310BD03685B6A25
:109B8000184700BF03681B6A184700BF70B44E1C1B
:109B90000568C2728672AC69A44670BC604700BF9B
:109BA0002DE9F041044618460D4616461F4644F07E
:109BB000B9F92844A0722068E672294645693B46F7
:109BC00032462046AC46BDE8F0416047036810B518
:109BD00004461B689847236820469B689847A37BE8
:109BE0000133A37310BD00BF10B5036804469B6822
:109BF0009847FF2301226373227310BD38B50D46C9
:109C000008F0FEF8044650B136238371C571012176
:109C10000DF02CF92046BDE838400DF0C9B938BD2B
:109C200038B50D4608F0ECF8044650B13523837181
:109C3000C57120210DF01AF92046BDE838400DF01D
:109C4000B7B938BD0E4B984214D0A3F5784398426B
:109C50000ED003F5806398420ED10222094B03EB2C
:109C600002135A89013292B25A81588980B27047E0
:109C70000122F3E70022F1E74FF0FF30704700BF09
:109C80000030014018B60020F8B584894FF6FF7601
:109C90004FF47A7433B319B30F78013101E0B44251
:109CA00018D00589013CAD07A4B2F8D5BCB28481B7
:109CB0004FF47A7402E0BCB2B4420BD00589ED07D0
:109CC00004F1FF37F7D58589ADB20AB115700132BD
:109CD000013BDFE7FFF7B6FF003018BF0120F8BDFA
:109CE000FF27DEE70120F8BD30B5437F83B004468F
:109CF0001BB90120637703B030BD0523ADF80430F4
:109D0000056800BFA8680DF04DF96A4601A9022355
:109D10006868FFF7B9FFA8680DF04AF900BF9DF821
:109D2000013003F0010383F00100637703B030BD1D
:109D3000F8B5074C05460F46266803E023689B1BD1
:109D4000BB4204D82846FFF7CFFF0028F6D0F8BD65
:109D500094B60020F0B5077F83B004464FF0030CA3
:109D60000020009016461D468DF804008DF800C0B6
:109D70006FB30B0E8DF801300DF10203080C0A0AC7
:109D800099701870062120465A70FFF7D1FFE0B194
:109D9000236800BF98680DF005F9237F2268002B27
:109DA00014BF05230423694650680022FFF76CFFA7
:109DB00023683246002158682B46FFF765FF236869
:109DC00098680DF0F5F800BF284603B0F0BD0DF11E
:109DD0000103D3E72DE9F0418046806810B10468A3
:109DE00080886083D8F8040085894FF47A744FF630
:109DF000FF7613F1FF3320D341B30F78013101E037
:109E0000B44218D00589013CAD07A4B2F8D5BCB264
:109E100084814FF47A7402E0BCB2B4420BD005895D
:109E2000ED0704F1FF37F7D58589ADB2002AE0D000
:109E300015700132DDE7FFF705FFD8F8083013B1E0
:109E40001A689B8813830120BDE8F081FF27D9E7BA
:109E5000F0B5876983B0064617B13B68BA885A8364
:109E60007069DFF8A8E08389C3244FF47A734FF058
:109E7000060C6D464FF6FF710EF1010E03E0013B3B
:109E80009BB28B4220D002899207F8D5A3B283817E
:109E90004FF47A7302E0A3B28B4215D00289D20745
:109EA00003F1FF34F7D5828992B20DB12A700135E2
:109EB000BCF1000F0BD00CF1FF3CFF24BEF1000FF2
:109EC000E1D09EF80040D7E7FFF7BCFEB76917B1B5
:109ED0003B68BA881A839DF805009DF801509DF8EB
:109EE00002109DF803409DF804209DF8063041EAD9
:109EF000052143EA002342EA04220120A6F850107B
:109F0000A6F85220A6F8543003B0F0BDD8060508D4
:109F100008B540F2E93300E0A3B10289013B12F039
:109F2000020F9BB2F8D089B2818140F2E93300E0A0
:109F300043B10289013B12F0010F9BB2F8D0808936
:109F4000C0B208BDFFF77EFEC0B208BD427A4AB17A
:109F500010B5044604F10A01D0E900309847002307
:109F6000637210BD704700BF437A5A1C0344D2B2DB
:109F700042729972037A93420AD84AB110B50446E4
:109F800004F10A01D0E9003098470023637210BD44
:109F9000704700BF48B10123302803FA01F101D016
:109FA000312803D14A0709D1002070473228F9D05F
:109FB0003328F7D0342803D18B07F5D00120704720
:109FC0003528F9D02028F7D02128F5D01028E9D05D
:109FD0001128E7D01228E5D01328E3D01428EBD0BD
:109FE0001528E9D0162804D111F0030018BF01206C
:109FF00070471728D8D111F0030018BF012070470F
:10A00000302829D0312829D0322829D0332829D006
:10A01000342829D0352829D020282BD021282BD00E
:10A02000102825D0112829D0122829D0132829D06A
:10A03000142829D0152829D0162805D0172808BF9C
:10A040000F2302D0002070470E23114A03EB430375
:10A05000134493F8820070470023F6E70123F4E7E6
:10A060000223F2E70323F0E70423EEE70523ECE7FE
:10A070000823EAE70623E8E70723E6E70923E4E7FE
:10A080000A23E2E70B23E0E70C23DEE70D23DCE7FE
:10A0900060060508024A136823EA00001060704752
:10A0A000A0640020F8B50468C4F30D0405460E460C
:10A0B00004B32F6837F074F9092840F08880454CC4
:10A0C000236923F440732361236943F400732361FC
:10A0D000236943F0010323613E6037F061F923698E
:10A0E000092823F00103236171D12B6804332B600D
:10A0F000002035E0384B394A93422BD902F5804293
:10A10000934226D902F5804293422AD902F5804231
:10A11000934228D902F58032934226D902F50032C3
:10A12000934224D902F50032934222D902F500323B
:10A13000934220D902F5003293421ED902F58022C3
:10A1400093421CD9B3F1016F1BD3052008F0B8FE70
:10A15000FBE7082437F024F9092814D04FF0FF302A
:10A16000F8BD1024F6E71824F4E72024F2E72824A9
:10A17000F0E73024EEE73824ECE74024EAE748240F
:10A18000E8E75824E6E7134F3B6923F440733B614B
:10A190003B6943F400733B613B6923F0F8033B6187
:10A1A0003B6943F002031C433C613B6943F4803349
:10A1B0003B6137F0F5F83B6923F002033B613B69F3
:10A1C000092823F0F8033B613FF473AFC6E76FF053
:10A1D0000100C5E7003C024000400008FF3F0008C6
:10A1E000F8B504460D468E180027B542206900D107
:10A1F000F8BDE368591CE160234415F8012B1A727D
:10A200000429F2D118B9A1682046FFF74BFFC4E931
:10A210000370EAE730B402681146531C036011F87A
:10A22000024B0160D31C517803609378151D0560C3
:10A230001B0443EA0123D078234343EA006030BC87
:10A24000704700BF0368591C1A46016012F8021BD0
:10A250000260587841EA0020704700BF03685A1C2A
:10A2600002601878704700BF70B5044608460E4675
:10A2700043F058FE314605460246206844F08EFD04
:10A2800020682844206070BD38B504460068154633
:10A2900044F084FD22682A44226038BD036810B46B
:10A2A0000A0E5C1C04601A7003680A0C5C1C0460D3
:10A2B0001A7003680A0A5C1C04601A7003685A1C4E
:10A2C000026019705DF8044B704700BF036810B45A
:10A2D0000A0A5C1C04601A7003685A1C0260197038
:10A2E0005DF8044B704700BF03685A1C026010B44D
:10A2F000197003680A0A5C1C04601A7003680A0C6F
:10A300005C1C04601A700368090E5A1C0260197004
:10A310005DF8044B704700BF03685A1C0260197057
:10A320000368090A5A1C02601970704710EE103A4F
:10A33000C3F3160242F07E5207EE102ADFED167AC2
:10A34000DFED164A9FED165ADFED165A9FED166A9D
:10A35000DFED163ADFED166A9FED164AE7EE274A63
:10A36000DB1507EE903AA4EE875AF8EEE77AE5EEB1
:10A37000075A67EEA37AA5EE876AB5EEC00AE6EE45
:10A38000077AF1EE10FAD4BFB0EE440AB0EE660AD6
:10A3900037EE800A704700BFDACDFE3CB9D593BED8
:10A3A0005CB8903FAA841DC022E061401872313F22
:10A3B00007F1B3C2000080FFDFED1D3ADFED1D7A2B
:10A3C0009FED1D7A9FED1D4ADFED1D4A9FED1D5A41
:10A3D000DFED1D5A9FED1D6ADFED1D6AE0EE237A69
:10A3E000F4EEC77AF1EE10FA88BFF0EE477AF4EE99
:10A3F000C47AF1EE10FAB8BFF0EE447AFDEEE77AD7
:10A4000017EE903AC3F3160242F07E5207EE102A7E
:10A41000A7EE245A03F0FF4300EE103AE5EE075A88
:10A42000A5EE876AE6EE076A26EE800A704700BF4F
:10A430003BAA384B00007E4E0000FF4E000000009B
:10A44000ED185E3C81900FBBAF9D2A3EB2D19F3E7E
:10A45000E886023F07EE901AF8EE677A9FED837A5E
:10A4600027EE800A20EE070AFDEEC07A17EE903A3A
:10A470002033402B00F28180DFED7D7AB4EEE70AD5
:10A48000F1EE10FA40F3E680B0EE407A9FED796A83
:10A49000DFED796A01E0B0EE677AB4EEE67AF1EECC
:10A4A00010FA77EE467AF6DC9FED747AF4EEC77A0E
:10A4B000F1EE10FA40F1D1809FED6E6ADFED706A27
:10A4C00001E0F0EE477AF4EEE67AF1EE10FA37EEBC
:10A4D000867AF6D4DFED6B7AB4EEE77AF1EE10FA15
:10A4E00040F3A780DFED627A37EEC77A27EE076A7E
:10A4F000DFED655ADFED657ADFED656A9FED655A40
:10A50000E6EE257A67EE065AE6EE276AF7EE007A5F
:10A51000A5EEA67AF0EE675AE7EE055AE7EE457A21
:10A5200087EEA55ADFED577A30EE277AFDEEC76A3F
:10A5300016EE903A2033402B24D99FED577AF6EE51
:10A54000006AB7EE006AF7EE004AC4EEA57A00236F
:10A55000836143610362C36180ED045A67EEA66ABA
:10A5600027EE866A27EE877AC0ED006AC0ED026AA0
:10A5700080ED016A80ED037A7047B7EE005AF0EE85
:10A58000455ACFE7B4EEE70AF1EE10FA6BDD9FED26
:10A59000396ADFED396A01E0B0EE677AB4EEE67A47
:10A5A000F1EE10FA77EE467AF6DC9FED347AF4EEAF
:10A5B000C77AF1EE10FA53D59FED2E6ADFED306ABF
:10A5C00001E0F0EE477AF4EEE67AF1EE10FA37EEBB
:10A5D000867AF6D4DFED2B7AB4EEE77AF1EE10FA54
:10A5E00033DCDFED2E7AB4EEE77AF1EE10FA44BFF9
:10A5F000DFED227A37EEC77A27EE076ADFED224ACF
:10A60000DFED226ADFED227AE6EE246A67EE064A83
:10A61000E6EE267AB7EE006AA4EEA77AF6EE006AB6
:10A6200036EE476AF8EE007A27EE277A66EE266A5B
:10A6300089E7DFED1A7AB4EEE77AF1EE10FA44BF5B
:10A64000DFED0E7A37EEC77A50E7DFED097A37EEA5
:10A65000C77AD1E7F0EE407A26E7B0EE677A39E7BD
:10A66000B0EE677AB6E7F0EE477A9EE727D4D236A7
:10A67000DB0F4940DB0FC940E4CB1641DB0F49C07B
:10A68000E4CB16C1DB0FC93F92E741B99730083CD4
:10A6900015A82ABEF304353F00000000DB0FC9BF38
:10A6A000DFED2E7AB4EEE70AF1EE10FA4ADDDFEDC7
:10A6B0002C6A9FED2C7A01E0B0EE670AB4EEC70A6F
:10A6C000F1EE10FA70EE667AF6DC9FED277AF4EE82
:10A6D000C77AF1EE10FA3ED5DFED216A9FED237ABD
:10A6E00001E0F0EE407AF4EEC77AF1EE10FA37EEC0
:10A6F000A60AF6D4DFED1E7AB4EEE70AF1EE10FA00
:10A7000014DDDFED167A37EEC00A60EE006A9FEDC9
:10A71000196A9FED197ADFED197AA6EE867A20EE96
:10A72000266AE6EE877AA6EE270A7047DFED147AEE
:10A73000B4EEE70AF1EE10FA44BFDFED0B7A37EE24
:10A74000C00AE2E79FED087AF0EE407AF4EEC77AAD
:10A75000F1EE10FAC0D4B0EE670ACBE7DB0F494048
:10A76000DB0FC940E4CB1641DB0F49C0E4CB16C177
:10A77000DB0FC93F92E741B99730083C15A82ABEC4
:10A78000DB0FC9BFDFED317A30EE277AFDEEC76A05
:10A7900016EE903A2033402B02D99FED2D0A7047D8
:10A7A000B4EEE70AF1EE10FA4DDD9FED2A6ADFED17
:10A7B0002A6A01E0B0EE677AB4EEE67AF1EE10FABA
:10A7C00077EE467AF6DC9FED257AF4EEC77AF1EE65
:10A7D00010FA35D5DFED1F6A9FED217A01E0F0EE2A
:10A7E000407AF4EEC77AF1EE10FA37EEA60AF6D404
:10A7F000DFED167AB4EEE70AF1EE10FA1BDCDFEDBE
:10A80000197AB4EEE70AF1EE10FA44BFDFED137ADD
:10A8100037EEC00A60EE006A9FED136A9FED137A6F
:10A82000DFED137AA6EE867A20EE266AE6EE877AC8
:10A83000A6EE270A7047DFED0F7A37EEC00AE9E788
:10A84000B0EE670AD4E7F0EE477ABCE7DB0FC93F0A
:10A8500000000000DB0FC940E4CB1641DB0F49C00C
:10A86000E4CB16C1DB0FC9BF92E741B99730083C72
:10A8700015A82ABEDB0F49402DE90048FDF7D4FC9E
:10A88000054A064B1268B0EB020B61F1000CC3E9FC
:10A8900000BC0120BDE8008894B6002010700020A4
:10A8A0000F4B2DE93048D3E9004554EA05020AD19F
:10A8B000034640F2011200201880988098715A8057
:10A8C0001881BDE83088074B1A6814EB020B45F17C
:10A8D000000C5A466346FDF7EFFB0120BDE83088C7
:10A8E0001070002094B6002002B370B48E1803E0FC
:10A8F000121B14D1B14215D010F8012BA2F1410363
:10A90000192B11F8013BA3F1410598BF2032192DF5
:10A9100003F12004ECD9D21A01D1002BEAD1104660
:10A9200070BC70470022104670BC704710467047DC
:10A9300070B5044608460D4643F0F4FA064602E0B8
:10A9400014F8013F43B1324629462046FFF7CCFFB9
:10A950000028F5D1204670BD1C46204670BD00BFC2
:10A960004FF0FF32FFF7C0BFA0F16103192B98BF72
:10A9700020387047A0F14103192B98BF2030704751
:10A98000202805D0093804288CBF002001207047FA
:10A99000012070472DE9F0411F46064603461C780A
:10A9A0002046FFF7EDFF1D4601330028F7D12B2C81
:10A9B00051D02D2C24D0102A804628D04FF0FF33C0
:10A9C000B3FBF2F302FB03FC6FEA0C0C5FFA8CFCA6
:10A9D000013500200BE0303CE4B2944225DA984285
:10A9E0002E461DD81AD002FB004015F8014B392C19
:10A9F000F1D944F02004602C17D9573CE4B2ECE7BD
:10AA00004FF00108102A6C7805F10105D6D1302CE1
:10AA100023D06FF070434FF00F0CD9E76445E2D9B3
:10AA200007EA08084FF0FF30DFE701B10E60B8F128
:10AA3000000F08D027B1B0F1004F28BF4FF0004001
:10AA40004042BDE8F081002FFBD06FF000439842F8
:10AA500028BF1846F5E78046D4E76C782046FFF714
:10AA600089FF782805F1010605D035466FF070435F
:10AA70004FF00F0CACE7AC786FF0704302354FF03D
:10AA80000F0CA5E701230A22002183E7613819286A
:10AA90008CBF002001207047413819288CBF00204E
:10AAA00001207047303809288CBF002001207047F2
:10AAB000A0F13003092B07D920F0200041381928D4
:10AAC0008CBF002001207047012070470378202BA5
:10AAD000024600F10100F9D0092BF7D02D2B00F030
:10AAE000A4802B2B03BF5378B7EE000A0246B7EEC3
:10AAF000000AA3F13001C8B209289FED577A10D897
:10AB0000F2EE046A07EE901AF8EEE77A12F8013FC7
:10AB1000E7EE267AA3F13001C8B20928B0EE677AD1
:10AB2000F0D92E2B63D003F0DF03452B02D020EEAB
:10AB3000070A704710B451782D294FD02B2979D0AE
:10AB4000A1F13003092B02F101027AD8002400237D
:10AB500003EB830301EB430312F8011FA1F1300063
:10AB60000928A3F13003F3D9B3F59A7F1A4628BF19
:10AB70004FF49A72072B6CD9DFED386A1346F7EE63
:10AB8000007A083B072B67EEA67AFAD802F0070294
:10AB9000DAB1F2EE046A012A67EEA67A15D0022A2B
:10ABA00067EEA67A11D0032A67EEA67A0DD0042AA2
:10ABB00067EEA67A09D0052A67EEA67A05D067EE79
:10ABC000A67A062A18BF67EEA67A002C3BD087EE3D
:10ABD000277A5DF8044B20EE070A70479178A1F1BF
:10ABE0003003092B02F1020230D80124AFE7537879
:10ABF000A3F13001C8B2092802F1010293D8F2EEA4
:10AC0000046AF0EE665A07EE901AF8EEE77A12F848
:10AC1000013F87EEA66AA3F13001C8B2092866EEAB
:10AC2000A56A37EE067AEED97DE75378BFEE000AC3
:10AC300002465EE79178A1F13003092B02F102028E
:10AC400084D9F7EE007A27EE277AC2E7F7EE007A8A
:10AC5000BDE7F7EE007A9BE70000000020BCBE4C89
:10AC6000F8B5064615460846B6FBF2F434B905FBBE
:10AC700014640C4B1B5D00F8013BF8BDB4FBF2F70C
:10AC80005FB905FB1747074B05FB1464DA5D00F855
:10AC9000012B1B5D00F8013BF8BD3846FFF7E0FFD4
:10ACA000EFE700BF68560508B5EEC00ADFED677A2A
:10ACB000674AF1EE10FACCBF30EE270A30EE670A91
:10ACC000DFED647A20EE270A2DE9F047FDEEC07A29
:10ACD00088B017EE904A84EAE4760023A6EBE47687
:10ACE000CDE902330493A2FB06325FEAD20805469F
:10ACF00041D105AF58483946554BA3FB0623DB0825
:10AD000003EB8303A6EB4303002CC35C0B704FF0F3
:10AD10000002ACBF20232D234A7038468DF808303E
:10AD200043F000F90128394639D0022842D00328DF
:10AD300005BF302302A802A88DF8093044F09CF822
:10AD400002A843F0EFF80338C4B2224602A928460D
:10AD500044F0C8F800232B55284643F0E3F82E2290
:10AD6000431C02A92A542144E81844F0A1F82846BB
:10AD700008B0BDE8F087394BA3FB06235B0922D15D
:10AD800005AF35483946324AA2FB0832D20802EBF9
:10AD90008202A8EB4202835C01F8013BACE730235E
:10ADA00002A88DF809308DF80A308DF80B3044F088
:10ADB00063F8C5E7302302A88DF809308DF80A3012
:10ADC00044F05AF8BCE7264AA2FB06125FEA921941
:10ADD0000ED105AF204839461D4AA2FB03C2D20856
:10ADE00002EB8202A3EB4203C35C01F8013BCAE71A
:10ADF0001C4AA2FB06125FEA523A0ED105AF164872
:10AE00003946134AA2FB09C2D20802EB8202A9EB1F
:10AE10004202825C01F8012BDEE71348B6FBF0F03A
:10AE200058B905AF39460A20BAFBF0F200FB12A26E
:10AE30000948825C01F8012BE3E705AF39460A2295
:10AE40000193FFF70DFF019B0146ECE76F12033AF8
:10AE5000CDCCCCCC00007A44685605081F85EB5158
:10AE6000D34D62105917B7D1A086010070B406689F
:10AE70008E4217D90139751E002311F8014F08229F
:10AE8000634013F0800F4FEA430318BF83F0D503EC
:10AE9000013ADBB2F5D18D42EFD1721C0260337002
:10AEA00070BC7047721C00230260337070BC704726
:10AEB0000A44914215D010B40139541E11F8012FE3
:10AEC0000823504010F0800F4FEA400018BF80F078
:10AED000D500013BC0B2F5D1A142EFD15DF8044BE2
:10AEE000704770474840082310F0800F4FEA400039
:10AEF00018BF80F0D500013BC0B2F5D1704700BF4C
:10AF00000A44914215D030B40139551E41F2210254
:10AF100011F8014F082380EA042004044CBF82EAA0
:10AF200040004000013B80B2F7D18D42F0D130BCEF
:10AF30007047704770B502221349144C144E4FF6F7
:10AF4000FF70FFF7DDFF22884AB1A518B54218D27D
:10AF5000052A16D92146FFF7D3FF2C46F3E72146F1
:10AF60000222FFF7CDFF0222A118FFF7C9FF094B0C
:10AF7000E41A094B1C8041F60F53C31A584258413A
:10AF800070BD0020FCE700BF004000080240000840
:10AF900000800008FA3F0008648E00202DE9F0438D
:10AFA000002489B006460D461F46A04605E0252927
:10AFB0000CD030460134A847039A531C03931178F0
:10AFC0000029F4D1204609B0BDE8F083931CCDE9F7
:10AFD00003385078302842D0A0F13003DBB2092B7F
:10AFE0004FF0000945D96C282AD0642873D019D9AC
:10AFF000732858D063D9752840F0828007F1040C7B
:10B00000386805AB00220A216746FDF777F905ABE2
:10B01000049A009329464B463046FDF7C1F9039A3E
:10B020000444CAE725283CD051D958286BD063285E
:10B03000C2D139783046A84704370134039ABCE7B7
:10B04000039B5A1C03921B78642B52D016D8252BD5
:10B0500027D064D9582B18D0632BEAD0ADE7D31C86
:10B0600003939078A0F13003DBB2092B4FF0010974
:10B07000B9D804AA03A939F05DFAB4E7732B12D04A
:10B0800051D9752B2DD0782B97D1A3F15802B2FA54
:10B0900082F23868520905AB10210437FDF72EF90A
:10B0A000B5E7252185E73B68049A009329460023EC
:10B0B0003046FDF775F904370444039A7DE76E289E
:10B0C0007FF47AAF039A3B6804371C6075E7002869
:10B0D0003FF478AF70E7386805A9FDF7D9F8043771
:10B0E00095E7386805AB00220A21FDF707F9043718
:10B0F0008DE73B1D386805A91F46FDF7C9F886E7AF
:10B1000078287FF459AFA0F15802B2FA82F2386879
:10B11000520905AB1021FDF7F1F8043777E7002B52
:10B120003FF450AF49E76E2BCDD046E70EB400B5E3
:10B1300084B005AB019053F8042B0649039301A892
:10B14000FFF72CFF019B00221A7004B05DF804EB9E
:10B1500003B07047958300082DE9F04707468CB08F
:10B160001E469246002A5CD1154614460A88B2F55E
:10B17000FA6F36D38B78581E0B2832D891F803C05B
:10B180000CF1FF301E282CD891F804E0BEF1170F07
:10B1900027D891F80590B9F13B0F22D888793B2840
:10B1A0001FD8B1F80880B8F57A7F1AD24FF001089D
:10B1B0005EBB09890491002CB4BF2D212B21002CEA
:10B1C000B8BF6442CDE90290CDE905140795CDE9F9
:10B1D00000CE38462A49FFF7A9FF40460CB0BDE82B
:10B1E000F08700232749ADF828304FF0010C1846AE
:10B1F0008DF82A30ADF82C3099469E461A4698466E
:10B200000991634609A9002ED3D0CDE90290CDE97A
:10B2100000CE38461C49FFF789FF40460CB0BDE818
:10B22000F0871A4C84FB0234A318D417C4EB6314C0
:10B23000C4EB0415A2EB85052DB2002D0846B8BF5E
:10B240006D42FCF7F1FF4FF47A7200238046894685
:10B2500043F054FB3C230AFB030A4FF47A720023A9
:10B260004046494643F04AFB4FF47A7192B20023BC
:10B27000C1FB0A2309A8FCF71FFF24B209A975E73F
:10B28000B056050800000101905605088988888895
:10B2900010B44C09012250F8243001F01F0102FAC9
:10B2A00001F10B4340F824305DF8044B704700BFB8
:10B2B0004B0901F01F0150F82320012303FA01F18B
:10B2C000114214BF18460020704700BFF0EEC07A4C
:10B2D000B0EEE07AB4EEE77AF1EE10FAB4BFB0EE79
:10B2E000676AB0EE476AB5EE406AF1EE10FA46D0F2
:10B2F000B4EEE77AF1EE10FA8CBFF0EE675AF0EE9A
:10B30000475AC5EE866A9FED1F3A9FED1F6A9FED73
:10B310001F4A9FED1F5ADFED1F3ADFED1F4ADFED99
:10B320001F5AA6EEC36AE6EEA34AA6EE864AB7EE19
:10B33000006AA6EE845AA6EEA46AE6EE855AC5EE29
:10B34000866AB4EEE77AF1EE10FA48BFDFED147AC0
:10B35000F5EEC00A48BF77EEE66AF1EE10FA48BF94
:10B36000DFED107AB5EEC00A48BF77EEE66AF1EE7F
:10B3700010FA48BFF1EE666AB0EE660A7047DFED7C
:10B38000076ADEE739094E3DE3B59E3E88FA163E70
:10B3900045FE7F3F99FB243F69A2163EA7DFA834F4
:10B3A000DB0FC93FDB0F494070B544880546C4F345
:10B3B0000B04224608460E46002143F055FD2B693A
:10B3C000094A934202D3094A934205D35BB121460D
:10B3D0003046BDE870401847224630461946BDE861
:10B3E000704043F0DBBC70BD08070008520800083D
:10B3F00038B5064C064DAC4206D26168204614347E
:10B40000FFF7D2FFAC42F8D338BD00BF900100086F
:10B4100008070008084B09498B4203D309E014339D
:10B420008B4206D21A88C2F30B029042F7D118461B
:10B43000704700231846704790010008080700086D
:10B4400008B5064B186838B10CF0E6FC044B9B7845
:10B4500013B180F00100C0B208BD00BF2C5D002018
:10B460001C9B002008B538F017FE32F0E7FD1B20CA
:10B4700006F0C6FC18B1232200238271C37137F095
:10B48000F9FD18B1232200238271C3710C4B9B7804
:10B49000012B10D0022B0CD10A4B0B4A1A600B491E
:10B4A00001F12C0038F0F4FB094B002083F8230055
:10B4B00008BD012008BD034B064A1A60EFE700BF34
:10B4C0008085002010A5002034000020740000209A
:10B4D00000ED00E05400002008B5054B4FF0FF32AE
:10B4E0001A60012008F046FB72B643F029FC00BF49
:10B4F000F0FF012008B5FFF7A3FF0028FBD11420BF
:10B5000008F038FB00BFFFF79BFF0028FAD0FFF7D9
:10B51000E3FF00BF08B5054B1B6803B19847044B18
:10B52000044A1A6072B643F00BFC00BF106700209B
:10B53000F0FF01201010DDDD074A084B10781B7862
:10B54000074A834296BFC31AC3F1800300201268E2
:10B5500018441044704700BF106800208C6700201A
:10B5600018650020064A074B10781B7883428ABF73
:10B57000C3F18003C01AC018C0F17F00704700BF3C
:10B58000106800208C670020064808B54368DB6817
:10B59000984705480549064A002303700B7013605D
:10B5A00008BD00BFB0B80020106800208C670020E4
:10B5B0001865002038B504460D4600BF80680BF0C2
:10B5C000F1FC29466068FEF7A3FCA0680BF0F0FCD4
:10B5D00000BF38BDF0B5077F836983B004464FF0E4
:10B5E000020C002000900E4615468DF804008DF8E0
:10B5F00000C0002F34D01A0E8DF801200DEB0C0284
:10B60000180C1F0A93701070577006212046FEF721
:10B610008FFB06212068FFF7CDFF012363772368A6
:10B6200000BF98680BF0BEFC237F2268002B14BF7C
:10B6300005230423694650680022FEF725FB236892
:10B640003146002258682B46FEF71EFB2368986897
:10B650000BF0AEFC00BFA2692A44A26103B0F0BDAA
:10B660000DF10102CCE700BF10B4144681611A4607
:10B6700021465DF8044BADE710B5044645F20821BC
:10B68000FEF756FB20680621FFF794FF012363773E
:10B690002068C721BDE810408CE700BF10B5027FCD
:10B6A00082B000230446D82000938DF804308DF832
:10B6B00000002AB30B0E8DF801300DF102030A0AC7
:10B6C000080C997018705A7041F288312046FEF7C4
:10B6D0002FFB20680621FFF76DFF012363772468A5
:10B6E00000BFA0680BF05EFC69460523002260687D
:10B6F000FEF7CAFAA0680BF05BFC00BF02B010BDF9
:10B700000DF10103DBE700BF0348436813B19B6AF7
:10B7100003B1184701487047B0B80020100705086A
:10B720002DE9F04784B0FFF7EFFF8568ED0A1BD0E5
:10B73000DFF840800026C14604AFD8F80430AC19C9
:10B740006410D3F824A0E10210236A464846D0478B
:10B750000F2809DD6B4653F8042B013208D19F42B4
:10B76000F9D12546B542E8DCE80204B0BDE8F0872F
:10B77000661CF7E7B0B800202DE9F04F87B04FEA1C
:10B78000820A0491CDE9013000220B46514453F85E
:10B79000040B8B420244FAD1019B05922BB942481B
:10B7A00043681B689847002863D0FFF7ADFF4388C4
:10B7B0000393059B002B4AD03C4B029A3A4E1B68E0
:10B7C000DDF814B092440399B3FBF1F901FB19338E
:10B7D00003EB0B028A428CBFA1EB0309D946FFF7AA
:10B7E00093FF324B196883688B4248D973682E489F
:10B7F0001B6998477168029C049D4F46AC4655F8FA
:10B80000043B30461A468BB1D4F800E0D1F81480DE
:10B81000BB4271461FD2C04755F8042C236871689B
:10B82000134423600023BF1A45F8043C04345445F4
:10B83000E4D18B69304698471C4A13684B44136027
:10B84000019AABEB090B3AB3BBF1000FBBD10598E2
:10B8500007B0BDE8F08F4346E0463A469847226875
:10B86000D8F8003071683A44DF1B2260C8F80070D5
:10B87000DFE7019B0593059807B0BDE8F08F0598B9
:10B880000B490C4AA0EB0B000590059800230B70A8
:10B89000137007B0BDE8F08F059BA3EB0B03059376
:10B8A000059807B0BDE8F08FB0B8002018650020FB
:10B8B000106800208C67002070B5104D104E2B785A
:10B8C00031788B4284B016D00E4A03921A44029209
:10B8D0008CBF0C46CA1A04A98CBFC3F18002002495
:10B8E000012341F8102D02A802220194FFF744FF22
:10B8F000002333702B7004B070BD00BF8C67002034
:10B90000106800209067002010B5FFF7FDFE8368E7
:10B9100003B910BDFFF704FF0446FFF7CDFF014B4D
:10B920001C6010BD186500202DE9F0410546144645
:10B930000F46FFF7E9FE83682A199A4203D9FFF7F9
:10B94000E3FE8468641BFFF7B7FF0548466823469B
:10B95000746A3A462946A446BDE8F041604700BFF4
:10B96000B0B8002013460A4601461846DCE700BF7F
:10B970002DE9F04F012189B000200BF027FB38F0B2
:10B9800051F8FFF7C1FF41F62C720021BE48BF4DB0
:10B9900043F06AFA0024BC4B4C22291918191444AC
:10B9A00043F0FCF9E42CF6D1FFF7BAFE82460028FA
:10B9B00000F0B8800026B64FDFF8F0B235463446C6
:10B9C000122203A92846FFF7AFFF1222594603A807
:10B9D00043F076FA28BBAF4BAF49DFF8C48206EBE1
:10B9E000860206EB420203EB0209AC42A5EB04031C
:10B9F0004846019315D001363246FFF797FB019B6D
:10BA0000C7F80090C7E90433A44BFC600122642E00
:10BA1000C7E90733C7E90938BA6000F085804C37B9
:10BA20002C4605F50065AA45CAD8642EA04600F04C
:10BA30000A81A54272D006EB8602964C984B964935
:10BA4000019306EB420214442046721CFFF76EFB82
:10BA5000924A019B3C600121C7E90218C7E907220D
:10BA6000A5EB0805C7E904557A62351DBB620536AA
:10BA70004FF04C080193844B884FDFF8349208FB59
:10BA800005F55C1942460021204643F0EDF9424697
:10BA90000021204643F0E8F97B4B012243F8059052
:10BAA000019BA362A260C4E907776762FFF738FED3
:10BAB000C4E904004C27744B784DDFF8F88107FB8C
:10BAC00006F69C193A460021204643F0CDF93A4645
:10BAD0000021204643F0C8F96B490222012341F8B6
:10BAE00006800F46C4E9075565626271A360FFF7DF
:10BAF00017FEBD68C0F100604000C4E904000DB944
:10BB00003A79AAB94FF47A7008F034F8002108465F
:10BB10000BF05CFA002009B0BDE8F08FF51C002E98
:10BB200040F0E6800326C5E74346682667259FE781
:10BB30003B68002BE6D0FB6C3D64C7E91155FD6303
:10BB400043B3384629462A46466DC0F88C204C1E21
:10BB5000A6420346C0E92422C0F8882000F14C0028
:10BB600000F0AA804F1CBE426FD08E42CAD11C4644
:10BB70000029C7D0266CF76B0137F763C3F88C60D8
:10BB8000A064C36C002BDFD13F4B1C68002C00F07D
:10BB90009D801A793C4C002006460223114612E093
:10BBA000E16B236349011CBF01F6FF7107EB113301
:10BBB000C4E90D33C4E9046654F84C2F1946013525
:10BBC0000133E2B121795F1E0029E9D121692363A4
:10BBD000002944D001F6FF7107EB113261696263FD
:10BBE00019B101F6FF7307EB1333821AD018A36360
:10BBF00054F84C2F194601350133002AE2D1294B64
:10BC0000294ADA6001394FEA91794FEA81084022E6
:10BC10003E2498629A613F2058EA090259625D63A6
:10BC20004FEAC101C3E904401BD14231CC0D4D02A2
:10BC300042224120C3E90702134A9960C3E90B225B
:10BC4000C3E900545EE7164B6FE71C4621790029D3
:10BC50003FF458AF60643946C3F88C4091E71A4608
:10BC6000BCE740F2FF1418EB04064FF0000549EB67
:10BC70000507720A42EAC75202F140000244114429
:10BC8000CC0D4D02D6E700BF143200202007050876
:10BC9000F832002074290020F45605080068214C71
:10BCA00065B9000848BF002020570508E056050880
:10BCB000045705081457050800293FF423AF8E42A6
:10BCC0001C6C01D0314653E70F46BFE70A4B0B4EC1
:10BCD0005C633E253F2040224221C3E90502C3E9BF
:10BCE0000365C3E909440A464FF404454120A1E72E
:10BCF000034B0436BCE600BF48BF002020570508B0
:10BD000065B9000870B5194C194D23782978994206
:10BD100084B027D0174A03921A44029234BF0E46C9
:10BD2000CA1A04A934BFC3F180020026002341F8D7
:10BD3000102D02A802220196FFF71EFD2378184459
:10BD4000C0B203062B7848BF80F080008342207089
:10BD500002D0002004B070BD002301202B7023709E
:10BD600004B070BD012004B070BD00BF8C6700201E
:10BD7000106800209067002008B5FFF7C5FC8068B8
:10BD8000003018BF012008BD08B5FFF7BDFC806872
:10BD900000B908BD024843681B68984708BD00BF4A
:10BDA000B0B800202DE9F047A84F3B7803B1FEE77B
:10BDB000A74EB36801223A7013B11A689B88538367
:10BDC000A44B01228A461A70014640F2E93370689A
:10BDD00002E0002B00F07C810289013B12F0020F8F
:10BDE0009BB2F6D00023838140F2E93302E0002BBE
:10BDF00000F06E810289013B12F0010F9BB2F6D078
:10BE0000838940F2E93302E0002B00F0758102895A
:10BE1000013B12F0020F9BB2F6D00023838140F267
:10BE2000E93302E0002B00F067810289013B12F048
:10BE3000010F9BB2F6D0838940F2E93302E0002B78
:10BE400000F056810289013B12F0020F9BB2F6D03E
:10BE50000923838140F2E93302E0002B00F048819E
:10BE60000289013B12F0010F9BB2F6D0838940F2A8
:10BE7000E93302E0002B00F037810289013B12F028
:10BE8000020F9BB2F6D089B2818140F2E93302E021
:10BE9000002B00F029810289013B12F0010F9BB2B7
:10BEA000F6D08389DFF8B0810AF1FF3A00244FF021
:10BEB0000A090B2540F2E93302E0002B00F0E6808E
:10BEC0000289013B12F0020F9BB2F6D0A0F80C9051
:10BED00040F2E93302E0002B00F0D8800289013BF8
:10BEE00012F0010F9BB2F6D0838940F2E93302E0F1
:10BEF000002B00F0D7800289013B12F0020F9BB2A9
:10BF0000F6D0A3B2838140F2E93302E0002B00F0C7
:10BF1000C9800289013B12F0010F9BB2F6D08389E0
:10BF20001AF8011F40F2E93302E0002B00F0B28062
:10BF30000289013B12F0020F9BB2F6D0858140F2DC
:10BF4000E93302E0002B00F0A5800289013B12F0EA
:10BF5000010F9BB2F6D0838940F2E93302E0002B57
:10BF600000F09C800289013B12F0020F9BB2F6D0D8
:10BF700089B2818140F2E93302E0002B00F08E802B
:10BF80000289013B12F0010F9BB2F6D08389D8F8E9
:10BF9000003033B11A689B8851690B4214BF538338
:10BFA00013830134362C85D140F2E93302E0002BB3
:10BFB00000F096800289013B12F0020F9BB2F6D08E
:10BFC0000823838140F2E93302E0002B00F08880EF
:10BFD0000289013B12F0010F9BB2F6D0838940F237
:10BFE000E93301E0002B77D00289013B12F0020F08
:10BFF0009BB2F7D0A023838140F2E93301E0002B0C
:10C000006AD00289013B12F0010F9BB2F7D08389FD
:10C01000A024002140F2E93301E0002B46D0028940
:10C02000013B12F0020F9BB2F7D0848140F2E9335A
:10C0300001E0002B3AD00289013B12F0010F9BB2C4
:10C04000F7D0838940F2E93309E000BF7364002030
:10C0500008B600207464002060B6002053B3028943
:10C06000013B12F0020F9BB2F8D0818140F2E9331C
:10C0700000E0FBB10289013B12F0010F9BB2F8D046
:10C080008089C0B283061AD57068C3E7FDF7DAFD70
:10C0900070682AE7FDF7D6FD70685DE7FDF7D2FD11
:10C0A000706874E7FDF7CEFD706839E7FDF7CAFDEB
:10C0B0007068C7E7FDF7C6FDC0B28306E4D4B36875
:10C0C00013B11A689B88138300233B70BDE8F08787
:10C0D000FDF7B8FD706894E6FDF7B4FD706897E76A
:10C0E000FDF7B0FD70687AE7FDF7ACFD7068D9E642
:10C0F000FDF7A8FD7068BAE6FDF7A4FD70689BE641
:10C1000038B51E4D40F2E9326B6800E05AB31C8925
:10C11000013A14F0020F92B2F8D080B2988140F246
:10C12000E93200E0FAB11889013A10F0010F92B239
:10C13000F8D09A8940F2E93200E0CAB11889013A90
:10C1400010F0020F92B2F8D089B2998140F2E93230
:10C1500000E06AB11989013A11F0010F92B2F8D0EA
:10C160009889C0B238BD1846FDF76CFD6B68E1E7F1
:10C170001846FDF767FDC0B238BD00BF08B6002005
:10C180002DE9F84FDFF828A4DAF8083013B11A685F
:10C190009B885383DAF8040040F2E93302E0002B75
:10C1A00000F089820289013B12F0020F9BB2F6D0A7
:10C1B0000523838140F2E93302E0002B00F07B820B
:10C1C0000289013B12F0010F9BB2F6D0838940F245
:10C1D000E93302E0002B00F069820289013B12F092
:10C1E000020F9BB2F6D00023838140F2E93302E0D4
:10C1F000002B00F05B820289013B12F0010F9BB221
:10C20000F6D0838940F2E93302E0002B00F0678228
:10C210000289013B12F0020F9BB2F6D00623838104
:10C2200040F2E93302E0002B00F059820289013B21
:10C2300012F0010F9BB2F6D0838940F2E93302E09D
:10C24000002B00F047820289013B12F0020F9BB2E3
:10C25000F6D00023838140F2E93302E0002B00F0A6
:10C2600039820289013B12F0010F9BB2F6D083891B
:10C27000DFF8409399F8681540F2E93341F0010482
:10C2800002E0002B00F021820289013B12F0020F34
:10C290009BB2F6D00423838140F2E93302E0002B05
:10C2A00000F013820289013B12F0010F9BB2F6D01D
:10C2B000838940F2E93302E0002B00F00182028919
:10C2C000013B12F0020F9BB2F6D0A4B2848140F27F
:10C2D000E93302E0002B00F0F3810289013B12F008
:10C2E000010F9BB2F6D08389AE4D2B88002B49D02D
:10C2F000DFF8C4B2AC4F5E464FF02008072417F8B1
:10C30000011FFF2940F2E93303D17AE1002B00F04D
:10C31000A6810289013B12F0020F9BB2F6D0848104
:10C3200040F2E93302E0002B00F099810289013BE1
:10C3300012F0010F9BB2F6D0838940F2E93302E09C
:10C34000002B00F087810289013B12F0020F9BB2A3
:10C35000F6D089B2818140F2E93302E0002B00F08F
:10C3600079810289013B12F0010F9BB2F6D08389DB
:10C370003B7806F8013B2A88A6EB0B039A42BEDC09
:10C3800099F8681540F2E93302E0002B00F0B9811A
:10C390000289013B12F0020F9BB2F6D00723838182
:10C3A00040F2E93302E0002B00F0AB810289013B4F
:10C3B00012F0010F9BB2F6D0838940F2E93302E01C
:10C3C000002B00F099810289013B12F0020F9BB211
:10C3D000F6D0FF23838140F2E93302E0002B00F026
:10C3E0008B810289013B12F0010F9BB2F6D0838949
:10C3F00040F2E93302E0002B00F079810289013B31
:10C4000012F0020F9BB2F6D00423838140F2E9338D
:10C4100002E0002B00F06B810289013B12F0010F5A
:10C420009BB2F6D0838940F2E93302E0002B00F0A2
:10C430005B810289013B12F0020F9BB2F6D089B2F8
:10C44000818140F2E93302E0002B00F04D81028946
:10C45000013B12F0010F9BB2F6D083892B88002B91
:10C4600000F0C680514C0021FF27072603E0013170
:10C470008B4240F3BD8014F8012BFF2AF7D14FEA1D
:10C480002128DAF8040040F2E93302E0002B00F042
:10C4900008810289013B12F0020F9BB2F6D00523FE
:10C4A000838140F2E93302E0002B00F0FA80028938
:10C4B000013B12F0010F9BB2F6D0838940F2E933C1
:10C4C00002E0002B00F0E8800289013B12F0020F2D
:10C4D0009BB2F6D01FFA88F8A0F80C8040F2E9333E
:10C4E00002E0002B00F0D8800289013B12F0010F1E
:10C4F0009BB2F6D083895FFA81F840F2E93302E01B
:10C50000002B00F0C4800289013B12F0020F9BB2A5
:10C51000F6D00623838140F2E93302E0002B00F0DD
:10C52000B6800289013B12F0010F9BB2F6D08389DD
:10C5300040F2E93302E0002B00F0A4800289013BC5
:10C5400012F0020F9BB2F6D01FFA88F8A0F80C8008
:10C5500040F2E93302E0002B00F094800289013BB5
:10C5600012F0010F9BB2F6D0838940F2E93302E06A
:10C57000002B00F082800289013B12F0020F9BB277
:10C58000F6D0868140F2E93301E0002B75D00289B4
:10C59000013B12F0010F9BB2F7D0838940F2E933DF
:10C5A0000EE000BF7C010020535E0020545E00209E
:10C5B00008B6002058280020C42D0020002B58D099
:10C5C0000289013B12F0020F9BB2F7D0878140F243
:10C5D000E93301E0002B4CD00289013B12F0010F3E
:10C5E0009BB2F7D083892B8801318B423FF743AF51
:10C5F000DAF8083013B11A689B881383BDE8F88F06
:10C6000093B30289013B12F0020F9BB2F8D08481F0
:10C6100040F2E93300E03BB30289013B12F0010F25
:10C620009BB2F8D0838940F2E93300E093B10289EC
:10C63000013B12F0020F9BB2F8D0A0F80C8040F240
:10C64000E93300E033B10289013B12F0010F9BB2E4
:10C65000F8D08CE6FDF7F6FADAF8040088E6FDF784
:10C66000F1FADAF8040068E6FDF7ECFADAF804000B
:10C67000D9E7FDF7E7FA2B88F9E6FDF7E3FADAF8F0
:10C6800004008BE7FDF7DEFADAF804006DE7FDF74A
:10C69000D9FADAF804004BE7FDF7D4FADAF8040027
:10C6A00029E7FDF7CFFADAF8040007E7FDF7CAFA41
:10C6B000DAF80400A6E5FDF7C5FADAF8040086E525
:10C6C000FDF7C0FADAF804000EE6FDF7BBFADAF877
:10C6D0000400EEE5FDF7B6FADAF80400C8E5FDF768
:10C6E000B1FADAF80400A8E5FDF7ACFAB6E6FDF712
:10C6F000A9FADAF8040096E6FDF7A4FADAF80400DD
:10C7000076E6FDF79FFADAF8040056E6F8B59B4C9A
:10C71000A36813B11A6899885183994A606812789E
:10C72000012A00F08081C0F06381022A00F052816A
:10C7300094490A7812F0400F0CBF4FF4C3724FF4C3
:10C74000F072914D2A8013B11A689B88538310268A
:10C75000012740F2E93302E0002B00F04181028919
:10C76000013B12F0020F9BB2F6D0B3B2838140F2CC
:10C77000E93302E0002B00F033810289013B12F023
:10C78000010F9BB2F6D0838940F2E93302E0002B1F
:10C7900000F02A810289013B12F0020F9BB2F6D011
:10C7A000878140F2E93302E0002B00F01D8102890D
:10C7B000013B12F0010F9BB2F6D083890136202E87
:10C7C000C7D1A3681BB11A689B8813835383097868
:10C7D00040F2E93302E0002B00F02E810289013B98
:10C7E00012F0020F9BB2F6D00023838140F2E933AE
:10C7F00002E0002B00F020810289013B12F0010FC2
:10C800009BB2F6D0838940F2E93302E0002B00F0BE
:10C8100017810289013B12F0020F9BB2F6D089B258
:10C82000818140F2E93302E0002B00F009810289A6
:10C83000013B12F0010F9BB2F6D08389534A40F2BC
:10C84000E933117802E0002B00F0FE800289013B01
:10C8500012F0020F9BB2F6D00223838140F2E9333B
:10C8600002E0002B00F0F0800289013B12F0010F82
:10C870009BB2F6D0838940F2E93302E0002B00F04E
:10C88000E7800289013B12F0020F9BB2F6D089B219
:10C89000818140F2E93302E0002B00F0D980028967
:10C8A000013B12F0010F9BB2F6D08389384A40F267
:10C8B000E933117802E0002B00F0CE800289013BC1
:10C8C00012F0020F9BB2F6D00323838140F2E933CA
:10C8D00002E0002B00F0C0800289013B12F0010F42
:10C8E0009BB2F6D0838940F2E93302E0002B00F0DE
:10C8F000B7800289013B12F0020F9BB2F6D089B2D9
:10C90000818140F2E93302E0002B00F0A980028926
:10C91000013B12F0010F9BB2F6D083891D4B93F8B7
:10C92000681540F2E93341F0040102E0002B00F009
:10C930009B800289013B12F0020F9BB2F6D00423C8
:10C94000838140F2E93302E0002B00F08D80028900
:10C95000013B12F0010F9BB2F6D0838940F2E9331C
:10C9600001E0002B65D00289013B12F0020F9BB25F
:10C97000F7D089B2818140F2E9330FE008B6002098
:10C9800054B60020690300207C0100205BB6002023
:10C990005CB6002058280020002B4AD00289013BB9
:10C9A00012F0010F9BB2F7D08389A36813B11A6804
:10C9B0009B8813832E4C2A882E48002142F054FA7B
:10C9C00094F8BC3003B9F8BDFFF7DAFB002384F814
:10C9D000BC30F8BD284908220A704FF4C372B0E693
:10C9E000FDF730F96068CFE6FDF72CF96068E5E601
:10C9F000A021FDF78DFA00216068FDF789FA00F0AB
:10CA00000603022B09D000F00500012805D11A49C0
:10CA10004822D4E901030A7008E017490822D4E942
:10CA200001030A70D9E7144948220A704FF4F072E2
:10CA300087E6FDF707F9B8E7FDF704F96068E2E675
:10CA4000FDF700F96068F9E6FDF7FCF8606812E7A9
:10CA5000FDF7F8F8606829E7FDF7F4F8606842E749
:10CA6000FDF7F0F8606859E7FDF7ECF8606875E7E6
:10CA700000000020C42D0020690300202DE9F041B2
:10CA8000574CA36813B11A689B885383606840F2BF
:10CA9000E93301E0002B4BD00289013B12F0020F79
:10CAA0009BB2F7D08023838140F2E93301E0002B71
:10CAB0003ED00289013B12F0010F9BB2F7D083896F
:10CAC00040F2E93301E0002B2ED00289013B12F045
:10CAD000020F9BB2F7D00023838140F2E93300E0DC
:10CAE00013B30289013B12F0010F9BB2F8D0808989
:10CAF000C0B2A36813B11A6899881183394D3A4EB0
:10CB00002A78376882420CD1384A12783AB9DFF86D
:10CB1000E880D8F84C27BA1AB2F57A7F0CD8BDE86D
:10CB2000F081BDE8F041F1E5FDF78CF8C0B2E0E737
:10CB3000FDF788F86068C3E713B11A689B885383D0
:10CB4000A0216068FDF7E4F900216068FDF7E0F9D5
:10CB5000A36813B11A689B881383254C2378182B7C
:10CB60000FD12B78234A03F04003002B00F007017C
:10CB70000CBF4FF00D0C4FF0100C13805180A2F839
:10CB800006C0410706D50023C8F85037C8F84C77CF
:10CB9000BDE8F08100F00500012819D00028F5D18A
:10CBA0002B785B06F2D5D8F850273368A2B19B1AD0
:10CBB000642BEBD9FFF7AAFD2378182BE6D1B8F840
:10CBC00054370C4A01339BB2A8F854379380DDE701
:10CBD0002B785A06E7D5D9E7C8F85037D6E700BF13
:10CBE00008B600206903002094B6002054B6002047
:10CBF00049B600204CB60020582800202DE9F84FF7
:10CC00002E4A2F4E01231370FFF738FFB6F8562730
:10CC10002C4BDFF8BCE0B3F8008002F1640C1FFA83
:10CC20008CFC00234FF0050B4FF0060A4FF007096C
:10CC300001E062453ED0B4181EF8020094F86C156D
:10CC4000814202F1010503F1050111D07718F118B5
:10CC500084F86C05140A81F858B781F85AA781F84E
:10CC60005B2781F85C9781F85947063387F85807A6
:10CC7000AAB24245DDD30022A6F8562723B90F4AAF
:10CC800000231370BDE8F88F0F4CA26812B1116831
:10CC900092884A8300220D496068FCF7F5FFA3687B
:10CCA000002BECD01A689B881383044A002313706E
:10CCB000BDE8F88FA6F85627E0E700BF73640020B0
:10CCC000582800207C01002008B60020B02F00204A
:10CCD000545E00200F4B10B41C889CB10E4B0F4AC1
:10CCE000187892F86C15884210D11C4402F26C52EC
:10CCF000013305E013F8011B12F8010F884205D13A
:10CD0000A342F7D101205DF8044B704700205DF885
:10CD1000044B70477C010020545E002058280020FE
:10CD20001378C3B130B41E240B4D14FB0101294408
:10CD3000801A84181D2C07DC01F8013B12F8013F12
:10CD4000002BF6D130BC704712F8013F0131002BA7
:10CD5000EFD130BC70477047545E002038B5264C88
:10CD6000C1F10301A36841EA8005EDB213B11A686D
:10CD70009B885383ADB21021606840F2E93301E033
:10CD8000002B31D00289013B12F0020F9BB2F7D089
:10CD90008BB2838140F2E93300E02BB30289013B7F
:10CDA00012F0010F9BB2F8D0838940F2E93300E022
:10CDB000F3B10289013B12F0020F9BB2F8D08581DA
:10CDC00040F2E93300E09BB10289013B12F0010F10
:10CDD0009BB2F8D0838901312029CDD1A36813B14A
:10CDE0001A689B88138338BDFCF72CFF6068DCE76A
:10CDF000FCF728FFEFE700BF08B6002010B5274B6F
:10CE000093F8684500283FD104F0F704244983F8DB
:10CE100068458B6813B11A689B885383486840F251
:10CE2000E93301E0002B35D00289013B12F0020FFB
:10CE30009BB2F7D00423838140F2E93300E04BB387
:10CE40000289013B12F0010F9BB2F8D0838940F2B6
:10CE5000E93300E0DBB10289013B12F0020F9BB223
:10CE6000F8D0A4B2848140F2E93300E07BB10289BA
:10CE7000013B12F0010F9BB2F8D083898B6813B18C
:10CE80001A689B88138310BD44F00804BEE7FCF7C2
:10CE9000D9FEF3E7FCF7D6FE4868D8E7582800200B
:10CEA00008B60020144B984223D003F580639842C3
:10CEB0001FD0038823F040031B041B0C038003884E
:10CEC00023F038031B041B0C69B141F48071002965
:10CED00091FAA1F1B1FA81F108BF4FF0FF310139A8
:10CEE00043EAC1039BB20380038843F040030380FD
:10CEF00070474908DDE700BF003800400B4A0C4B83
:10CF000090421B6810D0A2F5806290420CD002F5CE
:10CF10008042904208D002F58062904204D002F52F
:10CF20008062904218BF5B081846704700040140B9
:10CF300064DA0020F0B587B000236A4A00930193B9
:10CF4000136843F48033136003E0009BB3F5A04FF4
:10CF500009D0136803F400330193009B013300935D
:10CF6000019B002BF1D05F4B1B6813F4003318BFFB
:10CF700001230193019B012B75D05B4D594B5B4AFB
:10CF8000EA605B49586F5B4A0860AA605E6B5A4C66
:10CF90005A4F5B4A5B4826F080065E635E6F46F040
:10CFA00080765E67196B0C431C63596B5963996BF0
:10CFB0009963196C39431964596C06AC0A4348F2F9
:10CFC000FF715A6444F8101D0123002621468DF894
:10CFD0000F304FF6FF778DF80C608DF80D608DF8EF
:10CFE0000E6034F075FE21464748029734F070FE1B
:10CFF00021464648029734F06BFE2146444834F0FF
:10D0000067FE2146434834F063FE2146424834F02F
:10D010005FFE2146414834F05BFE2146404834F033
:10D0200057FE21463F4834F053FE204634F088FA3C
:10D030003D4B3E4C1B68029A3D483E49A4FB0343CE
:10D040009B09A0FB0202013B920CB3F1807F0A60B6
:10D0500007D2394AF0200721536085F823009660F3
:10D06000116007B0F0BD1F4B344C1A6C344942F0CC
:10D0700080521A64206840F44040D1E93052D1F81F
:10D08000C8102060986898609868120640F40040C4
:10D09000986042EA8512986842F48002490842F09A
:10D0A0000802013942EA014240F4A05098605A60F7
:10D0B0001A6842F080721A601A689201FCD5214900
:10D0C000084A40F205700860996821F003019960F0
:10D0D000996841F002019960936803F00C03082BF2
:10D0E000FAD14AE70038024000ED00E00005FA05F9
:10D0F00098DA002000000008FF916700FFC9FE36A3
:10D10000335F0700000002400004024000080240B4
:10D11000000C0240001002400014024000180240BF
:10D12000001C02400020024064DA0020D34D62104F
:10D1300083DE1B4398B6002010E000E00070004042
:10D1400000000020003C0240074A08B51168074B68
:10D15000994208D1064B00201968106081F30888B5
:10D160005B689847FEE708BDD00B0120EFBEADDE3F
:10D170000000FF1F08B5054B1B6803B19847044B1F
:10D18000044A1A6072B641F0DBFD00BF1067002050
:10D19000D00B0120EFBEADDE08B5034B1B6803B119
:10D1A000984772B641F0CCFD10670020074A002373
:10D1B00002E00133102B07D05168814202F12002B6
:10D1C000F7D1581CC0B27047002070479C25002042
:10D1D00038B50121002502223123044641708270B6
:10D1E00003710570C57045710248FFF7DFFFE571F7
:10D1F000A07138BDB86002400138F0B540013C4C28
:10D20000DFF820C125583B4FDCF83060BD420CBF31
:10D210004FF400154FF4800527182E437D68CCF895
:10D220003060354EF960B54283B07B6151D0334BED
:10D230009D424ED0A3F57A739D4236D003F58063AC
:10D240009D4232D0A3F57A739D4246D003F58063A8
:10D250009D4242D0A3F57A739D4240D003F580638E
:10D260009D423CD0A3F57A739D4234D003F5806390
:10D270009D4230D0A3F57A739D4232D003F580638E
:10D280009D422ED0A3F57A739D422CD003F5806386
:10D290009D4228D0A3F57A739D4226D01849194B98
:10D2A0008D420CBF1D46002500E0174D0444920935
:10D2B000667CE5610021012301A88DF804608DF8EA
:10D2C00005208DF806108DF8073033F05DFF03B0B0
:10D2D000F0BD0E4DEAE70E4DE8E70E4DE6E70E4DC8
:10D2E000E4E70E4DE2E70E4DE0E7064DDEE700BF56
:10D2F0009C25002000600240106002401064024043
:10D30000B8640240008000280088001020800010CF
:10D31000208000200080201000800018008800205D
:10D3200000802020003802400138F0B44401094850
:10D33000094D0359094F2E6B2044BB420CBF4FF4DB
:10D3400000134FF4800333432B6301764276F0BC25
:10D35000704700BF9C25002000380240006002405A
:10D360002DE9F04F534C54F8204083B0002C00F0CE
:10D370009C80656E002D00F09A809846174604F157
:10D380006A034D4A064628692260636104F1EA0295
:10D390008023A261E3604FF480726B68A160226118
:10D3A000E365A24668B1FFF701FF721CD2B20C21FF
:10D3B000FFF7BAFFE36DA9682A69A2630433216409
:10D3C000A365E868A0B1FFF7F1FE721C8146D2B2F6
:10D3D0000B21FFF7A9FF2346EA7F38494846FFF7AC
:10D3E0000BFFD5E90212E36D616404336365E26308
:10D3F00094F8690004F004FD814694F8680004F094
:10D40000FFFC8346287F00284CD118F0080F36D146
:10D41000BA070DD5B9F1000F0AD00B22731C89F899
:10D42000062089F8073048466A7F222104F082FBF3
:10D43000FB0715D4236C7BB995F82020A97F8DF8C4
:10D44000063001A8930901228DF805308DF80410EB
:10D450008DF8072033F098FE504603B0BDE8F08FFA
:10D46000BBF1000FE6D0701C0C238BF807008BF883
:10D47000063058466A7F222104F05CFBDAE7B9F1F6
:10D48000000F05D0701C0B2389F8070089F80630BF
:10D4900018F0100F484614BF022112216A7F04F0D1
:10D4A00049FBC7E735F058FDAFE7A246D4E7AA46E7
:10D4B000D2E700BF3C0A00109C0805088D8A0008CE
:10D4C0000348D0F8EC3113B100F5F07018477047FD
:10D4D0009C2500200348D0F8CC3113B100F5E07052
:10D4E000184770479C2500200348D0F8AC3113B191
:10D4F00000F5D070184770479C2500200348D0F8ED
:10D500008C3113B100F5C070184770479C2500207E
:10D510000348D0F86C3113B100F5B070184770476C
:10D520009C2500200348D0F84C3113B100F5A070C1
:10D53000184770479C2500200348D0F82C3113B1C0
:10D5400000F59070184770479C2500200348D0F8DC
:10D550000C3113B100F58070184770479C250020EE
:10D560000348D0F8EC300BB1E0301847704700BFEB
:10D570009C2500200348D0F8CC300BB1C0301847B0
:10D58000704700BF9C2500200348D0F8AC300BB199
:10D59000A0301847704700BF9C2500200348D0F8F2
:10D5A0008C300BB180301847704700BF9C2500209D
:10D5B0000248C36E0BB16030184770479C250020AD
:10D5C0000248C36C0BB14030184770479C250020BF
:10D5D0000248C36A0BB12030184770479C250020D1
:10D5E0000248C36803B11847704700BF9C2500205C
:10D5F00003899B0746BF0089C0F3C0100120704714
:10D60000F8B50401654D664B2A5929199A4205EB74
:10D61000040704BF01230B730646387A35F09CFCDF
:10D620003B7A03F01F015B090122032B02FA01F28E
:10D630006DD0042B66D0022B5CD02B1901361879E3
:10D6400004F0DEFBF6B2074610B11223C6718371F7
:10D650002B19587904F0D4FB10B11323C6718371D0
:10D660002B19987904F0CCFB10B11423C671837187
:10D670002E190A21F279384604F05CFA707904F028
:10D68000BFFBF2790A2104F055FAB07904F0B8FB37
:10D69000F2790A2104F04EFA2B59424A934246D0BD
:10D6A000414A93424ED03E4A934256D03F4A93421B
:10D6B0005ED03F4A93422FD03E4A934263D02B190B
:10D6C0001B7BE3B9012002222B59198801F4415137
:10D6D00041F445710A4302431A809A8B22F4006296
:10D6E0001204120C07219A8319821A8842F0400210
:10D6F0001A80F8BD304B596A0A435A629DE70020F0
:10D700000246E1E72C4B19690A431A6195E72A4B57
:10D71000196A0A431A6290E702F568424FF48010D2
:10D72000536A43F48013536233F04CFEC7E702F5AB
:10D7300084324FF48050536A43F48053536233F081
:10D7400041FEBCE702F500324FF48040136A43F417
:10D750008043136233F03EFEB1E702F5FE324FF430
:10D760000040136A43F40043136233F033FEA6E72C
:10D7700002F582324FF40050536A43F4005353626F
:10D7800033F020FE9BE702F564424FF40010536A29
:10D7900043F40013536233F015FE90E718B60020EF
:10D7A000003C00400030014000380040003401409F
:10D7B000005001400054014000380240431C00F07A
:10D7C00005812DE9F04F4FEAC00B0BEB00039B00E6
:10D7D000DFF85C8258F803A087B008EB0304BAF1C5
:10D7E000000F00F0F080143308EB03010022DAF898
:10D7F000047048F80320C1E90122CA60D4E9025943
:10D80000431CDBB215B11522EB71AA71B9F1000FFF
:10D8100004D0162289F8073089F8062001909AF87A
:10D82000180035F099FBBB8823F440731B041B0CD4
:10D83000BB80284609F0BCFB484609F0B9FB112122
:10D84000284609F013FB1121484609F00FFB092671
:10D85000332405E0013C4FF00A0006D006F02CF915
:10D8600028460AF0D9FA0028F4D0284609F09AFB95
:10D87000052006F021F9284609F09AFB052006F05C
:10D880001BF9013EE4D1284609F08CFB052006F087
:10D8900013F9484609F086FB052006F00DF92846E5
:10D8A00009F086FB052006F007F9484609F080FBE1
:10D8B000019B0BEB030408EB84042846E37C227CE9
:10D8C000002B0CBF1221322104F034F9E37C627C7E
:10D8D000002B0CBF12213221484604F02BF94B4B90
:10D8E0009F4274D04A4B9F4200F08580494B9F4233
:10D8F00077D0BB88484A494C23F440731B041B0C67
:10D90000BB80019B9B443B8808EB8B0843F00103E1
:10D9100098F812103B80BD8802A8002918BF144651
:10D9200033F00EFE049A3E48B2FBF4F325F03F05B7
:10D93000A0FB02122D04900C2D0C0543BD803988EC
:10D94000384C4FF496729BB202FB00F2002BA4FB02
:10D95000020221F0010108BF01239209090443F4E6
:10D9600000430132090C39803A84BB833A882E4B3C
:10D9700042F001023A803A88134043F480634FF446
:10D9800080423B803A813B8823F080031B041B0CC0
:10D990003B809AF81A308DF808300024012302A841
:10D9A0008DF80B308DF809408DF80A4033F0ECFB10
:10D9B0009AF819308DF8083002A88DF809408DF8D2
:10D9C0000A4033F007FC07B0BDE8F08F7047174AF4
:10D9D000136A43F4001313624FF4001033F0FAFC9F
:10D9E00087E7124A136A43F4000313624FF40000FE
:10D9F00033F0F0FC7DE70D4A136A43F480031362B1
:10DA00004FF4800033F0E6FC73E700BF00540040A1
:10DA100000580040005C0040009F2400804F12002E
:10DA200083DE1B43D34D6210F5FBFFFF003802403D
:10DA3000305D00202DE9F0410578012D82B00646C9
:10DA40002FD0022D33D1806841F0800110B10468DD
:10DA500080886083706840F2E93401E0002C6FD068
:10DA60000589013C15F0020FA4B2F7D089B281817B
:10DA700040F2E93101E0002962D00489013914F053
:10DA8000010F89B2F7D081890021FCF7FDF8B36856
:10DA9000002B53D01A689B881383012002B0BDE885
:10DAA000F08190F90400441C01D0032803DD00201C
:10DAB00002B0BDE8F0814FEAC00EDFF8BCC00EEB4B
:10DAC00000070CEB87077C68002C48D076793A6217
:10DAD00076004FF00008F6B2BE75F97587F8198028
:10DAE000BD763B767D7587F81480A388FA61990529
:10DAF00012D42388DA050BD44FF4805501E0013DA0
:10DB00002FD023889B05FAD4238843F48073238085
:10DB1000A38843F44073A38086440CEB8E024FF439
:10DB2000805401E0013C13D0537D002BFAD10CEB63
:10DB30008E0E9EF8140080F00100B9E70120B7E7CF
:10DB4000CDE90023FCF77EF87068DDE900239BE750
:10DB5000084A138801339BB21380FFF72FFE20463B
:10DB6000A6E7044A138801339BB21380FFF726FE11
:10DB700028469DE7628E0020305D00207FB500259D
:10DB800000F10C060C460D804D808D8001230DF1B7
:10DB9000070206213046FFF74DFF10B9002004B000
:10DBA00070BD9DF807305B07F8D5062302AA294609
:10DBB0003046FFF73FFF0028F0D09DF809209DF880
:10DBC000083043EA022323809DF80B209DF80A3099
:10DBD00043EA022363809DF80D209DF80C3043EA50
:10DBE0000223A380DBE713B506230C466A46032114
:10DBF0000C30FFF71FFFA0B19DF800209DF8013009
:10DC000043EA022323809DF802209DF8033043EA73
:10DC10000223A3809DF804209DF8053043EA0223E7
:10DC2000638002B010BD07B5032301AA0021FFF7EE
:10DC300001FF9DF805309DF804001B0243EA0043F4
:10DC40009DF80600184303B05DF804FB08B5FFF724
:10DC5000EAFF014B586008BD5828002008B5FFF7BF
:10DC6000E2FF014B186008BD5828002007B50623C5
:10DC70006A46F721FFF7DEFE9DF801309DF800109F
:10DC80000B4A1B0143EA01339DF8021043EA1113CA
:10DC9000D3609DF804309DF803101B0143EA013363
:10DCA0009DF8051043EA1113936003B05DF804FB7F
:10DCB0005828002007B5032301AAF621FFF7BAFE72
:10DCC0009DF805309DF804201B0243EA02439DF8AD
:10DCD00006201343054AB2F92020C2F10802D340BE
:10DCE000034A536103B05DF804FB00BF7068002075
:10DCF0005828002007B5022301AAF621FFF79AFE53
:10DD00009DF804209DF8053043EA0223024A13825D
:10DD100003B05DF804FB00BF5828002070B582B046
:10DD20000446062310306A464321FFF783FEC0B144
:10DD30009DF804009DF800609DF801109DF80250C8
:10DD40009DF803209DF8053041EA062143EA0023AF
:10DD500042EA0522A4F85010A4F85220A4F8543046
:10DD6000012002B070BD00BF2DE9F04F90F8653082
:10DD700085B00546002B40F05184874B686993F8C5
:10DD8000B039002B00F0B080844B984200F034840E
:10DD900003F58063984200F02F84038823F040034A
:10DDA0001B041B0C0380038823F038031B041B0C8B
:10DDB000382213430380038843F04003038095F81F
:10DDC0005F30032B00F28E8095F86210012900F07D
:10DDD0003786A1F10201B1FA81F14909AB6913B1AA
:10DDE0001A689B88538340F2E93304E0013B9BB2FD
:10DDF000002B00F0938702899707F7D51A238381B8
:10DE000040F2E93304E0013B9BB2002B00F086872F
:10DE10000289D607F7D5838940F2E93304E0013B54
:10DE20009BB2002B00F0768702899407F7D5818199
:10DE300040F2E93304E0013B9BB2002B00F06A871B
:10DE40000289D107F7D58389AB6913B11A689B881A
:10DE50001383012005F030FE6A69504B9A4200F0AE
:10DE6000D88503F580639A4200F0D385138823F0A8
:10DE700040031B041B0C1380138823F038031B047E
:10DE80001B0C08210B431380138843F040031380BD
:10DE90004321062302AA05F11000FFF7CBFD00285D
:10DEA00000F0FE849DF80A609DF80B309DF8084054
:10DEB0009DF809109DF80C009DF80D2043EA0623FB
:10DEC0001BB2A5F852305BB241EA042142EA0022BB
:10DED0000133A5F85010A5F8542000F0E78405B0F0
:10DEE000BDE8F08F002179E72C4B984200F01B87AA
:10DEF00003F58063984200F01687038823F04003FF
:10DF00001B041B0C0380038823F038031B041B0C29
:10DF10004FF4807242F48072002A92FAA2F2B2FAAE
:10DF200082F208BF4FF0FF32013A43EAC2039BB2CC
:10DF300003800288AB6942F04002028013B11A6884
:10DF40009B88538340F2E93304E0013B9BB2002BF2
:10DF500000F0F78602899707F7D56B23838140F29B
:10DF6000E93304E0013B9BB2002B00F0EA86028912
:10DF7000D607F7D5838940F2E93304E0013B9BB231
:10DF8000002B00F0B18602899407F7D580238381A6
:10DF900040F2E93309E000BF582800200038004073
:10DFA000013B9BB2002B00F09F860289D107F7D579
:10DFB0008389AB6913B11A689B881383A44CDFF87B
:10DFC0009CA2DFF89C82A34EDFF898C2A24F4FF0CC
:10DFD000960BD8F80430C3F30803002B40F03886C2
:10DFE000EFF31183002B40F033862068B26823687A
:10DFF0009842FAD13B689A42F7D8DAF800E04FF439
:10E000007A7101FB0EF39B1AB3FBFEF301FB0030A8
:10E010004FF47A7ED8F80430C3F30803002B40F0A5
:10E020009E85EFF31183002B40F099852368B1683A
:10E0300022689342FAD13A689142F7D8DAF8009010
:10E040000EFB09F2521AB2FBF9F20EFB03231B1A64
:10E05000B3F57A7FDED3BBF1010BBAD1AB6913B153
:10E060001A689B885383686940F2E93304E0013BF6
:10E070009BB2002B00F03C8602899207F7D56823FB
:10E08000838140F2E93304E0013B9BB2002B00F0B6
:10E090002F860289D707F7D5838940F2E93304E058
:10E0A000013B9BB2002B00F01B8602899607F7D537
:10E0B0000323838140F2E93304E0013B9BB2002B50
:10E0C00000F00E860289D107F7D58389AB6913B1B9
:10E0D0001A689B881383DFF888815E4EDFF884C15D
:10E0E0005D4F4FF0960BD8F80430C3F30803002BB4
:10E0F00040F08A85EFF31183002B40F0858520687E
:10E10000B26823689842FAD13B689A42F7D8DAF8A5
:10E1100000E04FF47A7101FB0EF39B1AB3FBFEF3A0
:10E1200001FB00304FF47A7ED8F80430C3F30803C3
:10E13000002B40F03685EFF31183002B40F0318542
:10E140002368B16822689342FAD13A689142F7D8BD
:10E15000DAF800900EFB09F2521AB2FBF9F20EFB4C
:10E1600003231B1AB3F57A7FDED3BBF1010BBAD1BF
:10E17000AB6913B11A689B885383686940F2E9332D
:10E1800004E0013B9BB2002B00F0EC850289910773
:10E19000F7D56B23838140F2E93304E0013B9BB266
:10E1A000002B00F0DF850289D207F7D5838940F282
:10E1B000E93304E0013B9BB2002B00F0D8850289D3
:10E1C0009707F7D50323838140F2E93304E0013B4D
:10E1D0009BB2002B00F0CB850289D607F7D5838947
:10E1E000AB6913B11A689B8813830F2005F064FC98
:10E1F000AB6913B11A689B885383686940F2E933AD
:10E2000004E0013B9BB2002B00F0B5850289940726
:10E21000F7D56A23838140F2E93304E0013B9BB2E6
:10E22000002B00F0A8850289D107F7D5838940F239
:10E23000E93304E0013B9BB2002B00F0A185028989
:10E240009207F7D51023838140F2E93311E000BF34
:10E2500094B6002010E000E09CB6002098B60020A4
:10E2600000ED00E090B60020013B9BB2002B00F0D7
:10E2700087850289D707F7D58389AB6913B11A68F7
:10E280009B8813830F2005F017FCAB6913B11A6844
:10E290009B885383686940F2E93304E0013B9BB2F9
:10E2A000002B00F0718502899607F7D56C238381D6
:10E2B00040F2E93304E0013B9BB2002B00F064859F
:10E2C0000289D407F7D5838940F2E93304E0013BA2
:10E2D0009BB2002B00F0E08402899107F7D5002360
:10E2E000838140F2E93304E0013B9BB2002B00F054
:10E2F000D3840289D207F7D58389AB6913B11A6831
:10E300009B8813830F2005F0D7FBAB6995F8641049
:10E3100013B11A689B885383686940F2E93304E0BB
:10E32000013B9BB2002B00F0BB8402899707F7D515
:10E330001923838140F2E93304E0013B9BB2002BB7
:10E3400000F0AE840289D607F7D5838940F2E9331D
:10E3500004E0013B9BB2002B00F0A78402899407E4
:10E36000F7D589B2818140F2E93304E0013B9BB2E9
:10E37000002B00F09A840289D107F7D58389AB6915
:10E3800013B11A689B8813830F2005F095FBAB69C6
:10E3900013B11A689B885383686940F2E93304E03B
:10E3A000013B9BB2002B00F0848402899207F7D5D1
:10E3B0001B23838140F2E93304E0013B9BB2002B35
:10E3C00000F077840289D707F7D5838940F2E933D3
:10E3D00004E0013B9BB2002B00F070840289960799
:10E3E000F7D51823838140F2E93304E0013B9BB267
:10E3F000002B00F063840289D407F7D58389AB69C9
:10E4000013B11A689B8813830F2005F055FBAB6985
:10E4100013B11A689B885383686940F2E93304E0BA
:10E42000013B9BB2002B00F04D8402899107F7D588
:10E430001C23838140F2E93304E0013B9BB2002BB3
:10E4400000F040840289D207F7D5838940F2E9338E
:10E4500004E0013B9BB2002B00F03984028997074E
:10E46000F7D51823838140F2E93304E0013B9BB2E6
:10E47000002B00F02C840289D607F7D58389AB697D
:10E4800013B11A689B8813830F2005F015FBAB6945
:10E4900013B11A689B885383686940F2E93304E03A
:10E4A000013B9BB2002B00F0168402899407F7D53C
:10E4B0003723838140F2E93304E0013B9BB2002B18
:10E4C00000F009840289D107F7D5838940F2E93346
:10E4D00004E0013B9BB2002B00F0388402899207D4
:10E4E000F7D51023838140F2E93304E0013B9BB26E
:10E4F000002B00F02B840289D707F7D58389AB69FD
:10E5000013B11A689B8813830F2005F0D5FAAB6905
:10E5100013B11A689B885383686940F2E93304E0B9
:10E52000013B9BB2002B00F0158402899607F7D5BA
:10E530003823838140F2E93304E0013B9BB2002B96
:10E5400000F008840289D407F7D5838940F2E933C3
:10E5500004E0013B9BB2002B00F00184028991078B
:10E56000F7D50123838140F2E93304E0013B9BB2FC
:10E57000002B00F0F4830289D207F7D58389AB69B9
:10E5800013B11A689B8813830F2005F095FA6A6906
:10E59000204B9A4200F0B18303F580639A4200F069
:10E5A000AC83138823F040031B041B0C13801388D7
:10E5B00023F038031B041B0C042141F48071002953
:10E5C00091FAA1F1B1FA81F108BF4FF0FF310139A1
:10E5D00043EAC1039BB21380138843F040031380C6
:10E5E000012005F069FA0C4A6869012382F8B03904
:10E5F000084B98427FF4CCAB038823F040031B0404
:10E600001B0C0380038823F038031B041B0C3022EF
:10E61000FFF7CFBB00380040582800201E09013EFC
:10E62000032E03F00F0300F20282964A32F816001E
:10E6300040FA03F2D70740F1FA81012404FA03F308
:10E64000013B184040F0AAF98F4B904A9B5D18445B
:10E6500012EBC00600F0EB8120210023B171F371B1
:10E6600052F830308A4903F13F4202F57E02920AA5
:10E67000895C01F01F024909032904FA02F200F043
:10E680006982042900F06182022903D18149486C22
:10E6900002434A64B288D4070BD5196821F00301FC
:10E6A000196019681960D96821F00301D960D96827
:10E6B000D96090070BD5196821F00C011960196811
:10E6C0001960D96821F00C01D960D968D960510767
:10E6D0000BD5196821F03001196019681960D968E3
:10E6E00021F03001D960D968D96017070BD51968B6
:10E6F00021F0C001196019681960D96821F0C001C2
:10E70000D960D968D960D4060BD5196821F4407155
:10E71000196019681960D96821F44071D960D96805
:10E72000D96090060BD5196821F440611960196809
:10E730001960D96821F44061D960D968D96051065F
:10E740000BD5196821F44051196019681960D9680E
:10E7500021F44051D960D968D96017060BD51968E2
:10E7600021F44041196019681960D96821F44041C9
:10E77000D960D968D960D4050BD5196821F4403126
:10E78000196019681960D96821F44031D960D968D5
:10E79000D96090050BD5196821F4402119601968DA
:10E7A0001960D96821F44021D960D968D960510530
:10E7B0000BD5196821F44011196019681960D968DE
:10E7C00021F44011D960D968D96017050BD51968B3
:10E7D00021F44001196019681960D96821F44001D9
:10E7E000D960D968D960D4040BD5196821F040717B
:10E7F000196019681960D96821F04071D960D96829
:10E80000D96090040BD5196821F04061196019682E
:10E810001960D96821F04061D960D968D960510484
:10E820000BD5196821F04051196019681960D96831
:10E8300021F04051D960D968D96012040BD51A680B
:10E8400022F040421A601A681A60DA6822F04042E8
:10E85000DA60DA68DA6029460F4B41F80C3F30463F
:10E8600034F00CFCB388B3FA83F3C3F11F03012225
:10E8700012FA03F33FF481AA08490A6813430B60B4
:10E88000FFF77BBABC4C0508C44C0508A0B60020B5
:10E89000604A0508003802407D8A0008003C0140BB
:10E8A000B5F952305BB201337FF419AB95F95030B2
:10E8B00001337FF414AB0A23CB4CDFF844A3CB4FD6
:10E8C000CB4DCC4E019334F0B1F94FF4FA73DFF82D
:10E8D00034E300934FF010087B68C3F30803002B68
:10E8E00040F0EF80EFF31183002B40F0EA802068C6
:10E8F000AA6823689842FAD133689A42F7D8DAF8BE
:10E9000000C04FF47A7101FB0CF39B1AB3FBFCF3CC
:10E9100001FB00304FF47A7C4FF001097B68C3F3B0
:10E920000803002B40F0AE80EFF31183002B40F082
:10E93000A9802368A96822689342FAD1326891427B
:10E94000F7D8DAF800200CFB02FBABEB0101B1FBBE
:10E95000F2F10CFB03131B1AB3F57A7FDED3009B95
:10E96000013B0093B8D1072033F0BCFF4FF47A731A
:10E97000DFF890E200934FF010087B68C3F30803C0
:10E98000002B40F0C080EFF31183002B40F0BB80E0
:10E990002068AA6823689842FAD133689A42F7D867
:10E9A000DAF800C04FF47A7101FB0CF39B1AB3FB49
:10E9B000FCF301FB00304FF47A7C4FF001097B68D7
:10E9C000C3F30803002B3ED1EFF31183002B3AD1A0
:10E9D0002368A96822689342FAD132689142F7D835
:10E9E000DAF800200CFB02FBABEB0101B1FBF2F10A
:10E9F0000CFB03131B1AB3F57A7FE0D3009B013B9A
:10EA00000093BAD1019B013B01937FF45CAFFEF709
:10EA1000B1FB138823F040031B041B0C13801388E5
:10EA200023F038031B041B0C0021FFF72BBA2946E7
:10EA3000714B41F80C3F002034F020FBFFF79DB9EB
:10EA40000721FFF7CBB9EFF3118188F31288D5F8CE
:10EA500008B02B68DB0344BFCEF80090D5F808B0AF
:10EA60002368DEF80020C9B281F31188DAF80010BB
:10EA700013440CFB01F2A2EB0B02B2FBF1F20CFB14
:10EA80000323B7E7EFF3118188F31288D5F808B0B4
:10EA90002B68DB0344BFCEF80090D5F808B023689C
:10EAA000DEF80020C9B281F31188DAF800101344AF
:10EAB0000CFB01F2A2EB0B02B2FBF1F20CFB032305
:10EAC00049E7EFF3118388F31288D5F808C02A6864
:10EAD000D20304D50122CEF80020D5F808C0206862
:10EAE000DEF80090DBB283F31188DAF800104FF4FF
:10EAF0007A72484402FB01F3A3EB0C03B3FBF1F37E
:10EB000002FB003006E7EFF3118388F31288D5F893
:10EB100008C02A68D20304D50122CEF80020D5F817
:10EB200008C02068DEF80090DBB283F31188DAF8C1
:10EB300000104FF47A72484402FB01F3A3EB0C037C
:10EB4000B3FBF1F302FB003035E72C49086B0243BD
:10EB50000A639FE52949086C02430A649AE5EFF3CA
:10EB60001181102383F31288D6F808903368DB03F1
:10EB700004D50123CCF80030D6F808902368DCF8DF
:10EB80000020C9B281F31188DAF8001013440EFB9B
:10EB900001F2A2EB0902B2FBF1F20EFB0323FFF735
:10EBA00056BAEFF31181102383F31288D6F8089038
:10EBB0003368DB0304D50123CCF80030D6F8089085
:10EBC0002368DCF80020C9B281F31188DAF800105C
:10EBD00013440EFB01F2A2EB0902B2FBF1F20EFBB1
:10EBE0000323FFF7BEBA00BF94B6002000ED00E09B
:10EBF00010E000E09CB600207D8A0008003802404A
:10EC000098B6002090B60020EFF31183102282F313
:10EC10001288D6F808E03268D20304D50122CCF875
:10EC20000020D6F808E02068DCF80090DBB283F31F
:10EC30001188DAF800104FF47A72484402FB01F3AD
:10EC4000A3EB0E03B3FBF1F302FB0030FFF76ABA4C
:10EC5000EFF31183102282F31288D6F808E03268AD
:10EC6000D20304D50122CCF80020D6F808E02068B1
:10EC7000DCF80090DBB283F31188DAF800104FF46F
:10EC80007A72484402FB01F3A3EB0E03B3FBF1F3EA
:10EC900002FB0030FFF7BCB9FAF7D4FFFFF72DBB3A
:10ECA000FAF7D0FF6869FFF751BBFAF7CBFFFFF720
:10ECB00066BBFAF7C7FF6869FFF788BBFAF7C2FFC0
:10ECC000FFF79DBBFAF7BEFF6869FFF7BFBBFAF716
:10ECD000B9FFFFF7D4BBFAF7B5FF6869FFF7F6BBDA
:10ECE000FAF7B0FFFFF7F2B9FAF7ACFFFFF761B937
:10ECF000FAF7A8FF6869FFF7D0B9138823F040033B
:10ED00001B041B0C1380138823F038031B041B0CFB
:10ED1000022152E4FAF796FFFFF796B8FAF792FF4E
:10ED20006869FFF779B8038823F040031B041B0CC4
:10ED30000380038823F038031B041B0C8022FFF799
:10ED4000E9B8FAF77FFF6869FFF715B9FAF77AFFB4
:10ED5000FFF7D5BBFAF776FF6869FFF7F7BBFAF75D
:10ED600071FF0CE4FAF76EFF6869FFF720BAFAF753
:10ED700069FFFFF735BAFAF765FF6869FFF757BA19
:10ED8000FAF760FFFFF779BAFAF75CFF6869FFF7F7
:10ED90009BBA00BF70B582B00446062308306A46AD
:10EDA0003B21FEF747FEA8B19DF804009DF80060E6
:10EDB0009DF801109DF802509DF803209DF8053044
:10EDC00041EA062143EA002342EA0522E182228346
:10EDD0006383012002B070BDF0B5C60033189B00FC
:10EDE000244DEA585468A28A83B092B20192019AE3
:10EDF0002B4412F4706F1CBF01221A75019B13F48F
:10EE0000E06F07460CD1A38A3E4423F4706305EB00
:10EE100086051B041B0C0022A3826A7503B0F0BD9B
:10EE2000238BA38823F480631B041B0CA380019B0A
:10EE30009B05E8D423889805E5D42388D9050DD50A
:10EE40002388DA05FCD4238843F4007323802388C5
:10EE50009B05FCD43846FEF7B1FCD4E7238843F485
:10EE600000732380A38823F440731B041B0CA3802E
:10EE7000C9E700BF305D0020F0B583B0441C8DF8B9
:10EE8000073001D0032802DD002003B0F0BDC70029
:10EE9000274E3B1806EB83035C68002CF4D0490036
:10EEA000C9B2997501250021DA755D7699761D76CE
:10EEB0005D751975A1880DF107028905C3E907225F
:10EEC00012D42388DA050BD44FF4805501E0013DBC
:10EED00025D023889B05FAD4238843F480732380AC
:10EEE000A38843F44073A380074406EB87024FF4E2
:10EEF000805401E0013C09D0537D002BFAD106EB90
:10EF00008707387D80F0010003B0F0BD094A1388FF
:10EF100001339BB21380FEF751FC2046B5E7054A4A
:10EF2000138801339BB21380FEF748FC2846ACE7F8
:10EF3000305D0020628E00200378012B47D0022B29
:10EF400043D183682DE9F04101F07F0113B11C68C2
:10EF50009B88638305461746406840F2E93401E028
:10EF6000002C3FD00689013C16F0020FA4B2F7D066
:10EF700089B2818140F2E93101E0002932D0038970
:10EF8000013913F0010F89B2F7D0838940F2E931DA
:10EF900000E021B30489013914F0020F89B2F8D0DE
:10EFA000BFB2878140F2E93300E0C3B10289013B7F
:10EFB00012F0010F9BB2F8D08389AB686BB11A686D
:10EFC0009B8813830120BDE8F08100207047134621
:10EFD0000A46417990F904004EE70120F3E7FAF779
:10EFE00031FEEAE7FAF72EFE6868CFE710B500F1C8
:10EFF0000C0401220B212046FFF79EFF20B11D22A9
:10F0000009212046FFF798FF00F0010010BD10B560
:10F0100000F10C04702200212046FFF78DFF202212
:10F0200001212046FFF788FF002202212046FFF73A
:10F0300083FF642004F09EFD012010BD01224821C1
:10F040007AE70122582177E73122F42174E7044B53
:10F0500093F820209201343202F0FC02F4216BE795
:10F06000706800202E22F42166E700BF2DE9F04FE2
:10F0700085B090F865300090002B40F01687009B1B
:10F0800093F85C30072B01F048801823CDE9023358
:10F09000009A137C012B01F05D80022B12D1936941
:10F0A00013B11A689B885383009C6B216069FAF73F
:10F0B0002FFF80216069FAF72BFFA36913B11A684B
:10F0C0009B8813836423AE4CAE4EDFF8C4E2AE4897
:10F0D000DFF8C082AD4F01934FF01009DEF8043025
:10F0E000C3F30803002B40F02985EFF31183002BB5
:10F0F00040F024852568826823689D42FAD13B68E8
:10F100009A42F7D8D6F800C04FF47A7101FB0CF39D
:10F110009B1AB3FBFCF301FB05354FF47A7C4FF0EF
:10F12000010ADEF80430C3F30803002B40F0BC846E
:10F13000EFF31183002B40F0B784236881682268C5
:10F140009342FAD13A689142F7D832680CFB02FB3D
:10F15000ABEB0101B1FBF2F10CFB03135B1BB3F54D
:10F160007A7FDED3019B013B0193B7D1009A137CD8
:10F17000012B00F0F987022B12D1936913B11A68A1
:10F180009B885383009D68216869FAF7C1FE0721B7
:10F190006869FAF7BDFEAB6913B11A689B881383DF
:10F1A0006423DFF8ECE17848DFF8E881774F0193DA
:10F1B0004FF01009DEF80430C3F30803002B40F0D1
:10F1C0009B84EFF31183002B40F0968425688268BE
:10F1D00023689D42FAD13B689A42F7D8D6F800C01E
:10F1E0004FF47A7101FB0CF39B1AB3FBFCF301FBA8
:10F1F00005354FF47A7C4FF0010ADEF80430C3F392
:10F200000803002B40F03184EFF31183002B40F012
:10F210002C842368816822689342FAD13A6891422B
:10F22000F7D832680CFB02FBABEB0101B1FBF2F14A
:10F230000CFB03135B1BB3F57A7FDED3019B013B11
:10F240000193B7D1009A137C012B00F0A087022B09
:10F2500012D1936913B11A689B885383009D6B2167
:10F260006869FAF755FE00216869FAF751FEAB6943
:10F2700013B11A689B8813836423DFF814E14248B2
:10F28000DFF81081414F01934FF01009DEF8043090
:10F29000C3F30803002B40F09584EFF31183002B98
:10F2A00040F090842568826823689D42FAD13B68CB
:10F2B0009A42F7D8D6F800C04FF47A7101FB0CF3EC
:10F2C0009B1AB3FBFCF301FB05354FF47A7C4FF03E
:10F2D000010ADEF80430C3F30803002B40F0A783D3
:10F2E000EFF31183002B40F0A2832368816822682A
:10F2F0009342FAD13A689142F7D832680CFB02FB8C
:10F30000ABEB0101B1FBF2F10CFB03135B1BB3F59B
:10F310007A7FDED3019B013B0193B7D1009A137C26
:10F32000012B00F02B87022B12D1936913B11A68BD
:10F330009B885383009D6B216869FAF7E9FD0121E1
:10F340006869FAF7E5FDAB6913B11A689B88138306
:10F350000F23DFF83CE00C48DFF838800B4F0193B7
:10F360004FF01009DEF80430C3F30803002B40F01F
:10F370000784EFF31183002B40F002840CE000BF00
:10F3800094B6002098B6002010E000E09CB6002063
:10F3900000ED00E090B600202568826823689D4259
:10F3A000FAD13B689A42F7D8D6F800C04FF47A7188
:10F3B00001FB0CF39B1AB3FBFCF301FB05354FF487
:10F3C0007A7C4FF0010ADEF80430C3F30803002B07
:10F3D00040F00F83EFF31183002B40F00A83236882
:10F3E000816822689342FAD13A689142F7D832682C
:10F3F0000CFB02FBABEB0101B1FBF2F10CFB0313C5
:10F400005B1BB3F57A7FDED3019B013B0193A9D14E
:10F41000009A92F85F30032B09D992F86330012BE0
:10F42000029B0CBF43F0010343F002030293137CE1
:10F430009DF80850012B00F0BE86022B12D1936973
:10F4400013B11A689B885383009F1B217869FAF7D0
:10F450005FFD29467869FAF75BFDBB6913B11A684D
:10F460009B8813830F23DFF8DCE2B448DFF8D882EF
:10F47000B34F01934FF01009DEF80430C3F30803D3
:10F48000002B40F0E283EFF31183002B40F0DD838B
:10F490002568826823689D42FAD13B689A42F7D872
:10F4A000D6F800C04FF47A7101FB0CF39B1AB3FB42
:10F4B000FCF301FB05354FF47A7C4FF0010ADEF8CE
:10F4C0000430C3F30803002B40F07582EFF311837F
:10F4D000002B40F070822368816822689342FAD141
:10F4E0003A689142F7D832680CFB02FBABEB0101A2
:10F4F000B1FBF2F10CFB03135B1BB3F57A7FDED398
:10F50000019B013B0193B7D1009A137C012B00F0C2
:10F510004886022B12D1936913B11A689B885383D2
:10F52000009D1C216869FAF7F3FC03996869FAF7F2
:10F53000EFFCAB6913B11A689B8813830F23DFF8C4
:10F5400004E27E48DFF800827D4F01934FF01009FE
:10F55000DEF80430C3F30803002B40F05583EFF3CB
:10F560001183002B40F050832568826823689D42F8
:10F57000FAD13B689A42F7D8D6F800C04FF47A71B6
:10F5800001FB0CF39B1AB3FBFCF301FB05354FF4B5
:10F590007A7C4FF0010ADEF80430C3F30803002B35
:10F5A00040F0EB81EFF31183002B40F0E6812368FC
:10F5B000816822689342FAD13A689142F7D832685A
:10F5C0000CFB02FBABEB0101B1FBF2F10CFB0313F3
:10F5D0005B1BB3F57A7FDED3019B013B0193B7D16F
:10F5E000009A92F85F30032B00F25C8492F862502C
:10F5F000012D00F04B83A5F10205B5FA85F56D09E3
:10F60000137C012B00F04883022B12D1936913B1B4
:10F610001A689B885383009F1A217869FAF778FC4F
:10F6200029467869FAF774FCBB6913B11A689B889C
:10F6300013830F23DFF80CE14048DFF80C81404FC3
:10F6400001934FF01009DEF80430C3F30803002BD8
:10F6500040F00684EFF31183002B40F0018425680D
:10F66000826823689D42FAD13B689A42F7D8D6F85F
:10F6700000C04FF47A7101FB0CF39B1AB3FBFCF34F
:10F6800001FB05354FF47A7C4FF0010ADEF80430B7
:10F69000C3F30803002B40F00883EFF31183002B22
:10F6A00040F003832368816822689342FAD13A6864
:10F6B0009142F7D832680CFB02FBABEB0101B1FBC6
:10F6C000F2F10CFB03135B1BB3F57A7FDED3019BD6
:10F6D000013B0193B7D1009A137C92F86450012B3F
:10F6E00000F07385022B12D1926912B113689288CF
:10F6F0005A83009F19217869FAF70AFC294678692C
:10F70000FAF706FCBB6913B11A689B88138364235C
:10F71000DFF830E00948DFF83080094F01934FF0FF
:10F720001009DEF80430C3F30803002B40F07783A0
:10F73000EFF31183002B40F0728307E010E000E04C
:10F740009CB6002000ED00E090B60020256882689D
:10F7500023689D42FAD13B689A42F7D8D6F800C098
:10F760004FF47A7101FB0CF39B1AB3FBFCF301FB22
:10F7700005354FF47A7C4FF0010ADEF80430C3F30C
:10F780000803002B40F0CD82EFF31183002B40F0F3
:10F79000C8822368816822689342FAD13A6891420C
:10F7A000F7D832680CFB02FBABEB0101B1FBF2F1C5
:10F7B0000CFB03135B1BB3F57A7FDED3019B013B8C
:10F7C0000193AED1009A137C012B00F00885022B27
:10F7D00012D1936913B11A689B885383009D372116
:10F7E0006869FAF795FB10216869FAF791FBAB6934
:10F7F00013B11A689B8813830F23DFF8F4E2BA4829
:10F80000DFF8F082B94F01934FF01009DEF80430B1
:10F81000C3F30803002B40F0E182EFF31183002BC8
:10F8200040F0DC822568826823689D42FAD13B68FB
:10F830009A42F7D8D6F800C04FF47A7101FB0CF366
:10F840009B1AB3FBFCF301FB05354FF47A7C4FF0B8
:10F85000010ADEF80430C3F30803002B40F04382B2
:10F86000EFF31183002B40F03E8223688168226809
:10F870009342FAD13A689142F7D832680CFB02FB06
:10F88000ABEB0101B1FBF2F10CFB03135B1BB3F516
:10F890007A7FDED3019B013B0193B7D1009A137CA1
:10F8A000012B00F0A684022B12D1936913B11A68C0
:10F8B0009B885383009D38216869FAF729FB012151
:10F8C0006869FAF725FBAB6913B11A689B88138343
:10F8D0000F23DFF81CE28448DFF81882834F00937F
:10F8E0004FF01009DEF80430C3F30803002B40F09A
:10F8F0005482EFF31183002B40F04F822568826819
:10F9000023689D42FAD13B689A42F7D8D6F800C0E6
:10F910004FF47A7101FB0CF39B1AB3FBFCF301FB70
:10F9200005354FF47A7C4FF0010ADEF80430C3F35A
:10F930000803002B40F01382EFF31183002B40F0FB
:10F940000E822368816822689342FAD13A68914214
:10F95000F7D832680CFB02FBABEB0101B1FBF2F113
:10F960000CFB03135B1BB3F57A7FDED3009B013BDB
:10F970000093B7D105B0BDE8F08FEFF3118189F3A3
:10F980001288D0F808B00368DB0344BFC8F800A0B1
:10F99000D0F808B02368D8F80020C9B281F31188E4
:10F9A000316813440CFB01F2A2EB0B02B2FBF1F243
:10F9B0000CFB03230CE6EFF3118189F31288D0F8D6
:10F9C00008B00368DB0344BFC8F800A0D0F808B053
:10F9D0002368D8F80020C9B281F311883168134434
:10F9E0000CFB01F2A2EB0B02B2FBF1F20CFB0323C6
:10F9F00082E5EFF3118189F31288D0F808B003682B
:10FA0000DB0344BFC8F800A0D0F808B02368D8F8DA
:10FA10000020C9B281F31188316813440CFB01F254
:10FA2000A2EB0B02B2FBF1F20CFB0323E8E4EFF3D1
:10FA3000118189F31288D0F808B00368DB0344BF52
:10FA4000C8F800A0D0F808B02368D8F80020C9B2E0
:10FA500081F31188316813440CFB01F2A2EB0B0215
:10FA6000B2FBF1F20CFB032350E4EFF3118189F3B5
:10FA70001288D0F808B00368DB0344BFC8F800A0C0
:10FA8000D0F808B02368D8F80020C9B281F31188F3
:10FA9000316813440CFB01F2A2EB0B02B2FBF1F252
:10FAA0000CFB0323FFF7C6BBEFF3118189F3128828
:10FAB000D0F808B00368DB0344BFC8F800A0D0F852
:10FAC00008B02368D8F80020C9B281F311883168E2
:10FAD00013440CFB01F2A2EB0B02B2FBF1F20CFBA4
:10FAE0000323FFF73BBB00BF10E000E09CB6002003
:10FAF00000ED00E090B60020EFF3118389F3128847
:10FB0000D0F808C00268D20304D50122C8F800204A
:10FB1000D0F808C02568D8F800A0DBB283F31188BC
:10FB200031684FF47A72554402FB01F3A3EB0C03E6
:10FB3000B3FBF1F302FB0535FFF75BBBEFF311837A
:10FB400089F31288D0F808C00268D20304D50122D4
:10FB5000C8F80020D0F808C02568D8F800A0DBB2AB
:10FB600083F3118831684FF47A72554402FB01F334
:10FB7000A3EB0C03B3FBF1F302FB0535FFF7CDBAA2
:10FB8000EFF3118389F31288D0F808C00268D2031A
:10FB900004D50122C8F80020D0F808C02568D8F89C
:10FBA00000A0DBB283F3118831684FF47A725544B8
:10FBB00002FB01F3A3EB0C03B3FBF1F302FB0535EE
:10FBC000FFF7FDBBEFF3118389F31288D0F808C06B
:10FBD0000268D20304D50122C8F80020D0F808C07A
:10FBE0002568D8F800A0DBB283F3118831684FF4A0
:10FBF0007A72554402FB01F3A3EB0C03B3FBF1F360
:10FC000002FB0535FFF761BBEFF3118389F312881F
:10FC1000D0F808C00268D20304D50122C8F8002039
:10FC2000D0F808C02568D8F800A0DBB283F31188AB
:10FC300031684FF47A72554402FB01F3A3EB0C03D5
:10FC4000B3FBF1F302FB0535A1E4EFF3118389F374
:10FC50001288D0F808C00268D20304D50122C8F87F
:10FC60000020D0F808C02568D8F800A0DBB283F3E4
:10FC7000118831684FF47A72554402FB01F3A3EB0B
:10FC80000C03B3FBF1F302FB053514E4137C012BE9
:10FC90004FF007057FF4B8AC10462B46417D90F934
:10FCA00014001A22FFF7E8F8C3E4EFF3118189F397
:10FCB0001288D0F808B00368DB0344BFC8F800A07E
:10FCC000D0F808B02368D8F80020C9B281F31188B1
:10FCD000316813440CFB01F2A2EB0B02B2FBF1F210
:10FCE0000CFB0323EFE4EFF3118189F31288D0F8C2
:10FCF00008B00368DB0344BFC8F800A0D0F808B020
:10FD00002368D8F80020C9B281F311883168134400
:10FD10000CFB01F2A2EB0B02B2FBF1F20CFB032392
:10FD2000B4E5EFF3118189F31288D0F808B00368C5
:10FD3000DB0344BFC8F800A0D0F808B02368D8F8A7
:10FD40000020C9B281F31188316813440CFB01F221
:10FD5000A2EB0B02B2FBF1F20CFB03232AE5EFF35B
:10FD6000118189F31288D0F808B00368DB0344BF1F
:10FD7000C8F800A0D0F808B02368D8F80020C9B2AD
:10FD800081F31188316813440CFB01F2A2EB0B02E2
:10FD9000B2FBF1F20CFB0323E4E5EFF3118389F3EB
:10FDA0001288D0F808C00268D20304D50122C8F82E
:10FDB0000020D0F808C02568D8F800A0DBB283F393
:10FDC000118831684FF47A72554402FB01F3A3EBBA
:10FDD0000C03B3FBF1F302FB0535A2E5EFF311834E
:10FDE00089F31288D0F808C00268D20304D5012232
:10FDF000C8F80020D0F808C02568D8F800A0DBB209
:10FE000083F3118831684FF47A72554402FB01F391
:10FE1000A3EB0C03B3FBF1F302FB053515E5EFF3A0
:10FE2000118389F31288D0F808C00268D20304D580
:10FE30000122C8F80020D0F808C02568D8F800A032
:10FE4000DBB283F3118831684FF47A72554402FBB8
:10FE500001F3A3EB0C03B3FBF1F302FB053588E4DC
:10FE6000EFF3118389F31288D0F808C00268D20337
:10FE700004D50122C8F80020D0F808C02568D8F8B9
:10FE800000A0DBB283F3118831684FF47A725544D5
:10FE900002FB01F3A3EB0C03B3FBF1F302FB05350B
:10FEA000FFF7F0BB019DFFF7ABBB1D09013D032D23
:10FEB00003F00F0300F2AC819F4A32F8150040FABC
:10FEC00003F2D40740F1A481012404FA03F3013BB7
:10FED00018403EF063FD994B994A5B5D184412EB64
:10FEE000C00500F0958120210023A971EB7152F823
:10FEF0003030944903F13F4202F57E02920A895C58
:10FF000001F01F024909032904FA02F200F08E8170
:10FF1000042900F08681022903D18B49486C0243F1
:10FF20004A64AA88D0070BD5196821F0030119602B
:10FF300019681960D96821F00301D960D968D960BE
:10FF400091070BD5196821F00C0119601968196027
:10FF5000D96821F00C01D960D968D96057070BD551
:10FF6000196821F03001196019681960D96821F009
:10FF70003001D960D968D96016070BD5196821F00E
:10FF8000C001196019681960D96821F0C001D960F1
:10FF9000D968D960D4060BD5196821F4407119606D
:10FFA00019681960D96821F44071D960D968D9609D
:10FFB00090060BD5196821F4406119601968196021
:10FFC000D96821F44061D960D968D96051060BD550
:10FFD000196821F44051196019681960D96821F431
:10FFE0004051D960D968D96017060BD5196821F43A
:10FFF0004041196019681960D96821F44041D960FD
:020000040801F1
:10000000D968D960D6050BD5196821F4403119603B
:1000100019681960D96821F44031D960D968D9606C
:1000200094050BD5196821F44021196019681960ED
:10003000D96821F44021D960D968D96050050BD521
:10004000196821F44011196019681960D96821F400
:100050004011D960D968D96011050BD5196821F410
:100060004001196019681960D96821F44001D9600C
:10007000D968D960D7040BD5196821F0407119608F
:1000800019681960D96821F04071D960D968D960C0
:1000900096040BD5196821F0406119601968196040
:1000A000D96821F04061D960D968D96054040BD572
:1000B000196821F04051196019681960D96821F058
:1000C0004051D960D968D96010040BD51A6822F064
:1000D00040421A601A681A60DA6822F04042DA6018
:1000E000DA68DA600099194B41F80C3F284632F083
:1000F000C5FFAB88B3FA83F3C3F11F03012212FAE1
:1001000003F33EF4BCAF12490A6813430B60009B33
:1001100093F85C30072B7EF4B8AF009B93F8613006
:10012000002B6FD1009A1023CDE90233137C012BF1
:100130007EF4B3AF0EE000BFBC4C0508C44C05080C
:10014000A0B60020604A0508003802407D8A0008F9
:10015000003C014010468023417D90F914006B2241
:10016000FEF78AFEFEF7AEBF10460723417D90F9E9
:1001700014006822FEF780FEFFF712B810466B22CB
:10018000417D90F91400FEF777FEFFF7E1B81046C5
:10019000019B417D90F914006B22FEF76DFEFFF785
:1001A0006BB81046039B417D90F914001C22FEF7AA
:1001B00063FEFFF7C3B910462B46417D90F914004A
:1001C0001B22FEF759FEFFF74DB910462B46417D25
:1001D00090F914001922FEF74FFEFFF798BA104667
:1001E0001023417D90F914003722FEF745FEFFF7FA
:1001F00003BB10463822417D90F91400FEF73CFE07
:10020000FFF766BB18231021CDE90231FEF740BF8E
:100210000099094B41F80C3F002032F02FFFFEF708
:100220002EBF0649086B02430A637AE60349086C4D
:1002300002430A6475E600BF7D8A00080038024068
:100240002DE9F04F9D4B426983B09A42019000F036
:100250001F8103F580639A4200F01A81138823F00E
:1002600040031B041B0C1380138823F038031B046A
:100270001B0C30210B431380138843F04003138081
:10028000012003F019FC019C2046FEF7EFFEA36954
:1002900013B11A689B885383019B586940F2E93374
:1002A00002E0002B00F001810289013B12F0020FF5
:1002B0009BB2F6D06A23838140F2E93302E0002B3F
:1002C00000F0F3800289013B12F0010F9BB2F6D0DF
:1002D000838940F2E93302E0002B00F0EB800289D1
:1002E000013B12F0020F9BB2F6D01023838140F243
:1002F000E93302E0002B00F0DD800289013B12F0BF
:10030000010F9BB2F6D08389019B9B6913B11A68D8
:100310009B88138364236A48DFF8B0E1DFF8B0C13B
:10032000684CDFF8B081684E00934FF01009DCF89C
:100330000430C3F30803002B7ED1EFF31183002BAD
:100340007AD10568A26803689D42FAD133689A425F
:10035000F7D8DEF800704FF47A7101FB07F39B1AAF
:10036000B3FBF7F301FB05354FF47A774FF0010A41
:10037000DCF80430C3F30803002B3ED1EFF3118304
:10038000002B3AD10368A16802689342FAD132681F
:100390009142F7D8DEF8002007FB02FBABEB01012E
:1003A000B1FBF2F107FB03135B1BB3F57A7FDFD3DD
:1003B000009B013B0093BAD1019B5A693F4B9A4283
:1003C00059D003F580639A4255D0138823F0400337
:1003D0001B041B0C1380138823F038031B041B0C15
:1003E00008210B4313801388012043F0400313803E
:1003F00003B0BDE8F04F03F05FBBEFF3118189F369
:100400001288D4F808B02368DB0344BFC8F800A002
:10041000D4F808B00368D8F80020C9B281F3118875
:10042000DEF80010134407FB01F2A2EB0B02B2FB53
:10043000F1F207FB0323B7E7EFF3118389F3128887
:10044000A7682268D20303D50122C8F80020A76854
:100450000568D8F800A0DBB283F31188DEF800103D
:100460004FF47A72554402FB01F3DB1BB3FBF1F34B
:1004700002FB053578E7138823F040031B041B0CAF
:100480001380138823F038031B041B0C0021A8E7FA
:10049000138823F040031B041B0C1380138823F0E4
:1004A00038031B041B0C2821E4E6F9F7CBFB019B66
:1004B00058690EE7F9F7C6FB26E700BF0038004091
:1004C00094B6002010E000E09CB6002098B6002012
:1004D00000ED00E090B600200220F8F70FBD00BF4D
:1004E0000220FEF779BC00BF0120F8F707BD00BF6E
:1004F0000120FEF771BC00BF0020F8F7FFBC00BF71
:100500000020FEF769BC00BF044B187828B1044AEC
:100510001268520744BF0020187070470A5D00201F
:100520000020014043680B4A23F0407323F480739A
:1005300043F48073436083681A4042F00202826091
:10054000C36A0139C9B223F4700343EA0153C36299
:10055000704700BFFDF7FFC01F4B1B68032B30B473
:1005600033D81E4A1E4903EB43035B0098189B5A7D
:1005700042888088C1F8C030C1E93102B3FBF2F291
:100580001848194D19491A4B1A4C00FB02F22A60FF
:10059000D1F8882042F47002C1F888201A6800203F
:1005A00042F001021A6098601A6822F0847222F404
:1005B00080321A605C601A684FF0006422F4802276
:1005C0001A60D8608C6030BC7047054AD2F8C030E1
:1005D000D2F8C820D2E700BFD40B01202C140508A4
:1005E0000000002040420F0064DA002000ED00E02F
:1005F000003802401030002470B50C4C23689BB1C9
:100600005A68821A002A0FDB0546002603E05A6862
:10061000AA1A002A08DB99681E731A682160184616
:1006200090472368002BF2D170BD00BF40510020DD
:10063000436A8269D154436A0169C26B01338B42B8
:1006400028BF00234362DAB1EFF31183502282F313
:100650001288C26B1168C9070ED470B45468FCB913
:10066000D0E909518D4211D1012280F86020DBB21E
:1006700083F3118870BC7047DBB283F31188704735
:10068000C26DD36843F08003D360704786690E441F
:10069000D6600ED9691A51608562002180F8601019
:1006A000116841F00101DBB2116083F3118870BC65
:1006B00070470569691A51608462EEE7034610B419
:1006C000846BD968406954B11A6D8C1A013A005D87
:1006D0005DF8044B08BF0A46C0B21A6570471A6A33
:1006E000805C01328A4228BF2246C0B21A625DF89D
:1006F000044B7047C36B13B190F860007047D0E9AA
:100700000903181AB0FA80F040097047D0E90912BD
:100710000369914238BFC9188A1AC16B013B19B1EC
:1007200049680A449A4201D2981A704700207047DB
:10073000836B43B1026D5B689A4291BF981AC0689F
:100740009B1AC0187047D0E907239A422FBFD01ACE
:10075000C0688018C01A70470A4B30B503F11C04FA
:1007600093F900205D78072AC8BF143A8118043332
:100770000D7313F8025C855413F8012C0A769C4221
:10078000EED130BD6C12050803682DE9F0415D6AB9
:100790001DB12B46BDE8F0411847002A174611DD70
:1007A00004460E460F4400E023689B6820469847A5
:1007B0000028F9D0236816F8011B1B6820469847CB
:1007C000BE42F1D1BDE8F08103681B69184700BF44
:1007D000002329211E22017042708370C37070476C
:1007E0002DE9F843864D6B6846F2A712C31A93426F
:1007F0002DED028B03D8BDEC028BBDE8F883814B55
:1008000068601C6814F0040662D1304614F02004BD
:1008100029D1DFED7D7A27467C4B7D4A1B78117804
:1008200013F0010345D100294AD0D5E905C1137061
:10083000A0EB0C00791A2CBB0EB1764B1860764BEE
:100840001B780E2BD7D19FED757A754B67EE877AA3
:10085000BDEC028BFDEEE77A588017EE902A998066
:100860001A80BDE8F8836F4B1C7814F0020471D035
:100870006D4A138A9768002B40F0AA80DFED627AF8
:100880000124C9E70EB3B7EE007A77EE676A07EE88
:10089000100AB8EEC77A5F4B27EE267A06EE901A5A
:1008A000F8EEE66AA6EEA77ABDEEC77A83ED007A87
:1008B000C5E729B90123C5E9050713700846BAE75A
:1008C000D5E90531C01A791AB5E7524B1960B6E778
:1008D000DFF87491DFF8748199F80630B8F8006099
:1008E000AF68013BB7FBF3F7C6B3504A9FED500A20
:1008F0001368002B1946B8BFD91DA3EBE1031F44B1
:10090000002F3B46B8BFFB1DDB1007EE903AF8EE18
:10091000E77A176027EE800AF9F708FDDFED457AE0
:1009200020EE270AF9F748FDF7EE007A77EEC07A55
:100930009FED410A2B6967EE807A9F42FDEEE77AD0
:10094000C5ED037A56D0731E0026A8F800302F613B
:1009500030465BE7DFED2C7A27465DE707EE907ABD
:100960009FED330A354EF8EE677AB7EE008A27EE30
:10097000800AF9F7DBFCDFED2F7A20EE270AF9F782
:100980001BFDDFED2D7A38EE400A20EE270A3EF0FF
:1009900081FBB9F80830DFED2A6A07EE103AEB6800
:1009A000C01AB8EEC77A07EE900AA7EE668AB8EECC
:1009B000E70AD6ED097AF8EEE77A20EE080A67EE44
:1009C000A67AA7EE270A3EF065FB706201261DE7B6
:1009D00007EE903A9FED116ADFED1A6AB8EEE77AFA
:1009E000C6EE077AF4EEE67AF1EE10FA88BFF0EE82
:1009F000667A45E700231E46A8F80030184605E74A
:100A0000405100208C6B00209A99993E56A50020F9
:100A10003C840020DC73002049B600200000C8425E
:100A20004CB60020306E00201C6E0020000100201B
:100A300008942537B1DC423ED048874A906B0020AD
:100A40006F12833A6666663F748700205257002013
:100A50002DE9F8432D4B1B685B0701D4BDE8F883F3
:100A60002B4C2C4D94F81C90B9F1010F3BD1EB6944
:100A7000284698472B69284698472B6A04F120019D
:100A800004F124009847244AA6689179D4E90A839E
:100A9000D4E9082008F10107AA625A1C8F4208BF56
:100AA0000027032AE86228D01C49E26294F830202B
:100AB00041F823003ABB04EB880804EB8703C8F82D
:100AC00034005A6BAB89A762B61A30440022A0608A
:100AD0002277002BC2D0124A0A2B1268B8BF0A2311
:100AE0001361BDE8F8836B6928469847AB692846CF
:100AF00098470122EB892277EBE7084A84F8309087
:100B000000239060E36236F053F9D4E78C6B002049
:100B100040510020906B002074870020C0DA002034
:100B20009C0B00102DE9F0478C4A8D4B12781C78F5
:100B3000D207064648D58B4D012C00F091801ED37C
:100B4000022C40F09B808849884A09881288884F87
:100B5000914201D901241C70EB7AFBB12B89EBB1D6
:100B6000844B1B78D3B10FF0AFFF002800F0E28078
:100B70002B7B83422CBF012300233B700FE0DFF867
:100B8000E8C17B4F7C4CBCF800002288697B521A7C
:100B90008242DFDAEB7A0024002BDFD13B782A791E
:100BA000632A07D87549022C087800F0B88000281D
:100BB00040F0A0807249AA7A9C4238BF1C460C7053
:100BC000002A44D1BDE8F087DFF89CC1654DBCF830
:100BD0000000BCF8021095F803E06A4F411A0029A2
:100BE000A4F10302B8BF4942704597F80080D2B221
:100BF00011D32F7887420ED3012A45D9B8F1020FBD
:100C00009AD15C48604A007890800229CCBF0021CC
:100C10000121D18090E7B0EB4E0FEDDC012A40F2CC
:100C20008C800229EADC0324514F524852494F4A32
:100C30001C70B8F1020F4FF000033C7003700B8082
:100C4000138089D1504A01219380D18084E7012CFF
:100C50006BD0022CB6D10720BDE8F04721F084B953
:100C6000424A41491288687B0988121A914207DD7D
:100C7000414A12888A423CBF00241C703C4F6BE7FB
:100C800002241C703A4F67E70229B7DC95F800E0B0
:100C900090FBFEFE0EF1010EBEF1080FDFF8D4A0AE
:100CA000AA786978DFF8C490334C314FA8BF4FF071
:100CB000080E8AF800E01FFA8EFA11FB0AF112FB07
:100CC0000AF2DFF8B8A0A9F8001092B200214FF0A4
:100CD0006409B8F1020F228039701970CAF8041043
:100CE0008AF801907FF452AF274A0121A2F804E06C
:100CF000D18048E74868301A244EB042C8BF4A70D5
:100D00003FF758AFC2F16402214E00FB02F086FBB0
:100D10000062C017A0EBA250643048704AE7002878
:100D2000E8D101274E600F70ECE70820BDE8F047DE
:100D300021F01AB902233B7031E7032C7FF471AF25
:100D4000B8F1020F9AD10B4A0F4B12789A80022900
:100D5000CCBF00210121D980054FFDE656A500201A
:100D6000AC5600206E6C0020686E0020B05600204B
:100D70000C5700206E6E0020AE560020B4560020A6
:100D80006C6C002049B600204CB600207F9698007D
:100D90006BCA5F6B2DE9F04B84B02EF063FDE8B1B8
:100DA0009C4C41F29C03E358002B1ADC6378022B25
:100DB0001CD0032B12D141F2B813E35C2BBB41F2E0
:100DC000A403E35C4BBB41F2E803E35C0BBB41F2E1
:100DD0002C13E35C13B190482EF074FB04B0BDE813
:100DE000F08B2EF08BFC6378022BE2D1A3784FF0CE
:100DF0000109072BF2D8DFE813F05A00E900700070
:100E000051001700AA00B400140084482EF05AFBC9
:100E1000D5E783482EF056FBD9E782482EF052FBE7
:100E2000D1E703236370D9E72278237DDFF81482AA
:100E30007D4E032A14BF4FF480778027002B00F0EB
:100E4000B180012BFAD1794B62681968D8F800009B
:100E50004FEA412C00234FF0FF31B1FBFCF112EBC4
:100E6000010B43F1000C0021614500F1020008BFB5
:100E7000584538BF83465A466D4902202DF0AAFDD9
:100E8000032800F2C48001A353F820F0DD0D01080F
:100E90007B0F0108DD0D01087B0F010841F2701383
:100EA000E35C002B9AD063482EF00CFB96E70023FE
:100EB00003AD2946184609222DF024FA01288DD1C8
:100EC000039B93F8FE21552A00F0BE8041F2B41234
:100ED00002210123A154637080E7574B009303253F
:100EE0003023052255495348A57031F003FC75E7BE
:100EF00023690622652BA27033D92278032A14BFF6
:100F00006FF0FF026FF07F02A3F1650303EA0203B3
:100F100003F1010314BF4FF4807280229A422361CF
:100F20001FD2D8F80020E66802329F19974202D3F8
:100F30002DF0DCF82369424A6660D16FA760490250
:100F400003FB01F342E9073305211660A170A26893
:100F5000354901202DF020FC012840F011810623A5
:100F6000A370002133482DF055FB012840F0088183
:100F7000A3780133DBB2A3703BE7D4E901232569F1
:100F8000991AA94288BFC4E903210328B0D00133CC
:100F9000B3FBF7F207FB12320AB13B449B1A002263
:100FA00063602275D8F800203146023200202DF00F
:100FB00011FD03282BD801A353F820F0DD0D010803
:100FC00003100108DD0D0108F10E010803AD41F227
:100FD000FC162946A059002309222DF093F9012877
:100FE0007FF4FCAE0023039A2370B2F80B30B3F504
:100FF000007F6BD041F2B41203210123A15463702E
:10100000ECE6636884F814900133A3601BE7237D4A
:1010100014E700BF64E6002090F700201CF80020D1
:101020004CF7002008F7002068E6002074F8002044
:101030006CE60020D4F7002079D403084057050857
:10104000F8F700206CF8002093F8FF21AA2A7FF41B
:101050003DAFD3F8C61149B193F8C221A2F10B00FC
:1010600001282DD902F0F702062A29D0D3F8D6118B
:1010700049B193F8D221A2F10B00012820D902F046
:10108000F702062A1CD0D3F8E61149B193F8E22101
:10109000A2F10B00012813D902F0F702062A0FD0A3
:1010A000D3F8F61100293FF411AF93F8F231A3F110
:1010B0000B02012A04D903F0F703062B7FF406AFD5
:1010C00041F2FC120123A150A37080E7137C022B94
:1010D00090D192F8FE31552B8CD192F8FF31AA2B8A
:1010E00088D1D589A7592E492F440F60567B41F2EC
:1010F0001021731E7F2B66503FF67CAF734236EA99
:1011000003037FF477AF41F218217302013B635070
:10111000D18A01B9516A234841F20423E150B2F85F
:1011200011305B0103F2FF135B120360B2F813008E
:1011300000B9106A49001D440D44401B41F2082CBF
:1011400040F6F475B0FBF6F0A84244F80C0024D940
:101150004FF6F475A8421CD903202070D56A124AB4
:101160003B440B4441F20C2041F21C2112782350E5
:1011700065500AB92CF08EFFA3780133A3702DE6D9
:1011800002287FF42BAE41F2B4120123A354637002
:1011900024E6022222700025E1E70123237029E7DB
:1011A00064F8002084F8002044F8002030B504469C
:1011B000C06D21718389A26823F400531B041B0CAA
:1011C000838185B06379009213F0040F4FEA0332F4
:1011D0004FEA03230CBF00254FF4805503F48063CE
:1011E00002F40052ADF80450ADF80830002511F0BB
:1011F0000103ADF80620ADF80C501CD1ADF80A3053
:1012000008238A07694648BFADF80A3030F000FD70
:10121000637913F0080FE36D9A8A05BF22F0080284
:10122000120442F00802120C9A829A8942F4005287
:101230009A8105B030BD0423ADF80A300C23E0E7F5
:1012400030B50446C06DA160838923F400531B04AC
:101250001B0C8381637985B013F0040F009108BFE4
:101260000025217918BF4FF48055ADF804501A03BA
:1012700000251B0203F48063ADF80A50ADF80C5052
:10128000CD07ADF8083002F4005244BF0423ADF896
:101290000A30ADF806204CBF0C2308238A076946A4
:1012A00048BFADF80A3030F0B3FC637913F0080F93
:1012B000E36D9A8A05BF22F00802120442F0080288
:1012C000120C9A829A8942F400529A8105B030BD7C
:1012D000022810B504460BD8084B0949094A00EB0F
:1012E000400003EB401318460B60147039F0C0F84F
:1012F000601CC0B2BDE8104020F04EBFFC60002072
:10130000E473002054CB0020484B1B68B3F5FA7FF0
:1013100010B572D8464B9A89D989914224BF0022D0
:101320009A81598A1A8A914224BF00221A8241491D
:10133000DA7891F85C1072B1012A63D03E4C012238
:1013400000200A2922709A7098716CD00C2967D1FC
:101350009FED3A7A06E00A29987925D00C2956D1D2
:101360009FED377ADFED377A002818BFB0EE677A45
:10137000354CA278062A97BF3449DFED326A01EB7B
:101380008201D1ED076A217989B1013A032A0AD88D
:10139000B7EE000A80EE260A3DF07CFE23889842D4
:1013A00028BF1846208010BD9FED297ADAE79B7888
:1013B000214907EE903A0A78F8EEE77A67EE877AE5
:1013C00007EE102AB8EEC77A27EE277AF4EEC76A3E
:1013D000F1EE10FAE7DD86EEA77AFDEEC77A17EE9A
:1013E000903A102BA8BF1023012BB8BF0123DBB20A
:1013F0009A4238BF1A460A7010BD4FF00050F8F7F5
:1014000049FE87E70A299879CED00C29A8D0012A6D
:101410009FED107AA6D90A299AD19FED0F7AA1E7FC
:101420009FED067AA4E79FED0C7AA1E73C1200102D
:1014300064CC0020B40B00102C6800206F12833A9B
:101440000AD7A3396F120338C4CD00206C120508E7
:101450005304E9386F1203390F506E3A38B53C4BDC
:101460003C481A785B783C493C4C3D4D02EB4202CB
:1014700003EBC30301EB430300EB42122B6022603A
:101480003BF05AFC0021302236483DF0EDFC20684C
:1014900038F0EEFF344B03F1780102E006338B4263
:1014A00053D01A78002AF9D19C78D878844202D394
:1014B00058790028F2D02D492D4B08792D492E4C12
:1014C0000A70C822642111FB002100222B48DA6136
:1014D000C3E90112C3E90322C3E9052283F82020EE
:1014E00083F82120C4F8F40018F054FAB4F8F83066
:1014F0009FED235A234A94F8FA109FED236A5079FE
:1015000006EE903AF8EEE66A1388C5EE265A07EE24
:10151000103A1E4B1960538812791D4907EE903A14
:10152000B8EEC77AF8EEE77A1A4BC1ED005A27EE0B
:10153000067A67EE867A18725A7283ED017AC3EDE5
:10154000007ABDE838401CF01BBE0122B3E700BFA3
:1015500054CB0020FC60002046620020E473002091
:10156000E8730020B45C0020688E0020F483002023
:10157000346E00200C01002040510020DE6300206A
:10158000C0C9FB484488002017B7D138D0F80020E4
:10159000D4F80020A8F80020074B1B7853B9074B5C
:1015A00000F1200250F8041B43F8041B9042F9D1CB
:1015B00001207047002070475C8D00205D8D002069
:1015C00010B5154C94F83631002B144B14BF012282
:1015D00000221A700BD0042204F58E7110483DF0E1
:1015E00081FC142204F221110E483DF07BFC94F89A
:1015F0003731002B0C4B14BF012200221A7009D086
:101600000A4B0B4A03F1200153F8040B42F8040B78
:101610008B42F9D110BD00BF405100207D8D0020CC
:101620007E8D0020838D00205C8D00203C520020A8
:101630005D8D00200B4B1B7810B58BB90A4B0B4A04
:1016400003F1200153F8040B42F8040B8B42F9D14B
:10165000074B012483F83741FFF7B2FF204610BD46
:101660000020FCE75C8D00205D8D00203C520020B6
:101670004051002038B50C4B1B789BB90B4D0C49E1
:10168000042205F58E703DF02DFC01241422094939
:1016900005F221103DF026FC85F83641FFF790FF5A
:1016A000204638BD0020FCE77D8D00204051002001
:1016B0007E8D0020838D0020F0B50C2934D8DFE822
:1016C00001F08A3333335F3333333433333307003A
:1016D000048C9689B2F802C01788744D24F48054A3
:1016E0002404240C0484038C8488818B23F4005309
:1016F00021F4E6411B0409041B0C46EA0C06090C04
:1017000043EA063341EA0721A8429BB2A4B289B258
:1017100000F09E8005F58065A84200F099809268EF
:101720008480818302640384F0BD048C9589B2F8BF
:1017300002E017885D4E24F480742404240C048491
:10174000038CB0F804C0818B23F400731B0421F0D8
:10175000730145EA0E041B0C090443EA0423090C37
:10176000B0429BB21FFA8CF541EA07015BD0504CA6
:10177000A04258D0926885808183C2630384F0BD03
:10178000048C9589B2F802E0B2F800C0474E24F00C
:1017900010042404240C0484038C8788018B23F018
:1017A000200321F4E6411B0409041B0C45EA0E0446
:1017B000090C43EA041341EA0C21B0429BB2BFB2C8
:1017C00089B25BD03A4CA04258D09268878001839E
:1017D00082630384F0BD048C9589B2F802C0178837
:1017E000324E24F001042404240C0484018C8488E7
:1017F000038B21F0020123F0730309041B04090C7D
:1018000045EA0C051B0CB04241EA0501A4B243EACB
:10181000070324D0264DA84221D0926884800383F8
:1018200042630184F0BDD489168A578A23F4006389
:1018300043EA04234FF6FF341C40938825F44055B7
:101840003E4344EA032345EA06149BB2A5B291E75E
:10185000158A24F4804444EA8514A4B25FE7D6894B
:10186000158A578A21F008013143968824F4407480
:1018700021F004013D4331432C43CEE7D489168A3D
:10188000B2F812C023F0800343EA04134FF6BF748A
:101890001C40938827F4406546EA0C0644EA03138B
:1018A00045EA86049BB2A7B28FE700BF0000014063
:1018B000000401402DE9F84F4FF48C720021DFF84D
:1018C0005C828C488C4C8D4E8D4FDFF85492DFF843
:1018D00054A23DF0C9FA8B4A8B48DFF84CC2DFF8BE
:1018E0004CE208F5D87145462B68934200F0C3805E
:1018F000B3F1804F00F0C680A34200F0CA80B3422B
:1019000000F0D680BB4200F0D680634500F0D68060
:10191000734500F0D6804B4500F0D680534500F06B
:10192000D680DFF80CB25B4500F0D4800BF5806BFD
:101930005B4500F0D280ABF5983B5B4500F0D08072
:101940000BF5806B5B4500F0CE800BF5806B5B4543
:1019500000F0CC802435A942C6D16C4F6C4E4FF0BC
:10196000030A4FF0020998F80630002B7CD098F853
:1019700004301C09013C032C03F00F0374D837F822
:10198000140040FA03F2D2076ED54FF0010B0BFAA8
:1019900003F3013B18403DF001F85E4B1B5D18441A
:1019A00016EBC00460D056F830305B4898F8081049
:1019B00003F13F4202F57E02920A825C02F01F00B0
:1019C0005209032A0BFA00FB6CD0042A64D0022AC5
:1019D00004D14D48426C4BEA02024264B4F804C0A0
:1019E000BCFA8CF2C2F11F0292B2D00803EB800065
:1019F00002F00702046A92004FF00F0E0EFA02FE88
:101A000024EA0E040462046A01FA02F2224302622A
:101A10004FF0010E00220EFA02F434EA0C0120D13C
:101A20005000D3F800B00AFA00F1C9430BEA010BE9
:101A3000C3F800B0D3F800B009FA00F040EA0B0098
:101A4000186098680840986098689860586820EA1C
:101A500004045C6058685860D8680140D960D9684F
:101A6000D9600132102AD6D108F1240845457FF407
:101A70007AAFBDE8F88F4FF0010B436C43EA0B03DC
:101A8000436467E74FF0010B036C43EA0B03036405
:101A900060E74FF0020BF7E71B48026B4BEA0202CC
:101AA00002639BE71848026C4BEA0202026495E766
:101AB0004FF0040BE8E74FF0080BE5E74FF0100B91
:101AC000E2E74FF0200BDFE74FF0020BD5E74FF4D2
:101AD000803BD2E74FF4003BCFE74FF4802BCCE7BD
:101AE0004FF0400BD0E74FF0800BCDE74FF4807BF9
:101AF000CAE700BF98C7002000040040000800406B
:101B0000000C00400000014000380240BC4C0508B9
:101B1000A0B60020C44C0508604A05080C4B050817
:101B2000000401400040014000100040001400404B
:101B30000044014000B9704703682DE9F04F03F1FC
:101B40003F4404F57E04534EA40A0125345D04F09D
:101B50001F066409032C05FA06F500F09580042C95
:101B600000F08D80022C45D08588B5FA85F0C0F153
:101B70001F0080B2C40803EB840400F00700266A4B
:101B800080000F27874026EA07062662276A01F0B1
:101B900003068240701E3A4301282262C1F3810E7F
:101BA000C1F300184FF000024FEA51114FF0010C41
:101BB00025D94FF0030E0CFA02F0A84315D15000BE
:101BC0001F680EFA00F4E44327401F60D3F800803A
:101BD00006FA00F747EA08071F60DF683C40DC6050
:101BE000DC6801FA00F02043D8600132102AE2D10B
:101BF000BDE8F08F284C666C35436564B4E74FF060
:101C000003090CFA02F737EA050033D15000D3F884
:101C100000A009FA00F4E4430AEA040AC3F800A0A9
:101C2000D3F800B006FA00FA4AEA0B0AC3F800A09B
:101C3000D3F808A004EA0A0AC3F808A0D3F808B049
:101C40000EFA00FA4AEA0B0AC3F808A0D3F804A077
:101C50002AEA07075F60D3F804A008FA02F747EA08
:101C60000A075F60DF683C40DC60DC6801FA00F076
:101C70002043D8600132102AC3D1BDE8F08F064C52
:101C8000266B354325636FE7034C266C354325648B
:101C90006AE700BF604A05080038024003682DE982
:101CA000F04F03F13F4404F57E04534EA40A01258E
:101CB000345D04F01F066409032C05FA06F500F0F4
:101CC0009580042C00F08D80022C46D08588B5FAD2
:101CD00085F0C0F11F0080B2C40803EB840400F05B
:101CE0000700266A80000F27874026EA070626623B
:101CF000276A01F0030602FA00F0721E3843012A37
:101D0000C1F3810EC1F3001820624FEA51114FF068
:101D100000024FF0010C25D94FF0030E0CFA02F02F
:101D2000A84315D150001F680EFA00F4E443274081
:101D30001F60D3F8008006FA00F747EA08071F6023
:101D4000DF683C40DC60DC6801FA00F02043D860CA
:101D50000132102AE2D1BDE8F08F284C666C354381
:101D60006564B3E74FF003090CFA02F737EA0500A0
:101D700033D15000D3F800A009FA00F4E4430AEA92
:101D8000040AC3F800A0D3F800B006FA00FA4AEA41
:101D90000B0AC3F800A0D3F808A004EA0A0AC3F8A3
:101DA00008A0D3F808B00EFA00FA4AEA0B0AC3F802
:101DB00008A0D3F804A02AEA07075F60D3F804A0BC
:101DC00008FA02F747EA0A075F60DF683C40DC6018
:101DD000DC6801FA00F02043D8600132102AC3D138
:101DE000B9E7064C266B354325636FE7034C266C39
:101DF000354325646AE700BF604A050800380240A1
:101E000010B50409013C032C17D80E4B33F81420ED
:101E100000F00F0042FA00F313F001030FD001238A
:101E200003FA00F0013810403CF0B8FD064A074BB9
:101E3000125D104403EBC00010BD002010BD184619
:101E400010BD00BFBC4C0508C44C0508A0B600205E
:101E50002DE9F843304D2B8AB5F80C8018EA0308B9
:101E600027D02E4E4FF00047B8FA88F327FA03F236
:101E7000D24391B21B3B08EA02082982042B15D8F1
:101E8000DFE803F0372D23190300D6F81431002BB7
:101E900039D1EB6A1FFA83F9D6F8104134B12368BF
:101EA0002046494698476468002CF8D1B8F1000FE5
:101EB000DAD1BDE8F883D6F8F000696B036889B21F
:101EC0009847B8F1000FCFD1F3E7D6F8F400A96B2B
:101ED000036889B29847B8F1000FC5D1E9E7D6F891
:101EE000F800E96B036889B29847B8F1000FBBD1DD
:101EF000DFE7D6F8FC00296C036889B29847B8F18F
:101F0000000FB1D1D5E703F1FF3900231FFA89F99A
:101F1000C6F81431C0E700BF0040014098C7002058
:101F20002DE9F843304D2B8AB5F80C8018EA0308E8
:101F300027D02E4E4FF00047B8FA88F327FA03F265
:101F4000D24391B21B3B08EA02082982042B15D820
:101F5000DFE803F0372D23190300D6F8EC30002B0F
:101F600039D1EB6A1FFA83F9D6F8E84034B1236817
:101F70002046494698476468002CF8D1B8F1000F14
:101F8000DAD1BDE8F883D6F8C800696B036889B276
:101F90009847B8F1000FCFD1F3E7D6F8CC00A96B82
:101FA000036889B29847B8F1000FC5D1E9E7D6F8C0
:101FB000D000E96B036889B29847B8F1000FBBD134
:101FC000DFE7D6F8D400296C036889B29847B8F1E6
:101FD000000FB1D1D5E703F1FF3900231FFA89F9CA
:101FE000C6F8EC30C0E700BF0004014098C70020ED
:101FF0002DE9F843304D2B8AB5F80C8018EA030818
:1020000027D02E4E4FF00047B8FA88F327FA03F294
:10201000D24391B21B3B08EA02082982042B15D84F
:10202000DFE803F0372D23190300D6F8EC30002B3E
:1020300039D1EB6A1FFA83F9D6F8E84034B1236846
:102040002046494698476468002CF8D1B8F1000F43
:10205000DAD1BDE8F883D6F8C800696B036889B2A5
:102060009847B8F1000FCFD1F3E7D6F8CC00A96BB1
:10207000036889B29847B8F1000FC5D1E9E7D6F8EF
:10208000D000E96B036889B29847B8F1000FBBD163
:10209000DFE7D6F8D400296C036889B29847B8F115
:1020A000000FB1D1D5E703F1FF3900231FFA89F9F9
:1020B000C6F8EC30C0E700BF0004014098C700201C
:1020C0002DE9F843304D2B8AB5F80C8018EA030847
:1020D00027D02E4E4FF00047B8FA88F327FA03F2C4
:1020E000D24391B21B3B08EA02082982042B15D87F
:1020F000DFE803F0372D23190300D6F8C430002B96
:1021000039D1EB6A1FFA83F9D6F8C04034B123689D
:102110002046494698476468002CF8D1B8F1000F72
:10212000DAD1BDE8F883D6F8A000696B036889B2FC
:102130009847B8F1000FCFD1F3E7D6F8A400A96B08
:10214000036889B29847B8F1000FC5D1E9E7D6F81E
:10215000A800E96B036889B29847B8F1000FBBD1BA
:10216000DFE7D6F8AC00296C036889B29847B8F16C
:10217000000FB1D1D5E703F1FF3900231FFA89F928
:10218000C6F8C430C0E700BF000C004098C700206C
:102190002DE9F8432F4D2B8AB5F80C8018EA030877
:1021A00027D02D4E4FF00047B8FA88F327FA03F2F4
:1021B000D24391B21B3B08EA02082982042B15D8AE
:1021C000DFE803F0352B22190300D6F89C30002BF2
:1021D00037D1EB6A1FFA83F9D6F8984034B12368F7
:1021E0002046494698476468002CF8D1B8F1000FA2
:1021F000DAD1BDE8F883B06F696B036889B298479C
:10220000B8F1000FD0D1F4E7F06FA96B036889B281
:102210009847B8F1000FC7D1EBE7D6F88000E96B1B
:10222000036889B29847B8F1000FBDD1E1E7D6F84D
:102230008400296C036889B29847B8F1000FB3D1C4
:10224000D7E703F1FF3900231FFA89F9C6F89C305C
:10225000C2E700BF0008004098C700202DE9F843FE
:102260002C4D2B8AB5F80C8018EA030825D02A4E8D
:102270004FF00047B8FA88F327FA03F2D24391B23D
:102280001B3B08EA02082982042B13D8DFE803F07D
:10229000322920170300736F002B34D1EB6A1FFA29
:1022A00083F9346F34B123682046494698476468FF
:1022B000002CF8D1B8F1000FDCD1BDE8F883306D07
:1022C000696B036889B29847B8F1000FD2D1F4E77F
:1022D000706DA96B036889B29847B8F1000FC9D136
:1022E000EBE7B06DE96B036889B29847B8F1000F6E
:1022F000C0D1E2E7F06D296C036889B29847B8F164
:10230000000FB7D1D9E703F1FF3900231FFA89F98C
:102310007367C6E70004004098C700202DE9F84322
:102320004FF080452B8AB5F80C8018EA030825D0B9
:10233000294E4FF00047B8FA88F327FA03F2D24348
:1023400091B21B3B08EA02082982042B13D8DFE86C
:1023500003F0322920170300F36C002B34D1EB6A11
:102360001FFA83F9B46C34B1236820464946984774
:102370006468002CF8D1B8F1000FDCD1BDE8F88317
:10238000B06A696B036889B29847B8F1000FD2D17F
:10239000F4E7F06AA96B036889B29847B8F1000FB7
:1023A000C9D1EBE7306BE96B036889B29847B8F1A4
:1023B000000FC0D1E2E7706B296C036889B29847BF
:1023C000B8F1000FB7D1D9E703F1FF3900231FFAA5
:1023D00089F9F364C6E700BF98C700202DE9F843E8
:1023E0002C4D2B8AB5F80C8018EA030825D02A4E0C
:1023F0004FF00047B8FA88F327FA03F2D24391B2BC
:102400001B3B08EA02082982042B13D8DFE803F0FB
:10241000322920170300736A002B34D1EB6A1FFAAC
:1024200083F9346A34B12368204649469847646882
:10243000002CF8D1B8F1000FDCD1BDE8F88330688A
:10244000696B036889B29847B8F1000FD2D1F4E7FD
:102450007068A96B036889B29847B8F1000FC9D1B9
:10246000EBE7B068E96B036889B29847B8F1000FF1
:10247000C0D1E2E7F068296C036889B29847B8F1E7
:10248000000FB7D1D9E703F1FF3900231FFA89F90B
:102490007362C6E70000014098C700202DE9F843A9
:1024A0002C4D2B8AB5F80C8018EA030825D02A4E4B
:1024B0004FF00047B8FA88F327FA03F2D24391B2FB
:1024C0001B3B08EA02082982042B13D8DFE803F03B
:1024D000322920170300736A002B34D1EB6A1FFAEC
:1024E00083F9346A34B123682046494698476468C2
:1024F000002CF8D1B8F1000FDCD1BDE8F8833068CA
:10250000696B036889B29847B8F1000FD2D1F4E73C
:102510007068A96B036889B29847B8F1000FC9D1F8
:10252000EBE7B068E96B036889B29847B8F1000F30
:10253000C0D1E2E7F068296C036889B29847B8F126
:10254000000FB7D1D9E703F1FF3900231FFA89F94A
:102550007362C6E70000014098C70020F0B5066826
:10256000484CB30AA34200F08A8009D9464CA342E2
:102570007FD00F34A34265D0103CA34266D0F0BD9B
:10258000023CA34278D05AD8B3F5801FF7D1482730
:1025900001254379B6F80CE0022023FA00F4A040AC
:1025A0001FFA80FCA8002346441903EB4403374C70
:1025B000002953D04CEA0E0C03F1040E44F823100A
:1025C00044F82E20A6F80CC0E319EFF31181502235
:1025D00082F31288421904EBC202D2F810C0BCF197
:1025E000000F03D044F807C013690433421904EB09
:1025F000C202576917B11F6053690433421904EBD3
:10260000C202976917B11F6093690433421904EB42
:10261000C202D76917B11F60D36904330027CAB259
:102620001F6082F31188284404EBC004236A83B935
:10263000B38923F001031B041B0CB381F0BD982761
:102640000325A6E74FF488770625A2E72027002573
:102650009FE7B38943F00103B381F0BD2EEA0C0C70
:1026600003F1040EA6F80CC044F8231044F82E2001
:10267000AAE7E82705258CE77027022589E7C02708
:10268000042586E7030010004100100098C70020D1
:1026900010B503687C487D4C0139834282B02468C0
:1026A00089B200F0AF80A0F58060834200F0AA807C
:1026B00000F58040834200F0818000F58060834215
:1026C0007CD000F58060834278D018886408B4FB21
:1026D000F2F4013CA4B282B2B3F1804F0AD06C484C
:1026E000834207D000F58060834203D000F580600C
:1026F000834202D122F0700292B26648834200F017
:102700008F8000F58060834200F0938022F4407255
:1027100000F56C4092B283421A80D9621C8540F069
:102720009180012100221A86998219885A4841F025
:1027300001018342198049D0B3F1804F00F08D80B0
:10274000534A934200F08B8002F58062934200F07E
:10275000888002F58062934200F0858002F58062F5
:10276000934200F0828002F5806293427FD002F5AE
:10277000704293427DD002F5705293427BD002F5B5
:102780008062934279D002F58062934277D0A2F5BD
:102790009832934275D002F58062934215D002F5CB
:1027A0008062934208BF0D2210D002A84FF001238F
:1027B00040F8043D2EF0E8FC02B010BD1888B4FBD0
:1027C000F2F4013CA4B282B286E70C22334B03EB55
:1027D000C20201A854798DF80440012300228DF82B
:1027E00005308DF807308DF806202EF0CDFC1B2C1F
:1027F0000FD02E2CE0D12A4B019301A82EF0C4FC5F
:1028000002B010BD1888B4FBF2F4013CA4B282B24D
:1028100070E7244B019301A82EF0B6FC02B010BD66
:1028200001201A80D9621C8598821A8802431A8076
:1028300086E701201A80D9621C8598821A88024393
:102840001A8079E7104A93423FF46BAF01229A82D3
:102850001A8842F001021A806EE70122B6E70222CE
:10286000B4E70322B2E70422B0E70522AEE706226E
:10287000ACE70722AAE70822A8E70922A6E70A226E
:10288000A4E70B22A2E700BF0004014064DA0020A5
:10289000000400400010004000000140FC4C05080E
:1028A0002C010001190100012B4B98423CD0B0F1E2
:1028B000804F3BD0A3F57C43984239D003F5806329
:1028C000984237D003F58063984235D003F5806392
:1028D000984233D003F58063984233D003F57043B8
:1028E000984231D003F57053984229D003F58063A4
:1028F00098422BD003F58063984229D0A3F59833F2
:10290000984227D003F58063984207D003F580638F
:10291000984208BF0D2202D0002070470C220F4BB6
:1029200003EBC203187970470022F8E70122F6E7AB
:102930000222F4E70322F2E70422F0E70522EEE7A1
:102940000822ECE70622EAE70722E8E70922E6E7A1
:102950000A22E4E70B22E2E700000140FC4C0508F4
:1029600070B4104E002332461D46012403E00133AB
:102970000C2B0CD0947930EA040402F12402F6D135
:10298000A94207D0013301350C2BEDB2F2D1002062
:1029900070BC704703EBC30306EB830370BC18796C
:1029A000704700BF0C4B0508C0B110B40C4C13218C
:1029B0002246002300E01179884202F1240206D069
:1029C00001330C2BF7D100205DF8044B704703EB6B
:1029D000C30304EB83005DF8044B7047704700BFEE
:1029E0000C4B0508F8B5B8490B78A3F11702022A79
:1029F0000FD9B64A12F83300002840F02B81D800D6
:102A0000024452782AB1B24A12F83330002B00F057
:102A1000E4810024AF4EB04F2546315B4B0803F0F4
:102A200077334FEA910C0CF0333CCB1ACA08A3EB76
:102A30000C0302F011329B1A03EB231303F00F3344
:102A4000A7FB03C2D209C2EB02229A1A11F00103BA
:102A50001CBF0135EDB2012A06EB040004F10804A5
:102A60000BDD022A40F0E98013B111F42F7F04D16D
:102A70001AF090FF002800F0E080402CCDD1013DFD
:102A8000022D00F2DA8002201FF0C2F9002800F0C7
:102A9000DD80924A5378052B00F2CB80904903EBFE
:102AA000C30301EB430113788E488F4C0160022B66
:102AB00000F2BB8003EB430104EB411103EB430342
:102AC00004EB4313894D9A88D88829609042884D39
:102AD00024BF00229A80AB78042B00F0C48033B965
:102AE0002B88B3F5F07F84BF4FF4F0732B80814EB9
:102AF000FEF70AFC3568804B2B40002B00F07581F7
:102B0000EA0700F1BE806B0400F1C2802F0700F1DC
:102B1000C680A80400F1CA802904784E7DD5002320
:102B2000F37386F823303AF0F9F8002858D0737E12
:102B3000032B55D05A1E012A67D900232383A4F8FA
:102B40007830A4F8D8303AF0E9F800285CD10023B6
:102B5000EA0484F84F3084F8AF3084F80F3159D547
:102B6000674BDA79022A08BF01224FF00A0008BF3A
:102B7000DA7139F0E9FF002840F0D0804FF480602E
:102B80001FF046F9002800F02B814FF40070F7F792
:102B900081FA4FF40010F7F77DFA5A4C4FF00070AD
:102BA000F7F778FA4FF08060F7F774FAA388002BF4
:102BB00040F08180544A1368DB0DDB050BB1002324
:102BC0001360936823F4007323F002030BB1002316
:102BD00093601379013B042B01D901231371F8BDD4
:102BE0000023A3816382A4F86C30A4F87230A4F8A7
:102BF000CC30A4F8D2303AF091F800289DD0737E02
:102C00005A1E012A99D800E0737E023B022B9ED8FF
:102C1000EA04A5D42B06B1D4A2E7F37B002B00F085
:102C2000D080002386F823307DE7002321461370EF
:102C300044E700232A49537035E726481EF0D8FBA5
:102C400002201FF0E5F800287FF423AF8020F7F77B
:102C500021FA1EE7D80014186468002C7FF4D0AE67
:102C600017240C70CCE64FF48050F7F713FAAB8AB8
:102C7000B3F57A7F37BF4FF47A72AB78AB78AA821C
:102C80002DE72248F7F706FA35686B047FF53EAF6B
:102C90001F48F7F7FFF935682F077FF53AAF1D4852
:102CA000F7F7F8F93568A8047FF536AF1A48F7F753
:102CB000F1F9356830E72078FFF776FE00287FF4D9
:102CC00079AFA08076E700BFEC6600206C4D050868
:102CD000E45305086CE300208180808054CB002001
:102CE00046620020E8730020FC600020E4730020AE
:102CF000C4CD0020A0640020096000026CDA00202E
:102D0000F48300201A5D0020CC8F002008600002B0
:102D1000092000020160000209400002354F002234
:102D200007F1060E1146944601EB4100430017F8E7
:102D300010000A2807EB030540D05B1B28464E1CF9
:102D4000EABB7344142E1D443FF418AF10F8062F4D
:102D50000A2A08D00136142E1D443FF40FAF10F894
:102D6000062F0A2AF6D101229319132B15D803EB4B
:102D7000430007EB400117F810000A2808BF013391
:102D800005D012E011F8064F0A2C0ED10346132B82
:102D900002F1010203F10100F4D9C5F800C0A5F861
:102DA00004C0711C1429BFD1E8E603EB430307EB11
:102DB0004303196829609B88AB80F2E752B10E4645
:102DC000D2E742F201031D423FF4ADAE002386F884
:102DD0002330A8E60E460122C6E718230B7018E63A
:102DE0004FF00060F7F756F9CFE645F0080535607B
:102DF00086E600BF688E00202DE9F84F27F00AFE16
:102E00002B4B2C4A934250D22B4F03F114069B4676
:102E10004FF00108294C258862197DB1BA420DD2C4
:102E2000052D0BD936F8143C6188C3F30B03994286
:102E30000AD0144625886219002DEFD156F8101CCF
:102E40005846F8F7B1FA0FE0637913F0030AF0D1AE
:102E500056F8101C94F804905846F8F7A5FA36F87E
:102E6000141CB9EB113F11D04FF00008114B0BF1BE
:102E7000140B9B4506F11406CCD3FFF7B3FDFEF708
:102E8000EDFA27F0A7FD4046BDE8F88F36F8123C72
:102E900056F8100CAA1FC3F30B039A4204F1060163
:102EA000A8BF1A463BF07AFFE0E74FF00108E4E7DD
:102EB0009001000808070008008000080240000890
:102EC0002DE98048013085B0C3B20393954C964FED
:102ED000DFF860A2954D964E0A2302932FF0A6FECE
:102EE0004FF4FA73DFF850E201934FF01008DAF86C
:102EF0000430C3F30803002B40F0D280EFF31183BA
:102F0000002B40F0CD802068AA6823689842FAD14F
:102F100033689A42F7D8D7F800C04FF47A7101FBB2
:102F20000CF39B1AB3FBFCF301FB00304FF47A7CEB
:102F30004FF00109DAF80430C3F30803002B40F026
:102F40009180EFF31183002B40F08C802368A968F7
:102F500022689342FAD132689142F7D83A680CFB62
:102F600002FBABEB0101B1FBF2F10CFB03131B1AEB
:102F7000B3F57A7FDED3019B013B0193B7D1039870
:102F80002FF0B0FC4FF47A73DFF8ACE101934FF00F
:102F90001008DAF80430C3F30803002B40F0A180D6
:102FA000EFF31183002B40F09C802068AA6823680F
:102FB0009842FAD133689A42F7D8D7F800C04FF454
:102FC0007A7101FB0CF39B1AB3FBFCF301FB00309D
:102FD0004FF47A7C4FF00109DAF80430C3F30803A8
:102FE00013BBEFF31183FBB92368A96822689342EE
:102FF000FAD132689142F7D83A680CFB02FBABEB8E
:103000000101B1FBF2F10CFB03131B1AB3F57A7F3C
:10301000E2D3019B013B0193BBD1029B013B029395
:103020007FF45CAFFAF7A6F8EFF3118188F312880A
:10303000D5F808B02B68DB0344BFCEF80090D5F874
:1030400008B02368DEF80020C9B281F3118839681E
:1030500013440CFB01F2A2EB0B02B2FBF1F20CFBEE
:103060000323D2E7EFF3118188F31288D5F808B073
:103070002B68DB0344BFCEF80090D5F808B0236876
:10308000DEF80020C9B281F31188396813440CFBC3
:1030900001F2A2EB0B02B2FBF1F20CFB032366E799
:1030A000EFF3118388F31288D5F808C02A68D20399
:1030B00004D50122CEF80020D5F808C02068DEF83B
:1030C0000090DBB283F3118839684FF47A72484478
:1030D00002FB01F3A3EB0C03B3FBF1F302FB0030A3
:1030E00024E7EFF3118388F31288D5F808C02A6823
:1030F000D20304D50122CEF80020D5F808C02068FC
:10310000DEF80090DBB283F3118839684FF47A72ED
:10311000484402FB01F3A3EB0C03B3FBF1F302FB06
:10312000003055E794B6002098B6002010E000E08B
:103130009CB6002000ED00E090B600202DE9F04F95
:103140008DB0FFF74FFCDFF87C91594FDFF87881A5
:1031500027F060FC574A584B128FADF80620A3EBBE
:10316000090300934FF0030A0026CDE90866CDE974
:103170000A66009BCDF818900793D8F81030002B02
:10318000C0F28E8001238DF82C30F323C8F80C3068
:103190000222BDF80630ADF8083002A906A8F7F7FC
:1031A0001FF8022202A94FF6FF70F7F7A9FE434B62
:1031B000BB42834629D21C46658823888DF815605A
:1031C000C5F30B05C3F30B00A91D1B0B0622ADF8BD
:1031D0001010ADF8120004A906A88DF81430F6F707
:1031E000FFFF5846062204A9F7F78AFE6168834666
:1031F0002A4606A8F6F7F4FF616858462A46F7F70C
:103200007FFE1434BC428346D6D3022203A906A80B
:10321000ADF80C60F6F7E4FF022203A95846F7F771
:103220006FFE40BAC343022204A906A8ADF81030CD
:10323000F6F7D6FF099818BB0A989DF82C3033B9D9
:1032400068B1BAF1010A90D10520FFF739FED8F82C
:10325000103043F00043C8F810300028F1D199F83D
:103260000030AB2BF0D199F80130BE2BECD1F7F741
:1032700061FE0028E8D027F0ADFB0DB0BDE8F08F6F
:1032800008ABC0F10402002118443BF0EDFD0A98A0
:1032900018B9089906A8F6F705FFCDE90960CCE74B
:1032A000074BC8F8043003F18833C8F8043069E7E5
:1032B000080700086C12050800800008900100084B
:1032C0002301674500400008003C024008B5FFF7B5
:1032D00035FFFFF791FD0120BDE808401EF05CBFFF
:1032E0002DE9F047D54C2DED028B636820469847B9
:1032F000002800F0D080D24B1B780122042B84F8E8
:10330000342000F0CC80B4F9163006EE903AB4F9CF
:10331000183007EE103AB4F91A3007EE903AF8EE8A
:10332000E66AB8EEC77AF8EEE77AC4ED0A6A84ED89
:103330000B7AC4ED0C7AC34B1B88002B60D0C24BB8
:1033400094ED0A2AD4ED0B2A94ED0C3A93ED008A01
:10335000D3ED054A93ED090AD3ED0E3AD3ED120AE7
:1033600093ED174A93ED011A93ED065AD3ED0A1A1D
:1033700093ED0F6AD3ED137A93ED187AD3ED045AD7
:10338000D3ED0D6AE8EE024AE0EE223AA3EE204ABF
:10339000A1EE025AA1EEA26AA3EE277A93ED038A68
:1033A000D3ED167A93ED020AD3ED0C0A93ED0B1AC6
:1033B000D3ED151AC4ED0A4A65EEE45AA8EE645A34
:1033C00066EEE36AD3ED144A83ED055A67EEC47ADC
:1033D000E0EE025AA0EEE36AE1EE226AA4EE617A20
:1033E000E3EE247AC3ED065AC4ED0B3A83ED0E6A80
:1033F000C3ED0F6A83ED177AC3ED187A84ED0C4A9A
:10340000924EA17F9248934D16F05EF93288D5F81E
:10341000F430002A40F098808F4A126852075BD43B
:10342000B3F9002094ED0B6A94ED0C7A94ED0A5AEE
:103430008A4905EE902AB3F90220B3F9043006EE6A
:10344000902A07EE903AF8EEE55A854B0A68D3EDDC
:10345000003A93ED014AD3ED024AF8EEE66AF8EE3F
:10346000E77A75EE655A76EE666A77EE677AC4EDAE
:103470000A5A34EE266A73EEA55A34EEA77A013260
:10348000C3ED005AC4ED0B6A83ED016AC4ED0C7AFA
:1034900083ED027A0A60BDEC028BBDE8F087B4F9D7
:1034A0001600B4F91810B4F91A206E4B07EE900A02
:1034B000F8EEE76A07EE901AB8EEE77A07EE902A80
:1034C000F8EEE77AC4ED0A6A188059809A8084ED94
:1034D0000B7AC4ED0C7A2EE7634E3288322A00F064
:1034E000CD80002A40F01881604E3278002A97D0B3
:1034F0005F4FD5F85821D5F85011D5F8540187FB06
:1035000002ECD217C2EB2C12B4F814C0A2EB0C02DE
:103510009A8087FB01C287FB00C7C017C0EB27104A
:10352000C917544F5880C1EB221100223270198004
:10353000BA81FA81FFF702FEFFF75EFC01201EF060
:103540002BFED5F8F4306BE7B2F5C87F18BFD5ED88
:103550004E7AD4ED0A6A0CBF9FED477AB8EEE77A4F
:10356000DFED457A0022C4ED0A7A1A803288378866
:1035700037EE267AB2F5C87F18BFD5ED4F7ABDEE8B
:10358000C77A18BFF8EEE77A17EE101A85ED4E7A73
:1035900094ED0B7A77EE877A0020FDEEE77A4FF014
:1035A000000CB7F5C87FE06217EE902AA3F802C0BE
:1035B000C5ED4F7A00F0A680D5ED507A94ED0C7AE7
:1035C0002063F8EEE77A012F77EE877AA3F804C03C
:1035D000FDEEE77A17EE900AC5ED507A2AD1DFF8B2
:1035E00090E0B4F81480C8308EFB00A9C831C8320E
:1035F000C017C0EBE9108EFB01A98EFB02AED217FB
:10360000C2EBEE12C917DFF86CE05A80C1EBE9118A
:10361000A0EB080098801980AEF80CC0AEF80EC080
:10362000FFF78CFDFFF7E8FB38461EF0B5FD378845
:10363000D5F8F430013F3780EEE600BF600B001094
:1036400049B60020E8630020EC63002054570020B6
:10365000880B00104051002084CC002094F80020FA
:1036600098F800204CB60020A65C0020A45C002046
:103670001F85EB51D863002000000000384A19680C
:10368000D268C5F84C219FED377A9A88C5F8441165
:10369000A5F84821DFED337AD4ED0A6AC4ED0A7A41
:1036A00000221A80328837EE267A322A18BFD5EDEA
:1036B000557A3288BDEEC77A18BFF8EEE77A85ED05
:1036C000547A94ED0B7A77EE877A0020FDEEE77A54
:1036D0000021322AE062C5ED557A598036D0D5ED09
:1036E000567A94ED0C7A2063F8EEE77A012A77EEA9
:1036F000877A9980FDEEE77AC5ED567A11D0013AC6
:103700003280F1E6D4ED0C7A2063FDEEE77AA3F87F
:1037100004C0C5ED507A8DE7D5ED547AB8EEE77A5E
:10372000B8E71148114B01700B201A701EF01CFCF9
:10373000D5F8F430D5F8442109491A60B5F8487134
:10374000D5F84C019F803288C860D8E7D4ED0C7A58
:103750002063FDEEE77A9980C5ED567ACFE700BF8A
:10376000D863002000000000A85C0020A35C0020BB
:1037700008B5F7F73DFEFFF7E1FCBDE80840FDF7AF
:103780006DBE00BF2DE9F04F85B0CDE902109B4D15
:10379000DFF878A2029B013B0293013300F02A81FB
:1037A0002FF044FA964C974FDFF864E2964E4FF4B0
:1037B000FA7301934FF01008DEF80430C3F30803E6
:1037C000002B40F0F680EFF31183002B40F0F180E6
:1037D0002068AA6823689842FAD133689A42F7D8D9
:1037E000D7F800C04FF47A7101FB0CF39B1AB3FBBE
:1037F000FCF301FB00304FF47A7C4FF00109DEF856
:103800000430C3F30803002B40F0B580EFF31183BD
:10381000002B40F0B0802368A96822689342FAD157
:1038200032689142F7D83A680CFB02FBABEB01011E
:10383000B1FBF2F10CFB03131B1AB3F57A7FDED355
:10384000019B013B0193B7D1039B6F4E581CC0B243
:103850002FF048F8DFF8B8E14FF47A730193DEF8FF
:103860000430C3F308034FF01008002B44D1EFF3EA
:103870001183002B40D12068AA6823689842FAD1AE
:1038800033689A42F7D8D7F800C04FF47A7101FB39
:103890000CF39B1AB3FBFCF301FB00304FF47A7C72
:1038A0004FF00109DEF80430C3F30803002B44D1C4
:1038B000EFF31183002B40D12368A968226893425B
:1038C000FAD132689142F7D83A680CFB02FBABEBB5
:1038D0000101B1FBF2F10CFB03131B1AB3F57A7F64
:1038E000E0D3019B013B01933FF454AFDEF8043079
:1038F000C3F30803002BBAD0EFF3118388F31288C7
:10390000D5F808C02A68D20304D50122CAF80020DD
:10391000D5F808C02068DAF80090DBB283F311888C
:1039200039684FF47A72484402FB01F3A3EB0C03AD
:10393000B3FBF1F302FB0030B0E7EFF3118188F342
:103940001288D5F808B02B68DB0344BFCAF8009092
:10395000D5F808B02368DAF80020C9B281F31188DD
:10396000396813440CFB01F2A2EB0B02B2FBF1F23B
:103970000CFB0323B1E7EFF3118188F31288D5F82C
:1039800008B02B68DB0344BFCAF80090D5F808B034
:103990002368DAF80020C9B281F31188396813442A
:1039A0000CFB01F2A2EB0B02B2FBF1F20CFB0323C6
:1039B00042E7EFF3118388F31288D5F808C02A682C
:1039C000D20304D50122CAF80020D5F808C0206827
:1039D000DAF80090DBB283F3118839684FF47A7219
:1039E000484402FB01F3A3EB0C03B3FBF1F302FB2E
:1039F000003000E705B0BDE8F08F00BF10E000E048
:103A000094B6002098B600209CB6002090B6002006
:103A100000ED00E0224B5B68C3F3080330B4D3B978
:103A2000EFF31183BBB91F4A1F4D20481368846808
:103A300011688B42FAD129688C42F7D81C4A116868
:103A40004FF47A7202FB01F0001B30BCB0FBF1F0C6
:103A500002FB03007047EFF31182102383F31288F7
:103A600003F1E023D2B29C68196811F4803F114938
:103A70001EBF012008609C680A4B18680B6882F31F
:103A800011880B4A11684FF47A72034402FB01F06B
:103A9000001B30BCB0FBF1F002FB0300704700BF1D
:103AA00000ED00E094B600209CB6002010E000E09D
:103AB00098B6002090B600202DE9F84F8046274C9C
:103AC000274DDFF8A490274EFFF7A4FFDFF89CE016
:103AD000DFF89CC04FF0100A4FF47A77DCF804301E
:103AE000C3F30803CBB9EFF31183B3B92368A96813
:103AF00022689342FAD132689142F7D8DEF800206A
:103B000007FB02FBABEB0101B1FBF2F107FB031377
:103B10001B1A4345E2D3BDE8F88FEFF311818AF316
:103B20001288D5F808B02B68DB0304D50123C9F847
:103B30000030D5F808B02368D9F80020C9B281F365
:103B40001188DEF80010134407FB01F2A2EB0B0210
:103B5000B2FBF1F207FB0323DAE700BF94B60020C3
:103B600010E000E09CB6002090B6002098B600203F
:103B700000ED00E02DE9F04FDFF834C1494CDFF8EB
:103B800034E1DFF83481484E824648481AF1FF3A62
:103B9000C0F08680DCF80430C3F30803002B5ED14C
:103BA000EFF31183002B5AD10568A26803689D4288
:103BB000FAD133689A42F7D8DEF800704FF47A7180
:103BC00001FB07F39B1AB3FBF7F301FB0535DCF8A8
:103BD0000430C3F308034FF010094FF47A77F3B9B8
:103BE000EFF31183DBB90368A16802689342FAD14D
:103BF00032689142F7D8DEF8002007FB02FBABEBFE
:103C00000101B1FBF2F107FB03135B1BB3F57A7FF4
:103C1000BCD2DCF80430C3F30803002BE0D0EFF390
:103C2000118189F31288D4F808B02368DB0304D526
:103C30000123C8F80030D4F808B00368D8F8002091
:103C4000C9B281F31188DEF80010134407FB01F2BA
:103C5000A2EB0B02B2FBF1F207FB0323D5E7EFF374
:103C60001183102282F31288A1682268D20303D53F
:103C70000122C8F80020A168D0F80090D8F80050C0
:103C8000DBB283F31188DEF800704FF47A724D4492
:103C900002FB07F35B1AB3FBF7F302FB053596E76C
:103CA000BDE8F08F10E000E09CB6002094B6002044
:103CB00000ED00E098B6002090B6002030B4EFF39D
:103CC0001183102282F31288084809490268094DBD
:103CD000094C013202608A682A6000222260DBB24D
:103CE0000A6883F3118830BC704700BF94B6002087
:103CF00010E000E09CB6002090B6002038B5254BBF
:103D00001C69A26BE36D62B1E26BC2B1998A1A8839
:103D1000C90792B204D5120744BF4FF6F7721A8052
:103D200038BD99891A88890692B2EDD59206EBD5ED
:103D3000E26AFAB19888216B9047E36DE4E79989CC
:103D40001A880D0692B2E1D51006DFD5D4E9091222
:103D50008A420AD0A1692569885C98800132B2FB49
:103D6000F5F105FB1122A262D0E7DA6822F08002A9
:103D7000DA60CBE79B88E2696169DBB28B54E26968
:103D8000E068E36D0132B2FBF0F100FB1122E26169
:103D9000BAE700BF3C0A001038B5254BDC68A26BBF
:103DA000E36D62B1E26BC2B1998A1A88C90792B217
:103DB00004D5120744BF4FF6F7721A8038BD9989AF
:103DC0001A88890692B2EDD59206EBD5E26AFAB16D
:103DD0009888216B9047E36DE4E799891A880D066E
:103DE00092B2E1D51006DFD5D4E909128A420AD091
:103DF000A1692569885C98800132B2FBF5F105FB69
:103E00001122A262D0E7DA6822F08002DA60CBE702
:103E10009B88E2696169DBB28B54E269E068E36D1B
:103E20000132B2FBF0F100FB1122E261BAE700BF00
:103E30003C0A001038B5254B9C68A26BE36D62B15B
:103E4000E26BC2B1998A1A88C90792B204D51207E7
:103E500044BF4FF6F7721A8038BD99891A888906CF
:103E600092B2EDD59206EBD5E26AFAB19888216B51
:103E70009047E36DE4E799891A880D0692B2E1D57F
:103E80001006DFD5D4E909128A420AD0A169256952
:103E9000885C98800132B2FBF5F105FB1122A26229
:103EA000D0E7DA6822F08002DA60CBE79B88E2692B
:103EB0006169DBB28B54E269E068E36D0132B2FB09
:103EC000F0F100FB1122E261BAE700BF3C0A0010EA
:103ED00038B5254B5C68A26BE36D62B1E26BC2B191
:103EE000998A1A88C90792B204D5120744BF4FF6BF
:103EF000F7721A8038BD99891A88890692B2EDD571
:103F00009206EBD5E26AFAB19888216B9047E36D8F
:103F1000E4E799891A880D0692B2E1D51006DFD53B
:103F2000D4E909128A420AD0A1692569885C98807F
:103F30000132B2FBF5F105FB1122A262D0E7DA688B
:103F400022F08002DA60CBE79B88E2696169DBB22C
:103F50008B54E269E068E36D0132B2FBF0F100FBE3
:103F60001122E261BAE700BF3C0A001038B5254BC8
:103F70001C68A26BE36D62B1E26BC2B1998A1A88C8
:103F8000C90792B204D5120744BF4FF6F7721A80E0
:103F900038BD99891A88890692B2EDD59206EBD57B
:103FA000E26AFAB19888216B9047E36DE4E799895A
:103FB0001A880D0692B2E1D51006DFD5D4E90912B0
:103FC0008A420AD0A1692569885C98800132B2FBD7
:103FD000F5F105FB1122A262D0E7DA6822F0800237
:103FE000DA60CBE79B88E2696169DBB28B54E269F6
:103FF000E068E36D0132B2FBF0F100FB1122E261F7
:10400000BAE700BF3C0A0010002A12DD70B5044672
:104010000D468E18236820469B6898470028F9D0E3
:10402000236815F8011B1B6820469847B542F1D15B
:1040300070BD70470368DB6A03B11847704700BF63
:1040400003689B6A03B11847704700BF03682DE9F6
:10405000F0415D6A1DB12B46BDE8F0411847002ACA
:10406000174611DD04460E460F4400E023689B68A6
:10407000204698470028F9D0236816F8011B1B68D2
:1040800020469847BE42F1D1BDE8F08103689B69A4
:10409000184700BF03685B69184700BF0368DB6807
:1040A000184700BF03689B68184700BF03685B6838
:1040B000184700BF03681B68184700BF014B1B78F7
:1040C00013B17047D8710020C44B1B685B05F8D54D
:1040D0002DE9F04F2DED028BC14B1B7899B00546B1
:1040E0000BB915F0D5FABF4B1B78012B00F073828A
:1040F000BD4B1B78002B39D0BC4CBD4AD4F8803264
:10410000EB1A934200F2CE82DFF83C9399F80070EC
:10411000002F00F0CE83B74E37683FB3D4F890320B
:1041200040F6B732EB1A934220D994F88C32002B28
:1041300000F0028794F89522AF4994F894C2086879
:10414000013BDBB2013284F88C32D2B2002B00F09A
:10415000E88617F8011B84F8952201EB0C03376001
:1041600084F89432FFF7A6FFC4F89052FFF752FC90
:10417000A24B93F8008000F57A70B8F1010F10900F
:1041800000F0F1819E4B1B78002B00F0C6809D4F04
:104190003B68002B00F0C1809B4B944CD3F800800F
:1041A000D4F89C32A8EB0303632B40F2B680DFF80F
:1041B0009C92964EDFF898A2412018F01FFEB9F9A4
:1041C000023086FB0320DB17C3EBA00080B218F09F
:1041D000F9FDB9F9003086FB0320DB17C3EBA00023
:1041E00080B218F0EFFDB9F9043086FB0320DB172D
:1041F000C3EBA00080B218F0E5FD9AF80010386813
:10420000FFF758FF94F8A06216F0010B00F0AC869F
:10421000DFF84092D9F80030980670D57C4B7D4E7F
:104220001B78990742F16182B37C042B8CBF032376
:1042300002230293472018F0E1FD306818F08EFD4C
:10424000706818F08BFD744AB3893868A2FB0323A9
:10425000C3F3471B5946FFF72DFF9AF80010D9F812
:1042600000208BEA010312F0140F8AF8003002F0EC
:10427000E3826A4B186818F071FD029BB67C3868BF
:1042800043EA8606F6B23146FFF714FF9AF800308B
:1042900038685E4031468AF80060FFF70BFF94F8FB
:1042A000A06266BBDFF8B0914F2018F0A7FDD9F8E7
:1042B000000018F053FDD9F8040018F04FFD304607
:1042C00018F04CFD01213868FFF7F4FE504A9AF8C7
:1042D00000301678386806F00106314683F0010395
:1042E0008AF80030FFF7E6FE9AF8003038685E4042
:1042F00031468AF80060FFF7DDFE94F8A062484A74
:10430000C4F89C82731CDBB2A2FB0312D20802EB3E
:104310008202A3EB420384F8A032424F97F8008058
:10432000B8F1020F00F096833F4CA379032B00F005
:10433000A5833E4B1B78002B3CD03D4F3B68CBB355
:104340002A4CFFF767FBD4F8A832029044F61F62AC
:10435000C31A93422ED994F8AE32002B01F0EC83AD
:10436000013B84F8AE3294F8AF62002E01F0BE82B9
:10437000013E84F8AF6294F8B232002B00F08287DD
:10438000013B84F8B23294F8B6C2BCF1000F00F0E1
:1043900078860CF1FF3C84F8B6C294F8B792B9F174
:1043A000000F01F0238509F1FF3984F8B792029BD1
:1043B000C4F8A8321F4B1B78002B40F0DE821E4E43
:1043C0003378002B00F089801C4B1B78002B56D0D3
:1043D000064F1B4C1B4D07F582663FE084CC002046
:1043E0000F6700208D7400209A7400204051002037
:1043F0003F0D030004740020FC7300209B74002018
:10440000A8740020D073002094B60020676666660A
:10441000306E00201C6E00201F85EB51DC730020E5
:10442000CDCCCCCC6B8B002000010020B0740020E0
:10443000B47400202475002035890020BA7400204F
:10444000C0740020C474002008740020806E002016
:10445000D47300208C6B0020706F00202068FFF761
:1044600025FE60B12068FFF719FE2B7880465BB10E
:10447000013B20682B70FFF719FE0028F2D119B01C
:10448000BDEC028BBDE8F08F7549032230463AF04F
:10449000D2FC97F8101487F81384023911F0FF0149
:1044A00000F09582314432464FF6FF7312F8010B4B
:1044B0001B1A91429BB2F9D11A0A1FFA88F890454B
:1044C000CCD197F81224DBB29A42C7D1654818F0D4
:1044D000F9F92B7818442870C0E7634C94F8F53349
:1044E000012B40F21C8294F8F6136048604A4F1C7E
:1044F000194400EB8101A2FB07C25E48D1F8E090AD
:104500000178520802EB4202BA1A84F8F62329B164
:1045100059495A4A0968914200F00782B9F1000FDF
:1045200016D0574F11970DF16008A7F1120A48F8FD
:1045300020AD48F2A502152329464046A4F8F823E9
:1045400084F8FA33C847002840F0488494F8F533DB
:10455000474A0133A2FB0312520802EB42029B1AA4
:1045600084F8F53330E7474F386800283FF40AAE47
:104570004FF000098DF83890FFF798FD30B3424EA8
:10458000394C3868FFF78AFD83B27E2B00F07A84BD
:1045900072793968002A40F0698394F897C2BCF1B7
:1045A000000F00F0C5811B2B84F8972240F0658333
:1045B0000846FFF77BFD002800F05785386886F82D
:1045C0000580FFF773FD0028DBD1002010AA0EA99B
:1045D00018F02EFCD6E52D4B1B68002B3FF488AD60
:1045E000214C2B4AD4F87432EB1A93427FF780ADFA
:1045F000DFF8AC9094F87832D9F80020C4F87452FF
:104600000133900784F8783201F1BA8312F0140F65
:1046100041F08B83110794F8783215D513F0030617
:1046200012D11C4B1C49B3F9043081FB0321DB1769
:10463000C3EBA10109B2142019F00EF931461C2078
:1046400019F00AF994F8783213F0070601F03A8667
:10465000282B02F00380114B5E201B68984747E52A
:104660005155002050550020405100206C12050883
:10467000ABAAAAAA1F85002070670020E45D002075
:104680004D550020F073002000010020646E0020D2
:1046900047E80100806E002067666666F86B0020C0
:1046A0008C6B0020CC4FCD4ACD4BD4F884123868A7
:1046B0001B8892F809E0CB4A401A4FF47A71DEB2B7
:1046C00001FB0EF11B0A9677167588424FF0000623
:1046D000D37753759670167180F01484C24BC3481B
:1046E0001B68DFF850C3C24E0168DFF84CE38068F6
:1046F0009EF800E08CFB0387DB17C3EB671303F521
:10470000FA7386FB0179C91786FB00689FB2C1EB7B
:10471000A901C017B74E9776C0EBA8003F0AB64B69
:1047200011770912D7765177071296F812B082F8EE
:104730002000782147F230501EF0020F82F82170DD
:1047400083F81AB0508482F8241000F04483D6F81D
:104750000080AA49D6F804E0A94ADFF8E0A281FB6C
:1047600008704FEAE87781FB0E91C7EBA0574FEA3C
:10477000EE70C0EBA15002FB078102FB00E202EBEE
:104780004202520001EB4101029249008AFB0129D9
:10479000029A8AFB022A4FEAAA4200EB8000B6F88E
:1047A0000CA03689059200EB80000690029AACFBC3
:1047B000060607EB870707EB870776090497C817F4
:1047C000D7174FEAA94906F5FA724FEAD87803924B
:1047D00083F809808B4AA9EB0008404602FB1010C1
:1047E00016460499059A4FFA88F808EB8108D11B00
:1047F0003246029E0F4602FB1161069A9DF80C603C
:104800005E757FB207EB8207BBF1050F8CFB0029B9
:10481000DFF82CB2039E8CFB012C0AEBCA0A7A4A01
:104820004FEADE7E4FEA8A0A83F80EE01FFA88F824
:10483000A2FB0AE2BFB2BBF800E0DFF808A283F8EF
:104840000A804FEAE0704FEAE171C0EB6910C1EBFA
:104850006C114FEA17294FEA182B4FEA9212BAF857
:1048600000C083F8109083F80BB0DF734FEA162670
:104870004FEA202A4FEA21284FEA122B4FEA1E273F
:1048800034BF4FF032094FF03309187383F80DA08D
:10489000597483F812809E75DA7183F808B083F832
:1048A00013E01F7583F81B9083F81CC0C4F8805276
:1048B0002AE4DFF89481D8F80000FFF7F7FBC0B2D4
:1048C00001280ED90228514E40F0B3833379002BD2
:1048D00041F0A485D4F88832EB1AB3F57A6F81F0F1
:1048E0000C874B4E3768002F3FF440AC99F80030EE
:1048F000002B7FF413AC474BD8F800001B689B7863
:104900001E3B012B41F285853430022118F052FF05
:104910000122002389F8002084F8943224E43E4ADE
:1049200002EB8302D2F8E090F8E5DFF82091F8E599
:104930007D2B01F0788594F89A2222B180F0200333
:10494000DBB284F89AC2B4F8982294F896C21A445A
:10495000BCF1060F92B22BD804EB0C0E08460CF1FA
:10496000010CA4F898228EF85C3184F896C2FFF707
:104970009DFB00287FF405AE27E6284C227832B153
:10498000274B28491868FFF761FB00232370264F47
:104990003C78002C00F08280DFF8B4A0DAF8606088
:1049A000002E40F07F82214B3E70C3F8F05306E5A5
:1049B000D3B203EB1222FF2A86F80580A4F89822CE
:1049C00040F054810846FFF771FB1948FEE5FF22CD
:1049D0004FF6FF7371E500BF94B60020DC6B00203A
:1049E000686E0020C8740020DC730020706E002008
:1049F000676666661C6E0020F47400206BCA5F6BED
:104A0000806967FF40420F00D34D62100001002013
:104A100004740020007400206C1205088C740020BF
:104A2000207500204C740020267500204051002085
:104A30009C5200201F85EB51306E002083DE1B430B
:104A4000EC730020D8830020FC73002029AE0208FC
:104A50006C760020FEF7DEFF934B1B68C01A40F611
:104A6000B833984200F21581DFF870A29AF804304A
:104A70003A2B01F0E28400233B705AE48B4E3068FD
:104A8000FFF708FB00283FF454AC30680121FFF722
:104A9000FDFA02220023A2713B704AE4844E327870
:104AA000002A40F02181834F97F82B41002C40F0E1
:104AB000C582814B814A1B6812689A422DD897F8AB
:104AC0002031002B41F0748597F82131002B41F003
:104AD000A78797F82231002B41F0A68797F823315A
:104AE000002B41F09F8797F82431002B41F0A087DD
:104AF00097F82531002B41F0998797F82631002B44
:104B000041F0CD8797F82731002B41F0508597F879
:104B100028310824002B41F04B85694C694FD4F8AB
:104B2000F0233978684B93FBF1F313449D42FFF473
:104B300046AC664A94F8F433C4F8F053D65CF107F7
:104B400045D5DFF89C919FED628AB9F9023007EEF6
:104B5000903AF8EEE77A5F4B119367EE887A0DF1A1
:104B60006008FDEEE77AA3F13D0248F8202D17EE2C
:104B7000902A91B240F6C80223F8402C1E2203F876
:104B80003E2C4046F5F7A2FBB9F9003007EE903A0B
:104B9000F8EEE77A404667EE887AFDEEE77A17EEA0
:104BA000903A99B2F5F792FBB9F9043007EE903AD2
:104BB000F8EEE77A404667EE887AFDEEE77A17EE80
:104BC000903A99B2F5F782FB404618F0A9FEB20779
:104BD0003AD5404B404ADFF80C91118811930DF102
:104BE0006008A3F13D0248F8202D40F6C82C0822A9
:104BF00023F840CC03F83E2C4046F5F767FB0A2229
:104C0000D9F8003093FBF2F3404699B2F5F75EFB1A
:104C10000BF05AFFD9F80890109B4FEA1942591C23
:104C200010911A70109B4FEA1922591C10911A709A
:104C3000109B5A1C109283F80090109B5A1C1092E3
:104C40001870404618F06CFE730701F19586300726
:104C500001F1298694F8F4333978013393FBF1F2AA
:104C600001FB123384F8F433FFF7A9BB0846FFF7C2
:104C70001DFA00287FF485ACA7E40D2B7FF49EACD1
:104C80000846A4F89822FFF711FA00287FF479ACBF
:104C90009BE40B4AB2F8A23200210133A2F8A232FF
:104CA0003970FFF746BB00BF708B00209C8F00203F
:104CB000257500202875002094B60020248500204A
:104CC0004051002068760020A08601006476002014
:104CD00058A08B414C740020686E0020308B00205F
:104CE000806E0020706E0020954F964B0093A7F1C8
:104CF0003F014FF0C808CDE90E1707F8408C924BE2
:104D0000924A934910A8F6F711FA0E9F7B1C0E9356
:104D10003C700E9B2922591C0E911A700E9BEA22A0
:104D2000591C0E911A700E9B5A1C0E9210A883F8F3
:104D3000008039F0F7F800F1010810A942460E98FA
:104D40003AF02CF80E9A02EB080301330E9302F8A6
:104D500008400E9B5A1C0E921C700E9B5A1C0E9201
:104D60001C700E9B5A1C0E921C700E9B5A1C0E92AD
:104D70001C700E9B5A1C0E921C700E9B5A1C0E929D
:104D80001C700E9B5A1C0E921C700E9B5A1C0E928D
:104D90001C700E9B5A1C0E921C700E9B5A1C0E927D
:104DA0001C700E9B5A1C0E921C700E9B5A1C0E926D
:104DB0001C700E9B0122991818A80E911A7050F8B9
:104DC000283DDB1B3B7018F0ABFD624B3470C3F821
:104DD000F053FFF7F4BA2D22DA7667E5109B5345BE
:104DE00041F2BC84A7F1130000215F1E41F22105AE
:104DF00010F8012F81EA022212B293B2002AACBF4E
:104E00005B0085EA43039BB21A0454BF5B0085EA4A
:104E100043039BB2190454BF5B0085EA43039BB272
:104E20001A0454BF5B0085EA43039BB2190454BFC4
:104E30005B0085EA43039BB21A0454BF5B0085EA1A
:104E400043039BB2190454BF5B0085EA43039BB242
:104E50001A0454BF5B0085EA4303874299B2C7D165
:104E60004046F5F759FA3C49109D3C486D1A152DFE
:104E7000A8BF15252A4639F091FF94F8F53335700F
:104E8000FFF766BB38688DF8389084F8969284F8FE
:104E9000978286F80590FFF709F900287FF471AB37
:104EA000FFF793BB0024DFF8BC9026464FF0500874
:104EB0000BE01C44EFF3118388F31288DAF86020CA
:104EC000944218DADBB283F311881AF804B0601C3C
:104ED00059465044002217F03BFE0BF10103002815
:104EE000E7D049463A2017F095FD0BF1010B064338
:104EF000F6B25C44DEE70022DBB2CAF8602083F33E
:104F0000118850E5164B39681B78C4F88412013BB0
:104F1000012B3FF6E3AB1021022391701371FFF7D1
:104F2000DDBB0CF10103614684F8952284F89432CC
:104F3000FFF7C0F8FFF718B918F072FCFFF714B9C3
:104F40004C7400205BCB002068570508705705089B
:104F50007C5705084051002038550020208900204A
:104F60006C6C002055D90208B84B1B88DA0515D4A3
:104F7000DE0601F1BE83980601F16484590601F151
:104F80002D851A0701F19085DE0701F1938513F055
:104F9000020F0CBF4FF0040B4FF00C0BAC4AAD4BA3
:104FA00092F80090DB7809F001090BB149F0020991
:104FB000532017F023FFA84B1B8803EB830303EB5D
:104FC0008303980080B217F0FDFE002017F0FAFE70
:104FD00025F0B6FCA14BC0EB002083FB00231A1880
:104FE000C317C3EB6223FF2BA8BFFF23DEB23146FA
:104FF0003868FFF75FF89AF80030386873404BEA7A
:10500000090900218AF80030FFF754F8494638684A
:10501000FFF750F89AF80030386889EA0303DBB2EA
:1050200019468AF80030FFF745F894F8A062FFF7B8
:1050300038B918F0E5FB0123337152E48849894CF3
:1050400041F8404C18A8A1F13A0340F8203D4FF434
:10505000327321F83C3C87F82B21119118F060FC49
:10506000814BC3F8F053FFF7AAB938688DF8388040
:1050700086F80580FFF71AF800287FF482AAFFF768
:10508000A4BA7A4B94F8BEE2B3F90210B3F9002047
:10509000B3F904309FED766A84F869C107EE103ADF
:1050A000744B84F868E11B6810938EF06A0383EAFE
:1050B000031306EE902ADAB2130983F0D50343EA0C
:1050C000022383EAC2031BB283EA031AC3F307264F
:1050D0004B425FFA8AFA07EE903A86EA1A1646EAD7
:1050E0000A26F8EEE77AF8EEE66AB8EEC77A86EABC
:1050F000CA060FFA86FA67EE867A66EE866A27EEA9
:10510000067A00208AF0C806CDED127ACDED116A3C
:105110008DED137A14901590169086EA06180DF10D
:105120004009B9E80F005FFA88F8CAF3072686EA53
:10513000181646EA082686EAC806DFF83C8136B229
:10514000A8E80F0086F01E0C99E807008CEA0C1AFC
:105150005FFA8AFAC6F3072C8CEA1A1C4CEA0A2C6E
:1051600088E807000EF1010341F6FE418CEACA0C03
:10517000A8F110064FF005094FF01E0EC822A4F842
:10518000661184F8B69284F86BE184F86A2106F11E
:105190001C0184F8BE32A4F864C116F8013B83EA0E
:1051A0000C0383EA0313DBB21A0982EA1C2242EAE7
:1051B000032282EAC3031BB21FFA83FC8E42A4F8C7
:1051C00064C1EAD183F0270383EA0313DBB24FEA19
:1051D0001C2282EA131282EA032282EAC3031BB270
:1051E0009AB24FEA122EDEB2DFF890A0A4F8642142
:1051F00084F889E184F8886104F5B37904F5C3780B
:10520000D9F80000D9F80410D9F80820D9F80C30E2
:10521000D446ACE80F0009F11009C145E246EFD1D0
:10522000DFF85C80B9F80030ACF8003008F12409F0
:1052300084F80A6384F80BE318F8011F3868FEF756
:1052400039FFC145F8D1FFF7A8B800BF7C6E002038
:1052500056A50020346E0020686E002003082080D0
:105260004C740020C8057DEA40510020806E00206B
:1052700088C3E43A94B60020AC52002028540020A1
:1052800027540020DFF87C93D9F8003019229906C2
:1052900084F8B2227FF577A8D24BD34E1B789A07B9
:1052A00041F1C482B37C042B8CBF4FF003084FF054
:1052B0000208FEF7AFFBF389B168109003EB83039C
:1052C0005B00ADF85A304FF47A7033688DF85C802B
:1052D0001293B6F80CE0B27C7368ADF858E000FBAE
:1052E00001F14FF0000C4FF0FF300DF14008CDF808
:1052F00044C0149113938DF85D201590C246BAE80E
:105300000F00DFF8FCE2AEE80F009AE80F00AEE80D
:1053100007007146182221F81C39039194F8BE1237
:1053200084F86B2181F0780383EA0313DAB213095E
:1053300083F0F60343EA022383EAC2031BB283EA43
:105340000312D2B2C3F3072383EA121343EA022300
:1053500083EAC2031BB283F0C80282EA0212D2B20D
:10536000C3F3072383EA121343EA022383EAC20347
:105370001BB284F869C183F0180C8CEA0C1C5FFA2C
:105380008CFCC3F30722481C82EA1C1242EA0C225E
:1053900084F8BE02039884F8681182EACC0CC82312
:1053A00041F6FE620146A4F864C11E30A4F86621ED
:1053B00084F86A3111F8013B83EA0C0383EA031392
:1053C000DBB21A0982EA1C2242EA032282EAC30300
:1053D0001BB21FFA83FC8142A4F864C1EAD183F0B6
:1053E000180383EA0313DBB24FEA1C2282EA13128A
:1053F00082EA032282EAC3031BB29AB27B49A4F871
:105400006421DBB2120A04910692059384F88B2181
:1054100084F88A318A4604F5B37C04F5C37BDCF852
:105420000000DCF80410DCF80820DCF80C30D6466C
:10543000AEE80F000CF1100CDC45F246EFD1DCF8C1
:105440000000CEF800009DF81430DFF8BCB184F8FD
:105450000C339DF8183084F80D33DA461AF8011F22
:105460003868FEF727FE624B5345F7D1FEF7D2FAB4
:10547000D9F80030B268D6E9001C13F0140F4FF4CD
:105480007A7606FB02F601F00B825A4B1B6803EB9F
:1054900083034FEA430E94F8BEA210908AF06A0389
:1054A00083EA0313DBB2180980F0D50040EA032039
:1054B00080EAC303504A11911BB2B2F904204F484D
:1054C000CDF850E083EA0311C9B2C3F3072380FB90
:1054D000029083EA1113D217CDE912C6C2EBA002E3
:1054E00043EA0123ADF85A2083EAC1030022159252
:1054F000ADF858201EB2C446BCE80F0086F0C809BB
:1055000089EA09195FFA89F9C6F30726DDF80CE084
:1055100084F868A186EA191646EA0926AEE80F0063
:1055200086EAC9069CE8070033B283F0210686EAC2
:105530000616F6B2C3F307238EE8070083EA1613B4
:105540000AF1010143EA06232D4A84F8BE124FF006
:1055500000002B49039284F8690183EAC6062120E2
:1055600041F6FE42C823A4F864618C4684F86B01BE
:10557000A4F866211C3184F86A311CF8013B7340A1
:1055800083EA0313DBB21A0982EA162242EA0322F3
:1055900082EAC3031BB29EB28C45A4F86461ECD1CD
:1055A00083F0680383EA0313DBB2360A86EA131A30
:1055B0008AEA032A8AEAC30A0FFA8AFA1FFA8AF3E6
:1055C0004FEA13295FFA8AFAA4F86431DFF81CE085
:1055D00084F8899104F5C37384F888A104F5B3763F
:1055E000059313E0306E00201C6E0020285400202C
:1055F0004D540020DC730020806E002067666666D4
:10560000AC5200208C6B002027540020F3683068D7
:105610007168B268F446ACE80F00059B10369E42F4
:10562000E646F3D13388ACF80030049B84F80B9342
:1056300003F1230684F80AA3D94619F8011F386834
:10564000FEF738FD4E45F8D1A64A94F8BEE2A64EC4
:1056500084F868E1D2E9002311938EF0EB0383EA2A
:105660000313D9B20B0983F0C50343EA012383EA8C
:10567000C1031BB283EA0311C9B2C3F3072383EA50
:10568000111343EA012383EAC1031BB283F0C80C60
:105690008CEA0C1C5FFA8CFC4FF00009C3F3072363
:1056A000CDF8489083EA1C13109298E8070043EA6B
:1056B0000C2383EACC030FFA83F8039B84F86991E7
:1056C00088F0310C83E807008CEA0C1C5FFA8CFC34
:1056D000C8F3072383EA1C1343EA0C2383EACC03B1
:1056E00094F86CC194F86D0194F86E1194F86F21E0
:1056F0001BB28CEA030C8CEA0C1C5FFA8CFCC3F323
:10570000072383EA1C1343EA0C2383EACC030FFA32
:1057100083FC80EA0C0383EA0310C0B2CCF30723B6
:1057200083EA101343EA002383EAC0031BB2594003
:1057300081EA0111C9B2C3F3072383EA111343EAD3
:10574000012383EAC1031BB25A4082EA0212D2B299
:10575000C3F3072383EA121343EA022383EAC20353
:1057600094F870C194F8710194F8721194F873214F
:105770001BB28CEA030C8CEA0C1C5FFA8CFCC3F3A2
:10578000072383EA1C1343EA0C2383EACC031BB2EE
:10579000584080EA0010C0B2C3F3072383EA101315
:1057A00043EA002383EAC0031BB2594081EA011196
:1057B000C9B2C3F3072383EA111343EA012383EA3F
:1057C000C1031BB25A4082EA0212D2B2C3F30723CA
:1057D00083EA121343EA022383EAC20394F874C1F2
:1057E00094F8750194F8761194F877211BB28CEA3D
:1057F000030C8CEA0C1C5FFA8CFCC3F3072383EACE
:105800001C1343EA0C2383EACC031BB2584080EA02
:105810000010C0B2C3F3072383EA101343EA002346
:1058200083EAC0031BB2594081EA0111C9B2C3F334
:10583000072383EA111343EA012383EAC1031BB25E
:105840005A4082EA0212D2B2C3F3072383EA121348
:1058500043EA022383EAC2031BB283F0270C8CEADB
:105860000C12D2B2C3F3072C8CEA121C4CEA022CA5
:105870008CEAC20C0FFA8CFC1FFA8CF34FEA132946
:105880000EF1010E5FFA8CFC312040F6FE41C82279
:1058900084F8BEE2A4F8643184F86B01A4F86611C0
:1058A00084F878C184F86A2184F879913068F368C3
:1058B0007168B268B6F810E006F5C1760FC6049BB1
:1058C000A6F800E003F1130884F8FAC284F8FB920A
:1058D0001BF8011F3868FEF7EDFBD845F8D1FEF73D
:1058E00052BD00BF706F0020A65200208C4A8D4B25
:1058F0001178D3F800900A2384F8AF32002900F021
:10590000D486894B01291A88079241F2E3815A888B
:105910000492022900F09C879A880592032901F0DD
:10592000D381DA880392042901F0C98105291A89F3
:1059300001F0C1810629B3F80AB001F0B981072945
:10594000B3F80C8000D0DE89069224F0F9FF94F8B9
:10595000BEC2DFF8D8E1CDF840908CF0300383EA86
:105960000313DBB2C0EB002019098EFB002E81F07F
:105970007A01079A84F868C141EA03214FF00009CF
:1059800081EAC30362F30F09059A0FFA83FA86448A
:10599000C3170020C3EB6E2362F30F00069AFF2BA0
:1059A0004FF0000162F30F01A8BFFF23002268F34C
:1059B0000F029846049B8DF8558063F31F49039BA3
:1059C00066F31F4263F31F406BF31F41CDE9119053
:1059D000CDE913128AEA0A1E5FFA8EFE0026CAF388
:1059E000072A8AEA1E1A8DF854600DF14009B9E8B9
:1059F0000F004AEA0E2888EACE0E0FFA8EFE8EF0CD
:105A0000C80ADFF82C8184F869618AEA0A1AA8E8D2
:105A10000F005FFA8AFACEF3072E8EEA1A1399E87E
:105A2000030043EA0A2383EACA031BB248F8040BC3
:105A300083F0230E8EEA0E1E5FFA8EFE4046C3F3FD
:105A4000072282EA1E1242EA0E2220F8141982EA84
:105A5000CE0E0CF1010C4FF0230841F2FE62C82378
:105A600084F8BEC2A4F864E184F86B81A4F86621CE
:105A700000F1160184F86A3110F8013B83EA0E0345
:105A800083EA0313DBB21A0982EA1E2242EA0322E6
:105A900082EAC3031BB21FFA83FE8842A4F864E1C2
:105AA000EAD183F0F40383EA0313DBB24FEA1E2248
:105AB00082EA131282EA032282EAC3031BB21FFAAC
:105AC00083F95FFA83FED4F86A11D4F86E21D4F812
:105AD0006601D4F87231DFF85CC0A4F86491ACE8D8
:105AE0000F00D4F87601D4F87A11D4F87E2184F826
:105AF00082E14FEA1928ACE8070084F8838104F2B8
:105B0000E72604F2053984F8058384F804E316F8DF
:105B1000011F3868FEF7CEFAB145F8D1FEF72BBC6D
:105B20001C67002094B6002082E400200308208037
:105B3000AC52002028540020A34B1B6803F008023D
:105B4000002A4AF60B4048F6034149F607484BF64F
:105B50000F4204BF8846024613F0040F18BF904658
:105B600098069A4B1B7848BF48F480484FF01901BB
:105B700048BF48F02008022B84F8AE1240F2DF85BF
:105B800064204FF0FF3B4FF0000A94F8BEC2CDF8FE
:105B900040808CF0F10383EA0313DBB21E0986F028
:105BA000E706C8F3090246EA0326CDE9118286EA30
:105BB000C3064FF0000936B2ADF84EA0ADF850B0B4
:105BC0008DF85E00ADF84C90CDF85290CDF856901F
:105BD000CDF85A9086EA061E0DF14008B8E80F008D
:105BE0005FFA8EFEC6F3072686EA1E1646EA0E26E2
:105BF00086EACE06DFF8E4E184F86991AEE80F00AA
:105C000098E80F0036B286F0C80888EA08185FFAEC
:105C100088F8C6F30726AEE8070086EA181646EAB3
:105C2000082181EAC80109B22EF8023B81F0010681
:105C300086EA0616F6B2C1F30722714682EA161208
:105C40001B0C01F81E3942EA06224FF0010E82EACF
:105C5000C60641F6FE70C8220CEB0E03A4F86601DE
:105C600084F86BE184F86A2101F11F0084F868C1AF
:105C7000A4F8646184F8BE3211F8013B734083EAF2
:105C80000313DBB21A0982EA162242EA032282EAED
:105C9000C3031BB29EB28142A4F86461ECD183F0CD
:105CA0007C0383EA0313DBB2320A82EA131282EA2C
:105CB000032282EAC3031BB29AB24FEA122EDEB26B
:105CC000DFF81CA1A4F8642184F88CE184F88B61CE
:105CD00004F5B37904F5C378D9F80000D9F80410B5
:105CE000D9F80820D9F80C30D446ACE80F0009F1F7
:105CF0001009C145E246EFD1D9F80000CCF8000008
:105D0000DFF8E08099F804308CF8043008F12709B6
:105D100084F80D6384F80EE318F8011F3868FEF765
:105D2000C9F9C145F8D1FEF71EBB0021302017F09C
:105D300093FD94F8783213F003067EF485AC244A80
:105D4000D4F87412234B91421B6804D983EAE3769A
:105D5000A6EBE37636B2204BF71783FB0623C7EB9F
:105D6000631739B2102017F077FD642101FB17612A
:105D700009B2212017F070FDD9F80020FEF74ABCC7
:105D8000DFF864802427A8F12806B38AF8EC016ABA
:105D900007EE103AB8EEC77A3846C6EE877A013772
:105DA000FFB2FDEEE77A17EE903AC3EB431103EB37
:105DB0008103D90009B217F04FFD272FE5D1D9F89B
:105DC0000020FEF723BC00BF8C6B00206C6C002011
:105DD0003F4B4C00DC7300201F85EB51AC52002080
:105DE0002854002027540020880B0010954B1B6876
:105DF000052203F014019B0684F8B72240F15F846A
:105E0000914BDFED927A9A8907EE102AB8EEC77AA5
:105E100027EE277A002900F036868D4BDFED8B6A5E
:105E2000D3ED007AF8EEE77A67EEA67A94F8BEA290
:105E3000884B894AB3F90410B2F90620874E884886
:105E40008DED117A8AF0220383EA03135FFA83FC53
:105E50004FEA1C13B2F5FA6F83F05903A8BF4FF451
:105E6000FA6243EA0C2383EACC03B2F57A7F1BB2D1
:105E7000B8BF4FF47A72A2F57A7E83EA031C6422DB
:105E80005FFA8CFCC3F3072302FB0EF283EA1C1EAD
:105E9000A6FB023280FB0130CB174FF0000B4EEA1D
:105EA0000C26C2F38F12C3EBA0030DF14008CDF80E
:105EB00040B0CDF84CB0CDED127A86EACC06ADF804
:105EC0005220ADF85030C346BBE80F0036B286F022
:105ED000C80C8CEA0C1C5FFA8CFCC6F30726DFF8B2
:105EE00098E1DBF800B084F868A186EA1C16AEE8F9
:105EF0000F0046EA0C2686EACC031BB283F04A0662
:105F000086EA06117046C9B2C3F3072282EA11126B
:105F100042EA012240F810B982EAC1060AF1010AF8
:105F20004FF04A0E41F2FE4C0022C8230390014676
:105F300084F8BEA2A4F86461143084F86BE1A4F87C
:105F400066C184F8692184F86A3111F8013B734015
:105F500083EA0313DBB21A0982EA162242EA032219
:105F600082EAC3031BB29EB28142A4F86461ECD101
:105F700083F0140383EA0313DBB2360A86EA1316AE
:105F800086EA032686EAC30636B21FFA86FC354B3C
:105F9000D4F86A11D4F8660104934FEA1C2ED4F8A1
:105FA0006E21D4F87231A4F864C1DFF8B8C0B4F837
:105FB0007EB184F881E1ACE80F00D4F87601D4F822
:105FC0007A11ACE80300F6B204F2E72AACF800B0AC
:105FD00084F8806184F80263D34684F803E304F212
:105FE00003361BF8011F3868FEF764F85E45F8D1E8
:105FF0001D4B1E4A1B781278013B12F00100DBB2E8
:1060000014BFC0224022172B03D819490B4493F820
:10601000C890184B19888E071ABF002342F010024F
:10602000012311F0080F18BF022311F0100F18BF41
:10603000062311F0200F18BF1023002840F0E4833E
:1060400003211BE08C6B00201C6E00200AD7233C30
:10605000DC730020806E002082E40020D34D6210AB
:106060006766666628540020EC66002056A500206E
:106070006C1205087C6E0020AC52002094F8BE62C1
:10608000109386F0460383EA0313D8B2030983F022
:10609000920343EA002383EAC0031BB283EA03109E
:1060A000C0B2C3F3072E8EEA101E4EEA002E8EEA0F
:1060B000C00E0FFA8EFE8EF0C80383EA03134FF072
:1060C000000CDBB20320CEF3072E8DF844908DF840
:1060D00045C08DF846208DF847108DF848008EEAAF
:1060E000131E98E807004EEA032E8EEAC3031BB284
:1060F000DDF80CE084F86BC183EA0318AEE8030016
:106100005FFA88F8C3F3072383EA181343EA0823E6
:1061100083EAC80394F86C8194F86D0194F86E11C9
:106120008EF800201BB288EA030888EA08185FFA94
:1061300088F8C3F3072383EA181343EA082383EAA2
:10614000C8031BB2584080EA0010C0B2C3F3072353
:1061500083EA101343EA002383EAC0031BB25940C9
:1061600081EA0111C9B2C3F3072383EA111343EA99
:10617000012383EAC10394F86FE194F8708194F8E5
:10618000710194F8721194F8732184F869C11BB2FB
:106190008EEA030E8EEA0E1E5FFA8EFEC3F307230D
:1061A00083EA1E1343EA0E2383EACE031BB288EA76
:1061B000030E8EEA0E1E5FFA8EFEC3F3072383EAF8
:1061C0001E1343EA0E2383EACE031BB2584080EA33
:1061D0000010C0B2C3F3072383EA101343EA00237D
:1061E00083EAC0031BB2594081EA0111C9B2C3F36B
:1061F000072383EA111343EA012383EAC1031BB295
:106200005A4082EA0212D2B2C3F3072383EA12137E
:1062100043EA022394F87481DFF830E484F868617B
:1062200083EAC2031BB288EA030282EA0212D2B2F4
:10623000C3F3072383EA121343EA022383EAC20368
:106240001BB283F0320282EA0212D2B2C3F30723F6
:1062500083EA121343EA022383EAC2031BB29AB20F
:1062600040F6FE10C8214FEA122C84F86A11DBB206
:106270000136A4F86601DEF8000084F8BE6284F8F6
:1062800076C184F87531A4F86421DEF80410DEF8D4
:106290000820BEF80C90049E0EF5C17EAEE8070003
:1062A00010368EF80280AEF8009084F8F8C284F8B8
:1062B000F7321AF8011F3868FDF7FCFEB245F8D135
:1062C000FEF775B8FF2016F081FA002800F0B282C0
:1062D0000378FF2B00F0BA8290F90110022017F02A
:1062E000BBFAFF2016F072FA002800F08E810378C6
:1062F000FF2B00F08A81B0F90C30C549C54A897D71
:1063000003EB830303EB830349089B0093FBF1F347
:1063100082FB0312D917C1EBA20109B2BE4E0320C2
:1063200017F09AFA7379002B40F01B82D9F80030ED
:106330009A0640F1CD81B94FB94E3B789B0700F1E9
:106340008E820021012017F087FA0021092017F022
:1063500083FA318A94F87822B37CB1F5967F08D914
:1063600002F00F02072A04D842F20F738B4228BFB3
:106370000B46DFF8DC8298F80720CAB1203B07EE15
:10638000903A9FEDA87AF8EEE77AF6EE006A67EEAB
:10639000877ABEEE007AF5EEC07AF1EE10FA58BFB9
:1063A000B0EE667A77EE877AFDEEE77A17EE903AEE
:1063B00019B2052017F050FA3A7800239207CDE978
:1063C0000E3300F1288294F87C32012B00F02382F6
:1063D000B8F90030DFED946A07EE103AB8F90230F0
:1063E00007EE903AB8EEC77AF8EEE77A27EE267A0B
:1063F00067EEA67ABDEEC77AFDEEE77A10A88DEDBE
:10640000107ACDED117A17F03FFA94F87832FEF752
:106410001FB90221FDF73AFEFEF77ABAC4F8885296
:106420003771FEF75EBA084684F89A82FDF73EFEA1
:1064300000287EF4A6A8FEF7C8B89AF802105046C5
:1064400024F08AFF00287EF416AB784B1868FDF71D
:106450002DFE00287DF468AF744B754E1868754C9E
:106460004146FDF713FE9AF80330039396F8079020
:1064700094F8A43202930423B371B9F1000F00F031
:106480001D8396F808806C4BDFF8C8A108F101085D
:106490005FFA88F808EB480903EB89095FFA88F38B
:1064A000092B41465046337208F1010800F2D383AC
:1064B000F4F7FEFE28B999F80830FF2B09F10C0912
:1064C000ECD1327A5D4B06924FF00C0909FB023990
:1064D000DFF87081D9F844100591084637F022FDA5
:1064E000D9F8483004935FFA80F9184637F01AFD5E
:1064F0005FFA80FB069A059909EB0B00083088F8D3
:10650000070022F00F0088F80A0002F00F020BEBE0
:10651000C90088F80D2088F80E004A4608F10F00DF
:1065200038F03CFC049B08F1060A09F10900194601
:106530005A46504438F032FC98F8073003F1010E07
:10654000C3B1013B08F1070CDFF80C915CFA83FC46
:106550005046002310F8012F5A409300D10883EAD7
:10656000420301F01801534049FA01F253408445B7
:10657000DBB2EFD10EF80A30039830F0F9FDF37971
:10658000013BDBB2F37113B92D4B1B780293274B00
:1065900098F8022018682B49FDF758FD03239DF851
:1065A000082084F8A422B3713B70FDF7C2BE072413
:1065B000254B97F82A2111930DF16008A3F13901B9
:1065C000A3F1400648F8201DC821101D03F8401C07
:1065D0004FF4E4734EF67D2170707180404602FBEB
:1065E0000471B380B471F3F74FFE109B721C9B1AB9
:1065F0007370404617F094F93B190E4A002183F856
:106600002011C2F8F053FDF7DABE002186E600BF84
:10661000C4CD0020676666666E6C0020306E002078
:106620001C6E0020E4380E3F0050C3479C8F0020B2
:106630000001002040510020B01205086C1205082E
:10664000F8730020DCDA00204C740020A6520020F1
:10665000DC6B0020F47300200007090EB44AB54B30
:106660001768B54EA3FB07239B0BA6FB0321490923
:10667000C1EB0111A3EB8103190209B2002317201A
:1066800084F8783217F0E8F8AC4BA3FB07239B099A
:10669000A6FB03125209C2EB0212A3EB820319B24A
:1066A000182017F0D9F8FDF7D6BF88468B460A4662
:1066B0000391CDE9041107910E46FFF745B99FED0F
:1066C000A07A00297FF4A9ABF0EE477AFFF7AEBBC2
:1066D0001B077FF59AAE9B4B93E8030010AB83E852
:1066E0000300184617F0D0F88FE601230293FDF758
:1066F000A1BD4FF0340BFEF751BC0123D8F80000C8
:106700003371FDF7CBFC0646D8F80000FDF7C6FC58
:1067100077067EF4E6A88A2800F0A4818E287EF40D
:10672000E0A899F80030002B7DF4F5AC864E874B3D
:1067300033602D2384F88C323768FEF7D7B8844A4B
:1067400053799279002B40F05681002A40F07C82E8
:10675000924664204FF0FF3BFFF717BA0021FEF787
:106760007FBBDFF8108298F80030002B40F0628188
:10677000784F19461A460620A4F87A2217F06CF8CA
:10678000754AB4F87A0292F808C0398898F800304F
:10679000D27A0130BCF1010FA4F87A0200F0228114
:1067A00001EB81018FB212B10BB197FBF3F74FF000
:1067B000640A3A20B7FBFAF80FFA88F117F04CF8A0
:1067C0000AFB187189B205310A233B2091FBF3F1D2
:1067D00009B217F041F8B379002B3FF4A7AD5F4F32
:1067E0000A223B6893FBF2F3282019B217F034F821
:1067F0003389002B40F04D81B96881F3100109B253
:10680000042017F029F891E55549C97800290CBFF3
:106810000421052132E4D6E9002301210EA884F8E1
:106820007C12CDE90E2317F02FF8EEE54FF00108AA
:10683000FEF73FBD014651E5B368642000FB03F05D
:10684000FDF719BD4FF0240BFEF7A8BB314645E517
:10685000B046B346324603960596FFF775B8B18940
:10686000404B4FF4F368112008FB01F191FBF3F169
:1068700009B216F0F1FFB389642108FB03F393FB1F
:10688000F1F393FBF1F201FB123109B2192016F07A
:10689000E3FF3B78B16898077FF553AD09B251E546
:1068A000B646FEF7F8BD304B304E11930DF160083F
:1068B000A3F13D0248F8202D41F2C811022203F84D
:1068C0003E2C23F8401C40463168F3F7E7FC404675
:1068D0007168F3F7E3FCB389242101FB03F140461F
:1068E0000A23053191FBF3F189B2F3F7EFFCF38949
:1068F00003EB8303590089B24046F3F7E7FC1C4BD6
:106900001B78990740F1CD80B368642193FBF1F1C6
:1069100001F57A7189B24046F3F7D8FC109BB27C3E
:10692000591C109140461A7016F0FAFFFEF792B902
:1069300094B6002073B2E74589888888D34D6210E9
:1069400000000000A812050804740020C87400208C
:106950006E6C0020686E0020DC6B0020706E0020E2
:10696000346E0020A08601004C7400201C6E0020B4
:10697000306E00206E6E0020B94B1193A3F14008D9
:106980002122C820A3F13D0123F8400C88F8022001
:10699000109135F0DDFCB34BB349B44A1B88002895
:1069A00008BF1146580578D4DA0700F18180B04A53
:1069B00013F0020F18BF114610A8F3F755FC109BF7
:1069C000AC4A591C109100211970109B9B1A10A8F9
:1069D00088F8013016F0A4FFFEF739B94FF0100B1C
:1069E000FEF7DCBA12B10BB191FBF3F109B2392019
:1069F00016F032FFEFE6A04B1B8803EB830303EB9B
:106A000083034FEA830A1FFA8AFA002A00F06A8198
:106A10009A4BB3F900B00AF057F840B2FFF7B5B897
:106A20000124C5E50324C3E50224C1E50524BFE52F
:106A30000424BDE5904FB4F87A02398890FBF3F254
:106A40004FF0640C03FB12020CFB013192B25B00AD
:106A5000B1FBF3F10B0243EA0213C1F303210B4331
:106A600019B288E6864B1B689E067DF53AAF99F809
:106A70000030002B7DF44FAB824E834B33602D23CF
:106A800084F88C3258E6D3ED027AF8EEE77AFFF715
:106A9000CDB90AF019F801B2B2E67C498CE70624B8
:106AA00086E54FF47A7136E74FF0200BFEF776BAA1
:106AB000774981E74FF0080BFEF770BA6E4B6F4ACB
:106AC000588853680493734B92680A92B3F9042070
:106AD00071490892B3F902200792B3F90020069297
:106AE0000A680299DFF8C0810B9001F0F003844638
:106AF00003F110010498DDF808B0099288F80A3013
:106B0000664ACBB20CFB00FC08F10D0A6420059329
:106B10009CFBF0F00C905846059B83424ED90C2309
:106B200003FB0021431E91F84CC04CEA00118AF887
:106B300000100AF10101082B00F28380DFE803F066
:106B40007F7D7B79777573710500002394449CF8F1
